:020000040800F2
:1000000000A00020053E01086D3E0108392E0108C0
:100010006D3E01086D3E01086D3E010800000000C4
:100020000000000000000000000000006D3E01081C
:100030006D3E0108000000006D3E010857BA00083F
:100040006D3E01086D3E01086D3E01086D3E0108E0
:100050006D3E01086D3E01085D8800085988000862
:100060006D3E01086D3E01086D3E01086D3E0108C0
:1000700055F200086D3E0108C38A00086D3E010874
:100080006D3E01086D3E01086D3E01086D3E0108A0
:100090006D3E01086D3E01086D3E0108558800085F
:1000A00049FD000885FD000839FD0008A9FD00088C
:1000B00079FD000869FD000859FD00086D3E010842
:1000C0006D3E01086D3E01086D3E01086D3E010860
:1000D0006D3E0108CDFF0008C1FF0008B5FF000814
:1000E00065BA00086D3E01086D3E01086D3E0108CD
:1000F0006D3E01086D3E01086D3E01086D3E010830
:100100000000000000000000000000006D3E01083B
:100110006D3E01086D3E01086D3E01086D3E01080F
:100120006D3E01086D3E01086D3E01086D3E0108FF
:100130006D3E01086D3E0108000000000000000057
:100140006D3E01086D3E01086D3E01080000000093
:10015000000000000000000000000000000000009F
:1001600000000000000000006D3E01086D3E010827
:100170006D3E0108000000000000000000000000CB
:08018000000000006D3E0108C3
:100188002DE9F04F2DED028B6A4F6B4B3B60AFB002
:1001980000237B6010F063FB18B910F083FB0BF0B1
:1001A80039F90BF0F1F9654A654C137843F001030E
:1001B8001370644B4FF47002C3F88820002309932E
:1001C8000A93236843F480332360236803F40033DD
:1001D8000A93099B013309930A9B1BB9099BB3F541
:1001E800A04FF2D1236813F4003318BF01230A93F8
:1001F8000A9B012B68D0534E534BF360636ABB6074
:10020800636ADFF874B1DFF87481DFF874A143F032
:1002180080736362636943F4FC032EAD6361032357
:100228008DF86A3041F6FF7325F8503D4FF0904045
:1002380029460FF0FFF84FF6FF7358462946ADF8E8
:1002480068300FF0F7F8414829460FF0F3F84048B6
:1002580029460FF0EFF83F4829460FF0EBF82946FA
:100268003D480FF0E7F828460CF074FD1A9B3B4A0E
:10027800B3FBF2F33A4A3B4913603B4B00221A6046
:100288005A603A4B5960F02186F823109A60384E2C
:1002980007221A60B368CAF8003098E80300636957
:1002A80085E8030043F4802363610823CBF8183002
:1002B8001A981BA90FF0BEF8DAF8003013F0080FEF
:1002C800A8F10C0829D163E02A4B12221A6063684E
:1002D800636063686360636843F480636360636852
:1002E80023F47C136360636843F4E8136360236852
:1002F80043F0807323602268114B9001FBD55A6844
:1003080022F003025A605A6842F002025A60636897
:1003180003F00C03082BFAD16DE796F89231012B04
:1003280036D8044B96F893219B6813F0805900F057
:10033800D3852DE00001002087AC000800340020A0
:100348000010024000ED00E00005FA050008004832
:10035800000C0048001000480014004840420F00FC
:10036800441F00203F190100481F002010E000E052
:10037800202C00200020024000040048CC83010803
:10038800FC270020BD4B002283F893210BF098FA3C
:1003980064200BF052FBBA4800214FF48C7215F020
:1003A80046FEE369B74843F00703E361A36943F4F2
:1003B800E123A361636943F4C023636100F5887492
:1003C800837B416890F80FE003F00702DB0801EB3C
:1003D80083039200196A4FF00F0C0EFA02FE0CFA12
:1003E80002F221EA02021A62196A10304EEA010288
:1003F800A0421A62E4D10022A349002353540132D7
:10040800112AF9D1A14AFF2199540133072BF9D1B7
:100418009F4BDAF800409F4A1A609F4800213C220F
:1004280015F005FEC4F3801905234FF0000E9B4A12
:1004380099481EF802100C2202FB0EF21154B9F171
:10044800000F07D11E3901299FBFFF2103F1FF3398
:100458001154DBB20EF1010EBEF1050FE7D1904A3F
:1004680096F805B013708F4B8F4983F800B08F4B07
:100478007B62C0330B608E4B8E4A03EBCB03A10625
:100488005B7848BF0123936200238B4A40F2DC511A
:1004980022F813100133082BF7D113A800211C22CE
:1004A80015F0C5FD14F4007A1DBF844B199503930C
:1004B800CDF80CA0BBF10E0F03D00BF0EF03082B07
:1004C80002D101238DF85E30022007F061FA18B1DD
:1004D8004088003018BF0120C4F340038DF8523023
:1004E800C4F340338DF84C30C4F3C03300F001003E
:1004F8008DF84F3014F400638DF851008DF8549046
:1005080007D096F8863103F1FF3EDEF1000343EB96
:100518000E038DF85030C4F300438DF85530BB6A94
:10052800B6F84801ADF862001AF1000A18BF4FF09A
:10053800010A003318BF01238DF85730C4F3005364
:100548008DF85830B6F84A31ADF85C30B6F8563107
:10055800ADF85A3004F00101C4F38043C4F3C0027B
:10056800E40448BF45488DF85330B6F8543144BFC9
:10057800B0F85001ADF86200B3F5FA7FADF860301D
:1005880084BF0023ADF862304D4896F8D63187F81D
:100598002C30002387F82D3043709DF85E308DF89D
:1005A8004D10002B8DF84E208DF856A00CBF00235F
:1005B800022301B902B1013308EB83084FF00009A7
:1005C800D8F81430A3F1020A203304933AF8023F12
:1005D8004FF6FF72934200F0B1819DF85110DAB2E4
:1005E8001B0ADEB279B12748364C00EB021041688D
:1005F800A14208D10189B1F5806F00F09B81B1F566
:10060800006F00F097819DF8541031B111011D4819
:1006180040582D49884200F08D819DF8551079B1D8
:100628001101184C6018645828498C4200F08281E6
:100638004168B1F1904F03D1817B082900F07A819C
:100648009DF8521051B10F4800EB02104168B1F10A
:10065800904F03D10189102900F06C819DF84F104B
:10066800B1B30848174C00EB02104168A1422FD1E2
:100678000189042900F05E812AE000BF202C0020B7
:10068800941F002040A601080C0100201D01002035
:1006980014230020102E0020182300207BAE010810
:1006A800CD1000204009002028210020342C0020F3
:1006B80020AC01080001002038100020C083010888
:1006C8002D0100200004004800040040002C0140D7
:1006D8009DF8501051B1BE4800EB02104168B1F1CD
:1006E800904F03D10189202900F02481199C7CB105
:1006F800B74F216807EB02177868884208D1398913
:10070800A088884200F01681E088884200F01281B3
:10071800022B02D19DF84C3003E0012B04D19DF847
:100728004D30002B00F006819DF85710A84B17019B
:1007380059B19DF85E1041B9A2F10E01012904D802
:10074800D959A448814208BF04269DF85810DC19DD
:1007580031B19DF85E1019B9043A032A40F2D280EB
:10076800012E49D1DFF878820693D919FF2291F832
:100778000DE088F8742088F875204868C8F8844027
:1007880001F108020989ADF868104FF0000B022149
:100798008DF86B1088F878B01AA98DF86AE0059280
:1007A80088F830B0C8F834B0C8F838B0C8F83CB0E9
:1007B800C8F870B088F876B088F877B00EF03AFECE
:1007C800069B059AD85991785A4608F0BDFB2046F1
:1007D800594632460FF03AFB7F4BC8F888307F4BBA
:1007E800C8F88C30C8F890B0204608F1880108F1A4
:1007F8008C020FF081FB9DE0022E4BD15FFA89F34A
:100808001C2101FB03FC764BCDF81CC003EB0C0B41
:1008180001238BF8783006936D4B8BF87990D919B2
:100828004FF0000891F80DE048688BF87A8001F1E4
:1008380008020989ADF868108BF882801AA9CBF8EC
:1008480084408DF86AE005928DF86B600EF0F2FD39
:100858005F4B059AD8599178424608F075FB069B7C
:1008680020461A4641460FF0F1FA5D4BDDF81CC0F0
:100878005C4ACBF8882003EB0C015B4ACBF88C2050
:100888008831CBF8908020460A1D0FF035FB09F11E
:1008980001094FE0032E33D19DF85330504E534F8A
:1008A8003BB196F82E80204608214FF6FF720023B0
:1008B8001AE0BDF8602096F82E80BDF86230B2F5D7
:1008C800FA7F0BD94A49B1FBF2F22046082192B2CD
:1008D8000EF0D9FD474B47F828000AE04649B1FB1E
:1008E800F2F22046012192B20EF0CDFD434B47F8BB
:1008F8002800C36096F82E30013386F82E3019E0B0
:10090800042E17D1364EBDF85A2096F82D703A4B62
:1009180093FBF2F22046BDF85C30012192B20EF052
:10092800B2FD96F82D3006EB87070133C7F858015A
:1009380086F82D30049B9A457FF448AE284F304BFB
:1009480097F82D2087F878212E4A1678A6F11702F5
:100958000024022A1C709E461BD87B6A2344D3EDD0
:10096800007AF5EE407AF1EE10FA03D1BB6A002B5B
:1009780050D126E0244A04EB020C0FCB8CE80F0080
:100988009EF8003010340133C02C8EF80030E4D1CA
:10099800ECE71E4B13F836808EF8008003EBC60395
:1009A800D3F80490B9F1000FE0D04445DEDA164AD6
:1009B800230103EB020C4B440FCB01348CE80F00EE
:1009C800F3E7134B1A6812F4805F984648D141E068
:1009D80040A60108004001409DF000087DF1000894
:1009E80000010020E1F1000875F00008601F0020F8
:1009F80000127A009DF1000840420F008DF10008B6
:100A0800901F0020400900207C08002020AC01082D
:100A1800FC2700202B4B2C4A13F83600107003EBF0
:100A2800C6035C68002CCCD000238342C9DAC3EB30
:100A3800C3016218DFF89C80D2F8009041F8089052
:100A480001EB080C9188ACF8041092798CF8062018
:100A58000133EAE706F0EF03082B1C4B20D121E015
:100A68009EF80020012AF5D9194B03EB0212103227
:100A780010339342EED053ED047AB6EE007A67EE67
:100A8800877A43ED047A53ED057A67EE877A43ED6A
:100A9800057A53ED037A67EE877A43ED037AE7E741
:100AA8000E2E08D11A7842F010021A70182E13D19F
:100AB8000BF026FA10E01A7822F010021A70192E9C
:100AC800F5E700BF40950108B42000201011002070
:100AD80084080020B52000200BF0F6F9D8F8003083
:100AE800B14CB24E580358BFB14BB2485CBF01225B
:100AF8001A70B14A137843F0040313704FF400439B
:100B0800ADF8683063694FF0020943F400234FF0F1
:100B1800010B8DF86B9029468DF86AB063610EF071
:100B280089FCA64BA64A1A6000200AF0A5FFE369D3
:100B380043F48043E361236943F480432361636999
:100B480043F480236361736A23F470037362736AE6
:100B580043F4A0037362736A23F070637362736A69
:100B680043F0A0637362736A23F070437362736A1D
:100B780043F0A0437362736A23F470237362736A49
:100B880043F4A02373624FF460431A938DF86C907A
:100B980003234FF00009304629464FF4805A8DF858
:100BA8006D3004938DF86E908DF86F900CF044FAC8
:100BB800049B8DF86D3030462946CDF868A08DF835
:100BC8006CB08DF86E908DF86F900CF035FA236943
:100BD80043F480432361236923F480432361794BE1
:100BE8009A8822F480521204120C9A809A8892B23F
:100BF80042EA0A029A801A8802F4415242F4457283
:100C080042F003021A809A8822F470621204120CCD
:100C180042F4E0629A809A8B22F400621204120C69
:100C28009A8307221A821A8892B242F040021A80E6
:100C3800C6F818A0D8F8003003F41073B3F5107F85
:100C480000F09E80604B614E1E606369DFF85C9126
:100C580043F480236361E36943F40013E361236B86
:100C680023F010032363236B43F010032363D9F8A5
:100C7800203023F07063C9F82030D9F8203043F0D1
:100C88008063C9F82030D9F8203023F07043C9F8C0
:100C98002030D9F8203043F08043C9F820304FF095
:100CA80000084FF0020C4022484629464FF0030B3B
:100CB8008DF86CC0CDF818C01A928DF86E808DF83A
:100CC8006F808DF86DB00CF0B7F980224846294640
:100CD8001A920CF0B1F93268DFF8089122F001029B
:100CE800326031683A4A0A4032603A4A32613268C0
:100CF80042F001023260C6F80880C6F80C80C6F8D7
:100D08000880B26842F40042B260326832607268A9
:100D180022F0784222F400427260326842F0010206
:100D28003260D9F800502C4E05F400434FF0100AF9
:100D38000493524605F4006330464146059315F086
:100D480076F94FF6FF72DDF818C00E9215F002051D
:100D58008DF83DC08DF83E808DF83F808DF83CB011
:100D680042D02EA94FF0904041F880AD0CF064F9C4
:100D780001250723357086F80180F370B57033E0DC
:100D880016490A784B4616481E561F2E02BFFF26E4
:100D98001E5402F1FF3203F10C0308BFD2B23C2B00
:100DA800F1D10A704EE700BF00100240000400486D
:100DB800A80D00200008004800340020103400204E
:100DC800DDB800080038004004100020005400403E
:100DD800FFE0CF007A25E00080230020CD1000201E
:100DE80018230020FC270020049B7BB12EA9042394
:100DF80041F8803D92480CF01FF90C23337107230A
:100E0800F371012375711D44B371EDB2059B83B174
:100E18002EA9202341F8803D4FF090400CF00CF9AA
:100E2800022333730723F373012375731D44B373CC
:100E3800EDB2E36A834823F4F873E362E36A43F4A8
:100E4800D873E362636943F0805343F0020363613C
:100E58000BF02FFE1AA80BF001FE7B4B1A937B4B6D
:100E68001B93012D4FF0000394BF1A4680221F9256
:100E78004FF48072734C20924FF4806221922022AA
:100E8800204622921AA94FF400521C931E932392D3
:100E98002493ADF874500BF0EEFD236843F0010382
:100EA80023606B4CA36823F04053A360A36843F00E
:100EB8008053A3600A200AF0C0FDA36823F0804392
:100EC800A360A368A360A36843F00043A360A2687B
:100ED8005F4B002A31DAFAE7531E092B3FF658AA6E
:100EE800D8F858002860294658460EF0A3FA4FF45F
:100EF8000063CBF818303C200AF09FFD96F8933138
:100F08009945BFF63FAADFF838B108224FF40063CD
:100F1800CBF8182078200492ABF8283003930AF015
:100F280081FD049A039BABF828207820CBF8183071
:100F38000AF078FD09F10109E0E79A68454922F0CD
:100F480040529A609A6842F000529A608868424A11
:100F5800024042F468328A60D968404A0A4042F442
:100F68000052DA601A6B013D22F00F0215431D632F
:100F78000021012372189078002800F084805C1CFE
:100F8800042B16F801E0D278DFF8C4C0E4B20ED81A
:100F980003EB4303DCF830505B001F20984025EA40
:100FA80000000EFA03F30343CCF8303031E0092B8C
:100FB8000ED80620053B4343DCF834501F209840E8
:100FC80025EA00000EFA03F30343CCF8343020E09E
:100FD8000E2B4FF006050ED8A3F10A006843DCF883
:100FE80038801F23834028EA03050EFA00F32B43B9
:100FF800CCF838300DE00F3B05FB03F0DCF83C8003
:101008001F23834028EA03050EFA00F32B43CCF88C
:101018003C30BEF1090F0E4822D983698569AEF1CB
:101028000A0303EB43034FF0070E0EFA03FE25EA0B
:101038000E05856185699A402A43826122E000BFD6
:10104800000400480804024040010050902300209A
:101058000001005000030050E010FCFF07C0FFFD36
:10106800436945690EF1FF3303EB43034FF0380E34
:101078000EFA03FE25EA0E054561456903339A40D9
:101088002A4342612346043110297FF473AFBB4BD6
:101098009A6842F001029A601A461168B74BC9076C
:1010A800FBD5DA6822F00202DA60DA6842F002025E
:1010B800DA60DA6842F00102DA609A6842F0040203
:1010C8009A60AF4AB2F85C319046002B41F07480C8
:1010D800B8F95E21002A41F06F80B8F96021002A32
:1010E80041F06A80D9F800309B031FD5C8200AF068
:1010F800A4FCAE2009F0B1FC08B109F0B3FCA14C86
:1011080087F87901C8200AF098FC9F4BC7F87C3112
:1011180000210C22204614F08AFF0223E3700CF011
:10112800A6FD0AF065FC994B0344A360984B9948C7
:101138001B68B8F86461B3F8563098F863B198F84A
:101148006B4198F86C51049300210C22B8F80C906C
:1011580098F80FA014F06BFF8F4B069318460021E8
:10116800142214F064FF8D4A0592002111708C49F5
:10117800C7F880110EF0C7FD059A8046002832D0C6
:10118800069B88491960884959608849D960B6F52D
:10119800807F87491961874B01D1002116E0BB2E5A
:1011A80001D9012112E0612E01D902210EE0292E78
:1011B80001D903210AE0132E01D9042106E0092EE2
:1011C80001D9052102E0002EE7D006211970042379
:1011D8001370794B02221A70784A136843F001039E
:1011E80013605B460EE003200AF09AFC40E24FF0E1
:1011F800010B0BFA03F140F2B2320A4042B1012B63
:101208005FD900236E490022092B0A70F9D8EEE74E
:1012180011F04D0FF3D0624A0593C7F880210EF004
:1012280072FD059B0028EAD0062168200A460DEBCE
:1012380000030EF015FA9DF86D1001EA0B029DF8F7
:101248006B1001EA0B0101FA0BF343EA82019DF8E6
:10125800692002EA0B030B430AD05BB25B4501D15C
:10126800002302E0022B0ED1012387F8843111E01C
:101278000EAB68200C215A460EF0F2F99DF8383072
:1012880013F00F0303D105200AF04AFC02E0042BF7
:10129800EAD1E5E73F4B4B4A1A604B4A5A6097F848
:1012A8008421002A0CBF6F226E221A72444B04223A
:1012B8001A70414B03225A70404A136843F00203E4
:1012C8001360042D00F2D080DFE815F00500EB0074
:1012D8009800050098000A200AF0AFFB7720A021AB
:1012E80001220EAB0EF0BCF9002800F087801E2109
:1012F800012277200EF030FA4FF42F600AF092FBAB
:101308004FF0000BABF160010025C9B202221AAB05
:1013180077208DF868508DF869500EF0A1F99DF886
:1013280068209DF86930294943EA022301F5C37210
:101338002BF802300BF1020BBBF1100FE2D1B1F820
:10134800942102F00F0E02F47F42A1F894210120AB
:101358002B462946DFF874C021F001056544B5F82D
:101368008651002D18BF002011F0010F03D0EDB2F7
:101378006B4008252CE083EA1523FAE700010050AA
:10138800202C002078240020AA2D0020404B4C005F
:1013980048100020802800202C2100204021002017
:1013A800E4830108E9FB000859FA0008D9FA0008A3
:1013B80090C1793D00000020880000200C11002019
:1013C8002C34002061FC000899FA00080001002074
:1013D80013F4004F18BF83F4C053013D4FEA430391
:1013E800F6D101311029B5D16E4942EA0E02A1F8B1
:1013F800942118B9C3F303339E4538D0694D95F845
:1014080096B1BBF1000F40F0C68614200AF015FB18
:1014180005F297137620D02101220EF021F995F8D4
:101428009731582B3DD105F5CC73882118227620A9
:101438000EF016F931227620F4210EF08DF90123F1
:1014480085F89631584B594A9A60594A5A6045F678
:10145800D8125A80574ADA60574A1A61574AA3F88D
:1014680000B05A6100F097BE012D13D119E04E4B20
:1014780042F210721A805A80514A5A60514A9A6050
:10148800514ADA60514A1A61514A5A61B8F1000F5B
:10149800B4D003254F4B504A9D70136843F00403A2
:1014A80013604D4D2B689B0702D54C4B1B68984722
:1014B8004B4ABAF1000F25D016F0FF0F0AD12B685E
:1014C80013F0020F4FF07D0140F2712308BF4FF473
:1014D800FA7302E04FF47A731946994505DBB9F5BA
:1014E8007A6FA8BF4FF47A6900E099464B1E4B44C7
:1014F800B3FBF1F3013BDBB203FB011187F8B43115
:10150800116004E0274BC2F8009083F8B4A1354B72
:101518001B689847344A0023022C1370914604D064
:10152800032C20D0002C40F039862EAB002203F883
:10153800502D2E4AC7F8B8211E200A2101220EF08C
:101548008FF880B19DF86830482B0CD1284B294A78
:101558001A60294A5A60B8F1000F04D0042389F8A8
:10156800003002234EE02EAB002603F8506D0C200D
:10157800314601220EF074F880B19DF86830482B8E
:1015880040F042861A4B1D4A1A601D4A5A60464668
:10159800B8F1000F00F03886032333E0064600F068
:1015A80033BE00BF0001002070060020F9A100082A
:1015B800FBA10008CBA3000869A40008FB9F000852
:1015C80007FA000849FA0008FDF9000839FA000886
:1015D8003DF80008880000200C1100208028002019
:1015E800A82800202C21002028340020FC83010892
:1015F8004C060020D9A50008D5A3000841A500087D
:10160800B5A40008B84AD3702B6843F008032B60D0
:10161800B64B93F858210AB1B5490A7093F8592185
:101628000AB1B4490A7093F85A310BB189F80030FD
:101638002B68B14913F0080F00F0B685BDF910000A
:10164800DFEDAE6A642290FBF2F302FB130212B2E2
:1016580007EE902AB8EEE77A07EE903AF8EEE77AC6
:10166800E7EE267AB2EE047A67EE877AC1ED007A61
:10167800A34A137843F002031370A24B08229A611D
:101688000A24A04DAB8A9BB283F00803AB821920D1
:101698000AF0D3F901200AF0EFF919200AF0CDF980
:1016A800013C00200AF0E8F914F0FF04E9D108230E
:1016B800AB61954B1A6812F0080F984605D0934B0A
:1016C8001B689847924B01221A70924B9FED928AA1
:1016D8001B68924C1B7B00EE103AB8EEC00A20EE55
:1016E800080A09F099FD238807EE903AF8EEE77AA0
:1016F80027EE800A14F0AAFE894B9FED8A7A18809B
:101708002388894C07EE903AF8EEE77A874BC7EEC4
:10171800277A2046FF211A229FED857AC7EE877A1D
:101728009FED847AC3ED007A834BD3ED047A834B23
:1017380067EE887A67EE877AC3ED007A14F077FC53
:1017480000222270D8F800207D4B012112F0020FF0
:1017580018BF617019701FBF032119700221A17091
:10176800550748BF1978204641BF4C1C1C700324FC
:10177800445412F00A0F0CD01A7804218154511CD9
:10178800C9B205244454D11C0232D2B219700621C0
:1017980081546C4D29688C0641BF1A78541C1C7002
:1017A800072448BF84540A0608D51A7809248454A3
:1017B800941C0132D2B21C700A2484544B4E7479A2
:1017C800082C01D00E2C04D11A78571C1F700B2737
:1017D80087541A7811F4803F4FF00C0E00F802E09D
:1017E80002F101071CBFDFF858E10232FFB21F7097
:1017F8001FBF8EF800204C4A4FF00E0E02F807E08B
:101808004A0741BF1A78571C1F70102748BF8754D2
:101818001A78571CFFB24FF0120E11F4806F1F7028
:1018280000F802E00ED096F81CE2BEF1000F09D0D5
:10183800DFF80CE102328EF800203B4A4FF0130E1D
:1018480002F807E01A7811F4007F4FF0140E00F840
:1018580002E002F101071CBFDFF8E4E00232FFB248
:101868001F701FBF8EF800202F4A4FF0150E02F888
:1018780007E0182C0DD11A7816278754571CFFB289
:101888004FF0170E00F807E0D71C0232D2B21F70D3
:1018980084540C0341BF1A78511C1970192348BF8E
:1018A800835400219822284814F0C1FB0AF0B1FFA4
:1018B800264B274A27491A6000234B800B7126497B
:1018C8000A60B6F8982190B2244921F81300013330
:1018D800122BF9D12B68D8045CBFB6F89E0108809A
:1018E8001B0740F100813BE088000020202C0020ED
:1018F800402100202C340020701A00208988883C60
:1019080000340020000400480C1100204C06002080
:1019180064060020D421002035FA8E3C20000020E7
:10192800F02100200AE81C4111100020880700203F
:1019380000401C46BD3786352C210020D0210020D0
:1019480010100020FC27002070220020E40E002048
:10195800AA2D0020340E0020142C00203828002046
:1019680096F89241062C00F2B880DFE804F00407EC
:101978000E3D5878780045F2F05201E042F6F82220
:10198800804B1A800AF0E2FFA6E007EE902ADFED0E
:101998007E6A7C4BB8EEE77ADFED7C7AE7EE267A52
:1019A80042F6F82119800023FCEEE77A784A17EE10
:1019B800901A42F823100133122BF7D1754A764951
:1019C8001160764A4020137006F0BCF8002800F039
:1019D800848001234FF0070990F90000704A8DE8D0
:1019E800080240216F4B72E0664B42F6F8221A80DB
:1019F800684B6D4A1A60694B102240201A7006F035
:101A0800A1F8002869D001234FF0000C90F90000DC
:101A1800664A8DE8081040214FF4E13357E0594BEE
:101A280042F6F8221A805B4B614A1A605B4B082227
:101A380040201A7006F086F800284ED001234FF097
:101A4800000E90F900005B4A8DE8084040214FF4F1
:101A5800E13305F04DFF584BC3F8BC0139E0494B61
:101A680056485749DFF888C1DFF888E142F6F8227E
:101A78001A804A4B534A0C271F70062C4FF000035C
:101A880003700B7013700AD01B238CF800304E4B78
:101A98008EF8007005221A704FF4E13407E0212314
:101AA8008CF80030484B8EF800701C70474C394B4E
:101AB800474A1A60402006F045F870B10123002714
:101AC800444A90F9000040218DE88800234605F03B
:101AD8000FFF003018BF012028B9082009F060FC6A
:101AE8002C4B3D4A1A602B682C4A13F4804F1FBFB9
:101AF800082111702749394818BF086042F20101CE
:101B0800194003F0010003F4005479B11D4944F66B
:101B180020670F8024B1082111701E49304C0C60D9
:101B280020B10C2111701B492E4808601178180645
:101B3800A1F10401517040F196801F482A4CDFF84A
:101B4800B890C0F8C09100273946152200F5E27018
:101B5800DFF8A8A067706760A76014F068FAA9F1B9
:101B680005033846CAF8003006F090FB1F4B0220E8
:101B78001B68E36005F0E6FF002841D1802009F0EA
:101B88000FFC68E0E8070020CDCCCC3F0000B0C4D3
:101B9800242B00203C000020B12A01080C2300203F
:101BA800592C0108A08601009D2A0108AD2B0108C7
:101BB800892A0108612B010800010020102C00204F
:101BC80049220020482200206C22002090D00300E7
:101BD800F5C6000809C70008112B0108E52A010805
:101BE800012B0108F12A0108A40700202028002061
:101BF8006B2200200F2C0020102E0020C40700208C
:101C080047796378CE490C2202FB03125278BA4214
:101C180004D00133DBB2042BF4D900236370DAF863
:101C2800003062781B7890F90000002B4FF00C030D
:101C380003FB021314BF0327012700225B780097D8
:101C48000192022105F054FEBE4B1860002895D081
:101C5800012006F01BFBBC4B1868BC4B00F5C57295
:101C68001A6006F0C1FB2B6813F4007F1AAF59D035
:101C7800B74C039B2360B74BB7485A6942F480229C
:101C88005A619A6942F001029A61039B1B88ADF878
:101C980030304FF0010902230CA98DF833308DF84C
:101CA80032900DF0C7FB2368AB485B88ADF8303045
:101CB8004FF0000A0CA98DF832A00DF0BBFB236889
:101CC8004846197A0AF06EFF236858680AF0BAFE87
:101CD80023685B681A93384610238DF86D308DF8A9
:101CE8006CA08DF86E900FF093FA23685B7A8DF8EC
:101CF80038300EA803238DF839308DF83AA08DF8C6
:101D08003B900FF067FA954B954A1B683C3B136074
:101D1800D8F8003043F01003C8F80030914B4FF06A
:101D2800FF321A60904A914B1360914ADFF8608243
:101D3800803313602B680024D90388F8004040F1F1
:101D4800BC800EF0B5F9DFF84CC2DFF808A2CDF878
:101D580014C040F22A334FF001091A466046214662
:101D6800049388F8009014F062F9DAF81420DFF888
:101D780028824FF0904042F40032CAF81420426A98
:101D880022F00F024262426A032142F006024262D6
:101D98004FF4807B02228DF835100CA98DF8342081
:101DA80003928DF83640CDF830B08DF837900BF0AF
:101DB80043F9DAF81810039A41F40061CAF81810C8
:101DC800B8F8001021F45C710904090CA8F8001097
:101DD8001D21C8F82C104046A8F828200EA9A8F8FC
:101DE80030406022C8F814900E92ADF83E4010942E
:101DF800ADF84440ADF84640ADF84840ADF84A402B
:101E0800ADF83C900AF068FFD8F8182042F00802B4
:101E1800C8F81820D8F8442042F40042C8F84420F2
:101E2800DAF8142042EA0902CAF81420AAF6E47A79
:101E380050460AF03EFE38460AF010FE049B4D4A12
:101E4800ADF874308023DDF814C01A923946102298
:101E58001F9350464FF40053CDF86CC01C92239347
:101E68001E94CDF880B02194229424940AF003FEA5
:101E7800D8F80C3043F40073C8F80C30DAF80030A6
:101E880043F00203CAF800300BA80C238DF82C305D
:101E98008DF82D908DF82E408DF82F900FF09AF92F
:101EA8002146354B1A68354B43F82120013120294A
:101EB800F7D10DF0E1F90DF0DFF92B685A0540F183
:101EC80090802F4C2F4BD4F80495C3F80090042031
:101ED80005F038FE0421C4F8080505F00FFE2A4B6A
:101EE80084F80C050820C3F8009005F02BFE274B5A
:101EF800DFF8A8801860082105F000FE002184F8AA
:101F08000D052C22404614F092F88E2388F80130F3
:101F18004FF07C0BE0234FF07D0A88F8033088F8F7
:101F280000B088F82BA0DFF878802C2200214046EA
:101F380014F07DF88A2388F801301020A02331E0BE
:101F4800988401087424002048100020380F0020CD
:101F5800A0070020001002400004004820280020AC
:101F68009C07002068100020E01100204C2E002063
:101F7800B8240020342C014014840108AA0D002044
:101F8800000100200011002058110020A411002099
:101F9800A90D0020D9020020002C014028110020A2
:101FA8005D11002088F8033088F800B088F82BA06D
:101FB800C4F8109505F0C6FD1021C4F8140505F005
:101FC8009DFD84F818052020C4F81C9505F0BAFD7D
:101FD8002021C4F8200505F091FD84F824050BF0B4
:101FE8001DFD8D4A138823F040031B041B0C13802E
:101FF800138823F038031B041B0C138013889BB22F
:1020080043F04003138000249F2332208DF838309A
:102018008DF839408DF83A408DF83B4009F00DFDB8
:102028008DF869407D4C4FF480580422A4F828802C
:1020380038460EA90FF098F8C4F818809DF86A2061
:102048009DF86930120242EA03429DF86B301A4348
:10205800734B9A42734B17D008D873498A420CD0F5
:1020680001F51A4102318A4209D01CE06F498A42BF
:1020780005D001318A4207D015E0202200E08022F5
:102088001A804FF4807202E04FF480721A805A80EE
:102098009A88198812029A604A43DA60644A0121D0
:1020A80082F8251504E000221A805A809A60DA60C6
:1020B800DC680CB3240CA1464FF0000AA24514DAE0
:1020C8000AEB04084FEA68084FEA0840394610222C
:1020D80008F074FC002357F82320013268D101333B
:1020E800042BF8D1C1464446E8E706F049FB504BBB
:1020F8004FEA0942C3F828252B684E4A13F40023F7
:1021080018BF0123137009F073FC4B4B18607379E7
:10211800052B02BF494B4FF4C8721A80484B4FF445
:102128007A721A80474BC8221A80474A137843F0BC
:1021380008031370454A137823F0020313702A68C2
:1021480040F6020313406BB1414B42491960424BC0
:1021580003211970414B01211970414900230B805B
:1021680040490B80930341BF3F4B04221A71DA7830
:1021780044BF42F00102DA70B3682B603B4B012286
:102188001A703B4A137863F07F0313702FB0BDECCD
:10219800028BBDE8F08F0425FFF77CB9012C7FF690
:1021A80037AA1C46FFF7B6B900230B60FFF760BAE1
:1021B80008F1010AA04696E71BB207EE903ADFED58
:1021C8002D6AB8F95E312C4AF8EEE77A07EE103A34
:1021D80067EEA67AB8F96031CDED1A7A07EE903A33
:1021E800B8EEC77AF8EEE77A002127EE267A67EE8E
:1021F800A67A11701AA821498DED1B7ACDED1C7AAB
:1022080009F012F8FEF76EBF012C7FF601AA002430
:1022180089F80060FFF789B90038004000040048D9
:1022280018BA200010000020152020001740EF00E9
:1022380000010020A42800202C0E00209C21002052
:102248002634002020340020101100202A340020D9
:10225800F81000209C2D00205C1100208000002038
:10226800D80F0020DA0F002078240020A80D0020C5
:102278000034002035FA8E3C700000205C230020DA
:10228800874A2DE9F04F1368864C03F59C432033A9
:102298002DED028B2360A3880133A380824B19683C
:1022A80089B011F4804F0592019305D110F06EFDAD
:1022B80010B9237B0133237300277C4BDFF804829A
:1022C8001E78FDB2AE4230D9D8F800307748072DD5
:1022D80098BF595D764B88BF29461B689847032DE0
:1022E8001ED8D8F8002005F10E0302EB8303998865
:1022F800DA88A8B14FF47A73401A5843531A90FBFE
:10230800F3F040F6C90300F57A70984205DC40F214
:10231800EE239842B8BF184601E040F6CA0080B2E2
:1023280004EB45050137E881C7E70F23277B84F8CD
:102338003230032594F83330B7FBF5F505EB450546
:102348007D1B029394F834300393D8F800A0DFF88B
:102358007CB1EBB204930025B54255DA5549029B8E
:1023680031F815904FEA450853B910F00FFD28B120
:10237800039B002B08BF4FF0000901E0DDF808902F
:10238800BAF81400484503D8BAF8160048450ED2E2
:10239800E8B210F0D1FC032D8146DFBF94F832E09B
:1023A8000120A8402EEA0000D8BF84F8320010F0BF
:1023B800EDFC18B1404828F8009021E0049B94F8FF
:1023C8007E002BF8139028B9022F15D93549012022
:1023D80081F87E00BBF80210BBF800000844BBF887
:1023E80004100844354980B228F8010000B20321DE
:1023F80090FBF1F080B200E048462F4928F8010030
:1024080001350BF1060BA7E794F83250254BA5F1DF
:102418000F0EDEF1000545EB0E0584F898503DB12E
:102428009A8811B21429CCBF143A00229A800BE082
:1024380083F83350B54207DAE8B210F07DFC1E4B42
:1024480023F815000135F5E7019B1B68DF0405D566
:102458001B4B1B68DE0701D40FF010FF059B1968A2
:10246800184B1868837A9BB3013B134D027B35F8F0
:1024780013301AB1C3F53B6308339BB21BB2A3F503
:102488007A73B3F57A7FA8BF4FF47A7323EAE373BC
:1024980007EE903A9FED0C7AF8EEE77A51E000BF2C
:1024A80008340020300E0020FC2700200C230020D8
:1024B8003C0000203E0E002038280020B00E0020EE
:1024C8000C100020142C002000007A44660E002016
:1024D800019A1268150440D5D4F89C20AD4E8A1A8A
:1024E800002A3ADB01F59C422032C6F89C20AA4A11
:1024F800C07A5579A94A32F8152096F8A0500135C6
:1025080092B292FBF0F205F00F0086F8A00030447A
:1025180080F8A1201A46A248185C01330244102B07
:1025280092B2F8D112B292FBF3F31BB2642BA8BF9C
:10253800642323EAE37307EE903A9FED9A7AF8EE64
:10254800E77AC7EE877A984A9FED987A67EE877A96
:10255800FCEEE77A17EE903A1380019B944D1B68C6
:10256800DFF8708213F4807F7AD0924B994204D9B5
:10257800237A13B9874B01221A72B4F904E098F848
:102588000060844BBEF1140FCCBF4FF0000E4FF02B
:10259800010EC6F38006BEF1000F03D000279F721C
:1025A8005F7200E00327A07AD4F8B4B0D4F8B8C0BA
:1025B800B4F90490617AE3882A88032848D8DFE8C8
:1025C80000F0020E1B35BEF1000F02D02A80002257
:1025D8002AE0002E40F05A862A80A6723AE09CF83B
:1025E800000000EB8000814502DC2A8001221BE00C
:1025F80001206EB300F0D8BE3EB1BBF80E206A8051
:10260800AA80BCF80200E88002279CF800A09CF889
:102618000100504400EB8000814500F33A86002E0B
:1026280000F037862A800222A27213E02A80032251
:10263800A2726172E3807EB198F8003043F0020321
:1026480088F80030534B00225A720FF017FE03E04F
:102658002A80A0726172E38017B1384609F026FA21
:10266800554EB6F8520110F0C3FB834668B910F016
:10267800E5F9524BC3F800B0C3F804B0C3F808B08A
:102688004F4B00221A605A609A6098F800305A0737
:1026980036D5019B1B68DB0632D54A4B1B78DF0613
:1026A8002ED4494B1B7893B196F8DE31BBF1000F5D
:1026B80015D17BB1454B1A68D4F8BC309B1A002B56
:1026C80008DA0FF0DBFD334B83F8C0B018E0BBF13C
:1026D800000F0DD1102009F0E9F901230EE03BB1FC
:1026E8003A4A12684FF47A7101FB0323C4F8BC30EC
:1026F80094F8C03023B109F0C5F9002384F8C0303C
:10270800002296F8DCA196F8DD11B6F89A71B6F8B1
:102718009CE1134635F912009B08B842C4BF63F028
:102728007F03DBB201327045B8BF43F04003042A8F
:10273800F0D194F8C12017489A4205D190F8C220E8
:10274800F92A04D8013200E0002280F8C22084F877
:10275800C1301D4B0F4A18781D4F994600283ED1AD
:102768003B68D80709D5BBF1000F38D198F800307D
:10277800DB0734D50FF0E4FB31E098F80030580758
:102788002DD592F8333053B3537A43BB21B30FF0AE
:1027980075FD24E0300E00208023002090230020C7
:1027A800D10E00200000C8426C10002000C07F44F9
:1027B80038280020404B4C00202C0020A019002075
:1027C8005C1A0020101100200C0000202028002096
:1027D8000C1000202A340020BBF1000FD7D094F849
:1027E800C2307C4ADFF818B2142B40F0928099F876
:1027F80000301AF1000A18BF4FF0010A7BB392F8B3
:10280800C1305F2B12D198F8003003F0040303F0B5
:10281800FF0113B10FF032FD08E00B200391029283
:1028280009F044F9029A039982F8C210BAF1000F2C
:1028380015D094F8C1307D2B11D198F8003003F0F1
:10284800040303F0FF0213B10FF018FD07E00B209B
:10285800029209F02BF95F4B029A83F8C22098F88C
:10286800003003F0040303F0FF01002B51D194F86A
:10287800C130584A572B16D1574B4FF47A721A80E9
:10288800019B1B68190601D505F010FE534B1B6808
:102898005A0742BF524A0A21118013F0080338D15F
:1028A800504A138035E001980068400716D55A2B26
:1028B80014D14D4B187820B119704C4B01221A7065
:1028C80027E092F8C33083F0010382F8C3300BB1DC
:1028D8000C2000E00D2009F0E9F81AE05D2B00F06B
:1028E800DB845B2B00F0F8845E2B02D1032000F020
:1028F800F4BC562B01D108F0E3FF99F80030002B07
:1029080000F0008594F8C1306F2B40F0F5840FF08B
:1029180017FB019B1B68580733D594F8C330A3B144
:1029280098F80030590710D5B5F90620B6F89A314D
:102938009A420ADD3B6813F0010301BF2C4A322199
:102948001180244A08BF82F8C3303B68DA030AD5ED
:10295800284B1A782AB9244A127812B9244A322103
:10296800118001220CE0204A137853B198F8003006
:1029780003F0040303F0FF011BB91C4B1170012283
:102988001A70DBF8009000233B6009F17B0609F11F
:10299800CB0A3278737816F8010C9A420BD231467A
:1029A80008F0C6FF38B116F8022C012303FA02F228
:1029B8003B6813433B6004365645EAD10E4B1B78FF
:1029C80003B30E4E054F336813F0020F40F04183F6
:1029D80039E300BF300E0020263400200C110020FF
:1029E80020340020E8100020C9210020CA2100203E
:1029F800B0210020C82100202D3400200C10002018
:102A08004810002009F1CA0609F5897732787378E9
:102A180016F8010C9A4225D2314608F089FF08B30E
:102A2800B37896F804E0C04A96F80390BF480C21A2
:102A3800013B01FB0E4103EB43031344D1F8C820CB
:102A48009A420FD0C1F8C830002390F8F420C1F89A
:102A5800CC30012303FA0EF322EA030381F8C49071
:102A680080F8F4300636BE42D0D1B14BDFF8CCB294
:102A78001E68B04B1B68039394F83330049300230B
:102A88000293DBF80030002B00F0D48293F800901A
:102A9800B9F1000F00F0CE82DBF8042003998A1AFE
:102AA800002A0CDB01F5FA720299CBF80420012206
:102AB8008A4094F8F41021EA020284F8F420049A77
:102AC800002A00F0B7821BF8042C59780432D2B2DD
:102AD800002940F0718235F91210974A934FB2F8E5
:102AE800982102F1C800814202DD93F802A015E0A6
:102AF800C83A914203DA9978C1F1000A0EE0029AC5
:102B08000123934097F8F42022EA030387F8F4306E
:102B1800039B03F5FA73CBF804308BE297F8F43093
:102B2800029A1341DB0700F18582BAF1000FCCBF8E
:102B38000220012008F0DCFF09F1FF33132B00F21B
:102B48007082DFE813F0140021002F0043005C00BE
:102B58006300CA004001A701D70107026E024300C3
:102B680052006300CA0040019A00120177013778C9
:102B78005744FA2FA8BFFA2727EAE7773046377075
:102B880008F0BCFE01200BE077785744642FA8BFFB
:102B9800642727EAE7773046777008F0AFFE02200F
:102BA8003946D4E196F80390D144B9F1640FA8BF2F
:102BB8004FF0640929EAE97986F803903046D7F896
:102BC800F81004F0C5FF03204946C0E1717951446B
:102BD8006429A8BF642121EAE17171710D2008F010
:102BE800F3FEB9F10D0F00F01C82317951446429CC
:102BF800A8BF642121EAE17131710E20A7E1B17902
:102C0800514481F30801B1710520A0E1D7F8FC30E7
:102C18001A78022A22D107EE90AAF8EEE77AB2EEE5
:102C2800040A87EE800AD3ED097A30EE270AB5EE5A
:102C3800C00AF1EE10FA09D4DFED427AB4EE670A61
:102C4800F1EE10FAC8BFB0EE670A01E09FED3E0A48
:102C580083ED090A0F2008F0A2FE0AE09978514492
:102C6800C829A8BFC82121EAE17199700F2008F08E
:102C7800ABFEB9F10F0F00F0D481D7F8FC301A7809
:102C8800022A20D107EE90AAB8EEE78AB2EE040A2B
:102C980088EE008A93ED080A38EE000AB5EEC00AFD
:102CA800F1EE10FA09D4DFED277AB4EE670AF1EEF7
:102CB80010FAC8BFB0EE670A01E09FED230A83ED62
:102CC800080A12206BE159785144C829A8BFC821C5
:102CD80021EAE1715970122039E1D7F8FC301A78ED
:102CE800022A33D107EE90AAB8EEE70ADFED157A8B
:102CF80093ED0C7A80EE270A30EE070AB5EEC00A8B
:102D0800F1EE10FA07D4B4EE670AF1EE10FAC8BF74
:102D1800B0EE670A01E09FED0C0A83ED0C0A102063
:102D280008F03DFE1DE000BF90880108300E00202D
:102D38007010002020280020202C0020F80E0020F1
:102D480000007A440000C84200000000197B51448A
:102D5800C829A8BFC82121EAE1711973102008F019
:102D680033FEB9F1100F00F05C81D7F8FC301A7807
:102D7800022A1ED107EE90AAB8EEE78A5FED0F7A15
:102D880093ED0B0A88EE278A38EE000AB5EEC00AE2
:102D9800F1EE10FA07D4B4EE670AF1EE10FAC8BFE4
:102DA800B0EE670A01E01FED180A83ED0B0A132045
:102DB800F5E0D97A5144C829A8BFC82121EAE171B0
:102DC800D9721320C3E0D7F8FC301A78022A22D12E
:102DD80007EE90AA1FED260AF8EEE77A87EE800A3A
:102DE800D3ED0F7A30EE270AB5EEC00AF1EE10FAED
:102DF80009D45FED2C7AB4EE670AF1EE10FAC8BF79
:102E0800B0EE670A01E01FED300A83ED0F0A1120CA
:102E180008F0C5FD0AE0997D5144C829A8BFC8211A
:102E280021EAE1719975112008F0CEFDB9F1110F71
:102E380000F0F780D7F8FC301A78022A20D107EE84
:102E480090AA1FED410AB8EEE78A88EE008A93ED52
:102E58000E0A38EE000AB5EEC00AF1EE10FA09D4EF
:102E68005FED487AB4EE670AF1EE10FAC8BFB0EE2B
:102E7800670A01E01FED4C0A83ED0E0A14208EE06C
:102E8800597D5144C829A8BFC82121EAE171597563
:102E980014205CE0D7F8FC301A78022A20D107EE1B
:102EA80090AAB8EEE78AB2EE040A88EE008A93ED9B
:102EB8000A0A38EE000AB5EEC00AF1EE10FA09D493
:102EC8005FED607AB4EE670AF1EE10FAC8BFB0EEB3
:102ED800670A01E01FED640A83ED0A0A09205EE033
:102EE800D9785144C829A8BFC82121EAE171D9700D
:102EF80009202CE0D7F8FC301A78022A1ED107EEF8
:102F080090AAB8EEE78A5FED717A93ED0D0A88EE24
:102F1800278A38EE000AB5EEC00AF1EE10FA07D497
:102F2800B4EE670AF1EE10FAC8BFB0EE670A01E026
:102F38001FED7B0A83ED0D0A0A2030E0597B5144CE
:102F4800C829A8BFC82121EAE17159730A2008F0ED
:102F58003BFD66E0D7F8FC301A78022A22D107EE4A
:102F680090AA1FED890AB8EEE78A88EE008A93EDE9
:102F7800100A38EE000AB5EEC00AF1EE10FA09D4CC
:102F88005FED907AB4EE670AF1EE10FAC8BFB0EEC2
:102F9800670A01E01FED940A83ED100A0B2008F080
:102FA800FEFC3EE0D97D5144C829A8BFC82121EACA
:102FB800E171D9750B20CAE7012932D1987835F922
:102FC8001230B3F5617F05DB40F633029342A8BFA8
:102FD800134601E04FF46173B9F10C0F21D14FF49E
:102FE800966292FBF0F0AD4AA3F5617393FBF0F3A0
:102FF800DFB21378BB4214D0042F34BF3B46022300
:103008001370A74A09FB0323A64A0633136008F086
:1030180097FA4846394608F0D7FC781CC0B208F041
:1030280067FDA149029A0123934091F8F4201343C4
:1030380081F8F430029B0133042B02930BF10C0B43
:103048007FF41FADBDE4019B1B68DD050FD5637AD6
:103058006BB13B6898070AD5944B1B8813F00105A0
:103068000AD10FF0EBFC012008F08AF904E00120F6
:1030780008F075F9012300E00023326851070DD5E7
:1030880063B1012008F06BF9884B1B889A0708D4B4
:103098000FF0D4FC022008F073F902E0022008F0D7
:1030A8005EF93B6813F00A0F26D03368DB060BD5B0
:1030B8007E4B1B885D070AD4042008F061F97C4B1D
:1030C8001B88A4F8003102E0042008F048F93368AE
:1030D800980607D5754B1B88590606D4402008F07A
:1030E8004FF902E0402008F03AF933685A0642BF27
:1030F8006F4B1B88A4F802313B689B0608D43368E1
:103108001F0540F18F804FF4807008F039F98DE089
:10311800684B664F1B7813F0020F50D0664B1B7834
:10312800042B4CD93368DFF8809113F4007A0ED061
:103138003B88DD0637D4102008F022F9202008F05B
:103148000EF95E48011D05F005F9022327E03D88C8
:1031580005F01005ADB22DB1102008F000F90125D9
:1031680089F804A13368580512D5D9F808315449AB
:103178005A89B1F90030002BB8BF5B42934207DA95
:10318800B1F90230002BB8BF5B429342C0F2128102
:103198003B88990608D5202008F0E1F8002389F833
:1031A8000431012500E0002594F80C31B3B90E2054
:1031B80008F07CFC3C4B012283F80C210EE03B8894
:1031C80003F03003002B9AD0102008F0C8F8202014
:1031D80008F0C5F8002384F8043101E0002D8ED0F2
:1031E800384B002003F1280503F15004364A00212A
:1031F80022F81010354A596022F81010043269601C
:1032080022F8101000221A609A602A60AA602260D0
:103218006160A26014331435143400287FF46FAF52
:103228000120E3E74FF4807008F099F8284B5A79A9
:10323800082A1C4601D00E2A02D1402008F08FF837
:10324800019B1B685A0540F1CA8094F81C3223B9C7
:1032580098F8003013F0040F02E0336813F4002FDD
:103268000BD01C4B00221A703C2009F0B7FB002839
:1032780000F0B5800EF086FBF6E70AF0CFFB09B048
:10328800BDEC028BBDE8F04F09F0C3BA0120FFF78F
:1032980094B90320FFF791B901201EE060280020AF
:1032A800D033002070100020300E0020D4110020F0
:1032B800E8100020101100201611002078100020BE
:1032C800F0100020400F002022340020B80F00200A
:1032D800202C00201123002002205FFA80F909F138
:1032E800FF3386F8B43708F095F808F04DF94846EA
:1032F80008F0FEFBFFF70DBBBAF1000F02D07E2BE2
:103308003FF405AB94F8C130972B05D1364B4FF4F9
:10331800C8721A80FFF7FDBAA72B06D1334A137873
:1033280043F004031370FFF7F4BA0022BB2B079293
:1033380001D1022303E0B72B04D14FF6FE73ADF899
:103348001E3009E0BE2B01D1022303E0BD2B1AD1A8
:103358004FF6FE73ADF81C30DBF80030BDF81C10DA
:10336800B3F858200A44A3F85820BDF81E10B3F843
:103378005A200A44A3F85A2008F0A2FA002384F835
:10338800C230FFF7C6BA792B04D1194AD37823F093
:10339800010306E07A2B7FF4BCAA154AD37843F0E0
:1033A8000103D370FFF7B5BA013301469BB202207F
:1033B800FFF703B93B889B063FF5F6AE202007F0E0
:1033C800DFFF0C480C4B011D1A685B684360026004
:1033D80004F0C0FF094B012583F80451E4E609B065
:1033E800BDEC028BBDE8F08F9C210020101100205D
:1033F800782400208010002018110020300E0020B2
:103408002DE9F04FC14BB3F90610C14B2DED028BDE
:103418001F687A8989B0914201930EDBB1F5FA6F82
:10342800FC79BDBF8B1A6343A2F5FA64C4F1640446
:10343800BCBF93FBF4F4643400E06424B54AB64B93
:10344800B2F898A192F962211868049092B2059294
:10345800054600220293AD4B33F912300393CAEBB1
:10346800030303F2F31640F2E63086424FEA420BBA
:1034780003D8002BB8BF5B4201E04FF4FA73022A6D
:10348800049E4FF064002FD096F811E1BEF1000FB2
:1034980004D07345CCBFCEEB03030023DFF8C0E2B2
:1034A80093FBF0FC6FF063093EF81C809B4E09FB10
:1034B8000C390CF1010C3EF91CE00FFA88FCCCEB3E
:1034C8000E0E0EFB09FE9EFBF0FEC64426F80BE02E
:1034D800BE1836797343924E93FBF6F364339BB26E
:1034E800634393FBF0F02EE096F812E1BEF1000F73
:1034F80004D07345CCBFCEEB03030023DFF84C8226
:1035080093FBF0F06FF0630C0CFB003938F910E016
:103518000130002B38F91000CEEB000000FB09F950
:10352800BDF8140099FBFCF9CEEB090919FB00F969
:103538007A48A0F80490B879B8BF5B42434378480A
:1035480093FBF0F064306B78764E4FF0640E434393
:1035580093FBFEF3B354744EEB7A434393FBFEF3B1
:10356800B3546B7D6D4E5843704B90FBFEF0022AAE
:1035780098546F4B0FD183F802E0039B53450EDB41
:10358800644CB4F89A21914215DBB1F5FA6FA8BFE3
:103598004FF4FA6110E09C54039B534504DA36F863
:1035A8000B305B4226F80B300132032A05F1010586
:1035B8007FF451AFE4E71146891A4FF47A73DFF8C4
:1035C800A4E1564D59436FF06303C2F5FA626427CC
:1035D800B1FBF2F191FBF7F23EF8120003FB021186
:1035E800013203B23EF91220D21A514391FBF7F38C
:1035F8000344F3804F4B1B88580635D54E4B4F4A32
:103608001B881288DFED4E7A9B1A1BB208EE103A1F
:10361800B8EEC88A28EE278AB0EE480A07F0FCFD03
:10362800F0EE408AB0EE480A07F093FDB5F9023093
:1036380006EE903AB5F90030F8EEE66A07EE903AF1
:1036480020EE667AF8EEE77AA7EEA87A67EE807A37
:10365800BDEEC77AE6EEA87A17EE103AFDEEE77AE5
:103668002B8017EE903A6B80364D2B68990740F106
:10367800A180354B354F1A687B6945F20721D31A6B
:103688008B4240F397807A6109F0ECFD304BDFF80C
:10369800D8901A78032A9846B9F8003022D10A2B14
:1036A8002AD90023282088F8003008F0C6F909F044
:1036B800D9FD284B188809F0BFFD274B1A68D37825
:1036C80090FBF3F001300828244BA8BF082018709D
:1036D800537980B213FB00F33B83137913FB00F09B
:1036E800788309E00A2B07D803231C4A88F800309E
:1036F800002313703B837B8398F80030144A012B16
:103708003DD033D3022B4CD054E000BF38280020E2
:1037180070100020202C002048100020F0100020FD
:103728000CFEFFFF1C1A0020CE0F0020341A0020C8
:1037380080190020D4110020E8100020320F00204A
:1037480035FA8E3CFC27002008340020C00F0020EA
:103758005C11002098230020F81000208000002031
:10376800341F0020E6110020FC1000203A8BB9F825
:1037780000309A421EDD012388F800300FE0B9F8C6
:1037880000107B8B8B4202DD022313700FE0A34BEA
:103798001B8B0133994202DD002313700AE00820D5
:1037A80006E07B8BB9F8002001339A42E3DC07205E
:1037B80008F07CF92D682A0576D5994B974F1A6839
:1037C800FB69C3EB020845F2072398456CDD954B6E
:1037D800B6F906B0D3F80090FA6199F80A30B4F84F
:1037E8005201914E012B4FF47A71ABF57A7B98FB1D
:1037F800F1F803D041D3022B20D040E08B4B386A3C
:103808005A7B8B4B33F812204FF0080E92B290FB84
:10381800FEF3C01A8318BA843B6240F6E44293FB75
:10382800FEF39BB25343B9F80820C2EB1333594354
:10383800B9F9063091FBF3F1316020E07D4BB9F81E
:1038480008A01B78C6F800A05B0718D50FF0D0FABF
:1038580020B915F0100F18BF4FF0000B32220BFBE8
:103868000BF393FBF2F3B9F906205B445A434FF488
:103878007A7392FBF3F3534400E000233360D7E9F3
:103888000A0133686C4A03FB08F84FF47A7398FB13
:10389800F3F810EB080041EBE8710023C7E90A01CF
:1038A8000FF0E0FA654B1860654E3368D90427D5E8
:1038B8002A0622D5634B1B789B071ED5624B1878C6
:1038C80004281AD90022614BD7180521951C4FF0FE
:1038D8000A0E122AD154E9B287F801E004D0B0EBFD
:1038E800510F2A46EFD800E014215A18322002F866
:1038F800010CFF225A540F2000E00A2008F0D6F8E5
:10390800534D2A68002A50D0524B534F18683968D3
:103918008142984649D8514BDFF84C911978526842
:10392800E1B94FF0010A83F800A0B9F80030D35C80
:1039380023B3504608F0A0F8494B83F800A00FF0D5
:1039480031FAB9F80030CBB92B681B78053B5345E1
:1039580014D808F04DF8434B18600FE04FF0000AF8
:1039680083F800A0B9F80030D35C3BB1504608F0AA
:1039780083F83B4B83F800A00FF014FA2A68B9F8D3
:10398800003052683848D25CFE2A01D100230BE08F
:10399800FF2A02D108F076F807E0D8F800500A218B
:1039A80011FB02523A6001330380224D2B785F07E6
:1039B80003D52E4B08221A8570E03268D0075CBF09
:1039C80043F001032B701F4B1B7819075EBF2B7840
:1039D80023F001032B70D30248BF2B78204A44BF41
:1039E80023F001032B70224B1B6813F0040F02D045
:1039F8002049098851B92049098809B19F0705D488
:103A08001E4B1B88003318BF0123CBB3022313704E
:103A18002B7823F001032B7037E000BFC00F002084
:103A280008340020F8100020041100208023002012
:103A3800902300202A340020407E05000811002031
:103A48000C10002010110020161100208C280020D6
:103A58005C1F002020280020541F0020501F002039
:103A6800182C0020602A0020581F0020000400485D
:103A78000C110020203400209C2100202634002036
:103A88002978CE0758BF0223137007F0B1FFB34B54
:103A98001B68C01A002801DB0FF084F909F0BEFF8B
:103AA800AF4B03931E78002E00F0A880AD4F3B6803
:103AB800002B00F01D87386808F080F8002800F017
:103AC8001787A84BA84C186808F075F8092801D082
:103AD8003F2852D14FF000092668DFF8C8824D46CA
:103AE80036B1A248D8F80010324612F0EDFA10B9F3
:103AF800C14605B945469E4B08F110089845EFD3D5
:103B0800EDB1D5F800C0D9F8008023681CF803E0AF
:103B180018F80300704512D15A1C944958B92D2B36
:103B280009D8DFF844E2CEF800204FF0200E01F863
:103B380003E0885403E001F803E02260E5E7236826
:103B48000BB14D4510D08B480EF016F84D4507D8EF
:103B580055F8100B0EF010F809200EF005F8F5E7EF
:103B680085480EF009F8002623689E42A3D27F4BB1
:103B7800985D0DF0F9FF0136F6E72368002B40F059
:103B88009C86042840F0D38678480AF0A9FD00F006
:103B9800AFBED8F80000DFF8F0A108F00FF818B3AE
:103BA800DAF8000008F007F8D9F8003093F8482050
:103BB80083468ABB242868D1012283F84820D9F893
:103BC8000030DFF8C0A193F848B0BBF1060FE0D190
:103BD80093F8490000F03AFF002877D00DF020FF55
:103BE8003B68002283F84820644B93F83530002B5B
:103BF80040F051864C36982E00F07A86604BF218C9
:103C080092F84A100129F5D15E4FF3583A605E4A9E
:103C1800B94613609046BCE7012A04D14D2814BF69
:103C280000220222C9E7022A04D13C2814BF00223C
:103C38000322C2E7032A0AD140284FF000029FBF9F
:103C48001A71DA715871987198BF0422B5E7042A7D
:103C580008D19A7983F8490080EA020B83F806B004
:103C68000522AAE7052AAAD159791A7991429979A0
:103C780006D941409971511C1971134418729EE775
:103C880081420CBF0622002297E72B78590796D469
:103C98002328DAF800300CD103993C4801220A7035
:103CA800304A1360354A13630DF066FF32480DF051
:103CB80063FF374B1B681B785B4501BF354B364AA2
:103CC8001A60364B04BF364ADA6078E7DAF8002023
:103CD80092F849304C2B00F0B58400F2B780352BB0
:103CE80000F08B8260D82B2B00F0848420D8252B01
:103CF80000F05C8404D8232B00F0448200F013BE4B
:103D0800272B00F05984292B40F00D860DF064FE16
:103D1800A4F882010DF060FEA4F884010DF052FEB3
:103D280084F886010DF058FEA4F8880100F0AEBDB5
:103D38002F2B00F0278504D82D2B00F05F8400F08E
:103D4800F2BD312B00F03385332B40F0EC850DF0BC
:103D580039FE84F8940100F099BD00BF1C2C0020A6
:103D68002D3400207C280020B42400208424002046
:103D78008094010877AA01087CAA0108C00F0020D6
:103D880070220020B4110020B8110020ACAA01084C
:103D980014230020FC9F0020EFBEADDE00ED00E004
:103DA8000400FA05A0920108412B00F0A58418D858
:103DB800392B00F00E8404D8372B00F0AA8400F0C9
:103DC800B2BD3C2B00F0CC803E2B40F0AC850DF012
:103DD800F9FD84F8DE010DF0F5FD84F8DD0100F051
:103DE80055BD442B00F0178525D8432B40F09B8503
:103DF8000DF0E8FD0023A36060710DF0F7FD07F0FA
:103E0800D7FA0DF0DFFD84F892010DF0E5FDA4F876
:103E18005C010DF0E1FDA4F85E010DF0DDFDA4F8F4
:103E280060010DF0D9FDA4F882010DF0D5FDA4F8CC
:103E3800840100F02BBD482B00F04D834A2B40F045
:103E480072850DF0C9FDA08100F020BDD12B00F0D6
:103E58006C8320D8CC2B00F00F820FD8C82B62D0EF
:103E680004D84E2B00F01A8400F05DBDC92B00F079
:103E78003583CA2B00F0838000F055BDCE2B00F0AF
:103E88001D83C0F01283CF2B00F04A82D02B00F0A4
:103E9800018300F048BDD82B00F005810BD8D32B47
:103EA8003BD027D3D42B00F07F82D62B40F03B8524
:103EB8004FF000086DE2F22B00F0C48212D8EF2B0D
:103EC80040F03185DFF89083D8F800900DF084FD3C
:103ED800A9F85A00D8F800800DF07EFDA8F858001F
:103EE80000F0D4BCF32B00F09B84FA2B00F0EF8297
:103EF80000F019BD2B7803F0040303F0FF08002B32
:103F080040F0C4840DF05EFD022884F8B40740F246
:103F1800C782CD4B83F8B487C2E20DF05DFDCB4B71
:103F2800188000F0B3BC92F805804FEA5808B8F141
:103F3800120F03D908F04EFD00F0A8BC4FF000099D
:103F4800C14507D20DF048FDC14B23F8190009F10E
:103F58000109F5E7BF4B012283F8342000F096BC35
:103F6800DFF8F482D8F800900DF02CFD89F80000F5
:103F7800D8F80030187805F0E5FF00F087BCB64B9C
:103F88001A681278022A4FF00009984670D1D8F8BA
:103F980000A00DF017FD07EE900AF8EE677AB2EE72
:103FA800048AC7EE887A0AEB890ACAED087AD8F833
:103FB80000A00DF007FD07EE900A9FEDA87AF8EE35
:103FC800677A0AEB890AC7EE877ACAED0B7AD8F8BE
:103FD80000A00DF0F7FC07EE900A9FEDA17AF8EE2D
:103FE800677A0AEB890AC7EE877A09F10109B9F1FC
:103FF800030FCAED0E7ACAD1B9F1070FD8F800A09D
:104008001CD10DF0DFFC07EE900AF8EE677AC7EED8
:10401800887ACAED117AD8F800A00DF0D3FC07EE23
:10402800900AF8EE677AC7EE887ACAED127AD8F85D
:1040380000A00DF0C7FC8AF84C0012E00DF0C2FC9D
:10404800CA448AF80100D8F800A00DF0BBFCCA44A5
:104058008AF80B00D8F800A00DF0B4FCCA448AF81E
:10406800150009F10109B9F10A0FC5D100F00EBC1C
:10407800D8F800A00DF0A6FCCA448AF80100D8F8C8
:1040880000A00DF09FFCCA448AF80B00D8F800A0E5
:104098000DF098FCCA4409F10109B9F10A0F8AF830
:1040A8001500E5D1F2E38146DFF8AC819FED6C8A1B
:1040B800D8F800A00DF090FC07EE900AF8EE677AA9
:1040C8000AEB890AC7EE887ACAED087AD8F800A000
:1040D8000DF082FC07EE900AF8EE677A0AEB890A7F
:1040E800C7EE887ACAED0B7AD8F800A00DF074FCF8
:1040F80007EE900AF8EE677A0AEB890AC7EE887A23
:1041080009F10109B9F1030FCAED0E7ACCD1B9F161
:10411800070FD8F800A01CD10DF05EFC07EE900A3E
:10412800F8EE677AC7EE887ACAED117AD8F800A057
:104138000DF052FC07EE900AF8EE677AC7EE887A1F
:10414800CAED127AD8F800A00DF046FC8AF84C00A7
:1041580012E00DF041FCCA448AF80100D8F800A02A
:104168000DF03AFCCA448AF80B00D8F800A00DF00C
:1041780033FCCA448AF8150009F10109B9F10A0F9C
:10418800C5D183E30DF01EFC132882463FF6D2AE5C
:10419800DFF8C490D9F800B00DF014FC0023314AC0
:1041A8000C2101FB0322117A814222D10FFA8AF8ED
:1041B8000BEB8808137888F879300DF003FC88F841
:1041C8007A000DF0FFFB88F87B000DF0FBFB264B17
:1041D800264A1A6088F87C00254BD9F80000186038
:1041E8000021793007F0CAFB224B80F001001870DB
:1041F8004CE301331B2BD2D19CE60DF0E3FB0B28DB
:1042080080463FF697AE144BD3F800900DF0DAFBDA
:1042180003283FF68FAE0BFB089B8BF8CE000DF002
:10422800D1FB8BF8C9000DF0CDFB8BF8CA000DF05F
:10423800C9FB8BF8CB000DF0C5FB8BF8CC000DF05B
:10424800C1FB8BF8CD0021E3202C0020300F00208B
:1042580038280020C00F0020481000200000C84265
:1042680000007A44FC880108280F0020642D0020F3
:104278002C0F00200C0000205379092B7FF65AAE32
:10428800019BD3F800800DF09DFB019B88F800008E
:10429800D3F800800DF096FB88F801000DF092FB32
:1042A800019B64281B68A8BF642018710DF08AFB65
:1042B800019B64281B68A8BF642058710DF082FB1D
:1042C800019BFF281B68A8BFFF2098710DF07AFB9F
:1042D800019B6428D3F8008028BF642088F8070071
:1042E8000DF070FB019B88F80200D3F800800DF0F8
:1042F80069FB019B88F80300D3F800800DF06CFB84
:10430800DAF80030A8F80A005B790A2B40F2BE827E
:10431800D34BD3F800800DF055FB88F80800B5E2C0
:104328000DF05AFB6FF4AF6283189BB2C62B98BF8F
:10433800A4F898010DF050FBA4F844010DF04CFBD3
:10434800A4F846010DF048FBA4F848010DF044FB21
:10435800A4F8DA010DF036FB84F8EB010DF032FB1E
:104368000DF030FB84F8EC010DF02CFB84F887018C
:104378000DF028FB84F894010DF024FBB94BD3F819
:1043880000800DF029FB00EB80004000A8F85600E3
:104398001FE10DF021FBB44B23F8180008F10108C8
:1043A800B8F1080FF5D171E253790F2B7FF4C2AD44
:1043B8000DF008FB072880463FF6BCAD029BD3F8FA
:1043C80000900DF009FB0E2303FB08F8C144029B83
:1043D800A9F81901D3F800900DF0FEFAC144029B28
:1043E800A9F81B01D3F800900DF0F6FAC144029B1E
:1043F800A9F81D01D3F800900DF0E4FAC144029B1E
:1044080089F81F01D3F800900DF0DCFAC144029B33
:1044180089F82001D3F800900DF0D4FAC144029B2A
:1044280089F82101D3F800900DF0CCFAC144029B21
:1044380089F82201D3F800900DF0D8FAC844C8F8DA
:10444800230123E20DF0BEFA0F2880463FF672AD35
:104458000DF0B8FAC8EBC808A04488F8D4000DF0ED
:10446800B1FA88F8D5000DF0ADFA88F8D6000DF04D
:10447800A9FA88F8D7000DF0A5FA88F8D8000DF049
:10448800A1FA88F8D9000DF09DFA88F8DA0007F04B
:1044980037FDFBE12B785B0700F1F8810CF002FA9D
:1044A80006F0B8FF07F070F8F0E12B78580700F134
:1044B800ED816E4B4FF4C8721A80E7E12B785907EB
:1044C80000F1E4816A4A137843F004032BE02B7867
:1044D8005A07E5D527E204F091F9D7E10DF072FA11
:1044E800634B1A7810B142F0020201E022F0020296
:1044F8001A700DF067FA5F4BDFF8988118700DF0AD
:1045080075FAC8F800000DF071FAC8F804000DF04B
:1045180063FA594B18800DF05FFA584B584A1880C7
:10452800137843F002031370B0E10DF04BFA8346A1
:104538000DF05CFA82460DF059FA81460DF056FAF4
:1045480080460DF049FA0DF047FA0DF03BFABBF141
:10455800000F14D14B4B1020C3F800A0C3F80490EF
:1045680006F0FDFE424A137843F001031370B8F1D8
:10457800000F00F08B81444BC3F8008086E1BBF14B
:10458800100F40F08381414BC3F800A0C3F804909A
:10459800B8F1000F02D03C4BC3F800803B483C4BBD
:1045A8000222011D1A7003F0D5FE6FE1A0600DF024
:1045B8001DFA06F0FDFE69E10DF00EFAA4F85C01A3
:1045C8000DF00AFAA4F85E010DF006FAA4F86001ED
:1045D8005CE10DF0F7F984F87C010DF0F3F984F84B
:1045E80080010DF0EFF984F87F010DF0EBF984F804
:1045F80081014BE10DF0E6F9607147E10DF0E2F958
:1046080084F892010DF0E8F9A4F89C010DF0E4F9A2
:10461800A4F898010DF0E0F9A4F89A010DF0D2F988
:104628003B6884F893015B79DFF86C80082B40F2D3
:104638002D810DF0D1F9A8F89E010DF0CDF9A8F85B
:10464800A00123E10DF0BEF984F8D8010DF0BAF904
:1046580084F8D9010DF0C0F9A4F8DA0116E100BF19
:104668007010002048100020622800209C210020A3
:104678001011002016110020141100201211002022
:10468800761000207810002088100020801000206C
:10469800340F002018110020202C002092F80580EB
:1046A8000323B8FBF3F8B8F1120F3FF643ACDFF879
:1046B80098934FF0000AC24580F0E8800DF082F927
:1046C80089F8A2010DF088F940F2ED23984205DD42
:1046D80040F6CA039842A8BF184601E040F2EE200F
:1046E800A0F2EE2019230AF1010A90FBF3F009F178
:1046F800020989F8A101DEE781460DF063F904EBB0
:10470800090309F10109B9F1080F83F88A01F4D105
:10471800BCE053794FF00709B3FBF9F9C9EBC902BB
:104728009B1A13F0FF0F7FF405AC5FFA89F909F1C2
:10473800FF395FFA89F9B9F1FF0F00F0A7800DF092
:1047480041F95FFA80FA4FFA8AF003F021F98046BE
:1047580000283FF4EFAB80F800A00DF03DF9A8F871
:1047680002000DF02FF988F804000DF02BF988F8F5
:1047780005000DF027F988F807000DF023F988F8EF
:104788000600D4E7DFF8C08208F140090DF024F9EB
:10479800A8F8AC020DF016F988F8AE020DF012F97F
:1047A80008F1040888F8AB02C845EFD16EE00DF0B7
:1047B80009F91F2880463FF6BDAB3B685B79082B9B
:1047C8007FF4B8AB0DF008F908F18A0804EB880803
:1047D80000F03F00A8F806000DF0FEF8B8F8063023
:1047E800800100F4FE501843A8F806000DF0EAF81E
:1047F800000188F804000DF0E5F898F8043000F09E
:104808000F00184388F804000DF0DCF888F805005C
:104818000BF04EFC3AE0794B012283F8352035E065
:104828000DF0D0F8FF2881461BD100238DF81F30EA
:104838009DF81F30072B29D89DF81F00704A9DF856
:104848001F3052F8300002EBC30301215B68994026
:1048580089B2042202F0AEFF9DF81F300133DBB2AB
:10486800E4E707283FF666AB00200DF0FDF80DF0F1
:10487800D7F8D8F8000007F098F918B9322007F0EF
:10488800DCF8F6E74FFA89F002F0A2FF00200DF0FD
:10489800EBF8FFF7A3B95B4B985907F086F918B9FD
:1048A800322007F0CAF8F6E707F0EAFA06F088FDC2
:1048B800554B564ADA60FFF79DB90C2839D00A28BB
:1048C80040D1534D53480DF057F92846232111F094
:1048D800E4FB08B1401B20602368002B55D14C48ED
:1048E80023600021302211F0A2FB039B1B781BBB25
:1048F800494B1B689B060FD5484B40491B688A6B80
:104908009A1A002A08DB464A1278042A82BF03F55D
:10491800123303F5F8738B63424B9B68002B67D007
:104928004148984764E008F055F8FFF757B90C2854
:1049380004D13E480DF020F93D480DE07F2812D102
:10494800FFF7B9B80D28BCD07F2809D1013B304A00
:10495800384823600021D1540DF00EF9FFF7ABB8A9
:104968002F2B3FF6A8A8A0F12002D2B25E2A3FF66C
:10497800A2A813B920283FF49EA85A1C2260244AF2
:10498800D0540DF0F1F8FFF796B85A1EA95C20290B
:1049980001D11346A1E71E4A23600021D154264BBA
:1049A800264DD3F80090D5F800A0DFF86480504673
:1049B80011F081FB064632464046514611F084FB11
:1049C8001F4A28B918F806304B445B78580703D0BB
:1049D80010359542E7D306E0954204D2701CEB6887
:1049E8004044984702E017480DF0C6F8002376E7E0
:1049F80009B0BDEC028BBDE8F08F00BFC00F0020EE
:104A080014AE01087022002000ED00E00400FA0551
:104A180084240020E8B901080C1100200834002083
:104A2800161100202C210020FC0F002081AA01086B
:104A38007CAA0108A8AA010890000020A0920108F9
:104A4800809401088CAA0108202C00202DE9F04749
:104A58002DED028B4B28A0B0044600F0438600F2EF
:104A6800B480302800F0CE8651D8222800F08D84FA
:104A780023D8032800F0608114D8012800F0508161
:104A8800022840F02A8704200CF0EEFF43200CF0A7
:104A9800B6FF4C200CF0B3FF46200CF0B0FF4C20C2
:104AA80000F055BE042800F05181052840F0158714
:104AB8001A200CF0D9FF002459E1282800F0E085DD
:104AC80015D8242800F0C785262840F00687B44C5E
:104AD80006200CF0C9FFB4F85C010CF0C8FFB4F86C
:104AE8005E010CF0C4FFB4F8600100F0B1BD2C28E1
:104AF80000F0D9852E2800F055862A2840F0ED864A
:104B080001200CF0B1FFA64B587900F020BE3D28DB
:104B180000F016831ED8362800F02A860BD83228D3
:104B280000F00F86342840F0D88648200CF09CFF0F
:104B3800002500F04CBC3A2800F0B3823B2800F076
:104B48001D84382840F0C98604200CF08DFF944C51
:104B580000F087BD452800F0AD8627D8402800F032
:104B6800F985422840F0B9868D4C10200CF07CFF66
:104B780060790CF044FFA0680CF082FF94F8920171
:104B88000CF03DFFB4F85C010CF071FFB4F85E0165
:104B98000CF06DFFB4F860010CF069FFB4F8820105
:104BA8000CF065FFB4F8840100F052BD472800F00E
:104BB8005F86C0F04C86492840F08F8602200CF0B2
:104BC80053FF774B988900F043BD702800F0EB82C3
:104BD80058D8692800F045822AD8652800F0FA805C
:104BE80015D84D2800F08D85642840F0768607207A
:104BF8000CF03AFFE7200CF002FF694B58790CF0F3
:104C0800FEFE00200CF0FBFE042000F062BE6728C8
:104C180000F0AA8100F2188212200CF025FF614BE7
:104C28001B88B3F5806F8CBF0825012500247EE121
:104C38006C2800F0298217D86A2800F08D846B2828
:104C480040F04B8605200CF00FFF574B18880CF0EE
:104C58000EFF564B18880CF00AFF554B93F8760058
:104C680000F0010000F073BD6E28514D00F0208265
:104C780000F2718206200CF0F7FE686E0CF000FF5F
:104C88004C4B0CE2782800F07C8119D8742800F08D
:104C9800BF830BD8722800F01F84732840F01D864C
:104CA80008200CF0E1FE012400F04FBC762800F04B
:104CB800738400F2F1832F200CF0D6FE3E4C55E3AE
:104CC800A42800F0918414D87B2800F0F582A0284D
:104CD80040F003860C200CF0C7FE384B18680CF027
:104CE800CFFE374B18680CF0CBFE364B186800F037
:104CF800F0BDF12800F08181FE2800F09C84F028A6
:104D080040F0EB852A4C04200CF0AEFEA36CB3F8FF
:104D18005A000CF0ACFEA36CB3F8580000F098BC35
:104D280003200CF0A1FE00200CF069FE20460CF0D8
:104D380066FE0C2000F00BBD0CF096FE01200CF076
:104D48005EFE0A200CF05BFE00F04CBC06200CF066
:104D58008BFE53200CF053FE52200CF050FE4620E0
:104D68000CF04DFE33200CF04AFE00F070BC164BE0
:104D7800185D01340CF043FE0B2CF8D10024134BC2
:104D8800185D01340CF03BFE082CF8D10024104BC0
:104D9800185D01340CF033FE072CF8D100F09BBDF0
:104DA800202C0020200000208A1100208C110020D7
:104DB80000100020E0100020CB880108ACF7FF1F8E
:104DC800B0F7FF1FB4F7FF1FA8A70108B4A7010891
:104DD80089A70108C94C0B200CF046FE20880CF06E
:104DE80046FE6268C64B9A420CBF2089608980B231
:104DF8000CF03DFEC34B1B68C3F3C000C3F3800235
:104E0800800040EA4200C3F340021043C3F340125B
:104E180040EAC20003F0100318430CF028FEBA4B16
:104E28001A88E36812F0010F14BF4FF0020C4FF01C
:104E3800000C12F0020F02F0080814BF4FF0040E25
:104E48004FF0000E03F4475912F0040F14BF102757
:104E5800002749EA080912F0400F03F4804814BFFC
:104E68002026002649EA080912F0100F03F400482A
:104E780014BF4FF40075002549EA080912F0200F05
:104E880003F4803814BF4FF48060002049EA080911
:104E980012F4807F03F4003814BF4FF4006100213E
:104EA80049EA080912F4007F03F48028974A49EA7E
:104EB800080903F4002849EA0809127803F480185D
:104EC80049EA080903F0007349EA0303C2F38002C0
:104ED80043EA020343EA0C0343EA0E0E4EEA0707CD
:104EE80046EA070645EA060540EA050041EA0001E8
:104EF80014BF4FF400184FF0000841EA08080020DA
:104F0800217C03468B420BD2814A9C5C012202FA27
:104F180004F414EA080F1CBF9A4010430133F1E768
:104F28000CF0AEFD7B4B93F8B40700F010BC7A4B45
:104F380033F9140090FBF5F0013480B20CF097FDC2
:104F4800032CF4D16D4CA08D0CF091FDE08D0CF08C
:104F58008EFD208E0CF08BFD608E0CF088FDA08EEF
:104F68000CF085FDE08E73E310200CF07DFD00242D
:104F78006A4B185D01340CF042FD102CF8D100F09A
:104F8800AABC70200CF070FD00265C4D0E24AB6CA2
:104F9800744323440136B3F819010CF068FDAB6C77
:104FA8002344B3F81B010CF062FDAB6C2344B3F847
:104FB8001D010CF05CFDAB6C234493F81F010CF051
:104FC8001EFDAB6C234493F820010CF018FDAB6C6C
:104FD800234493F821010CF012FDAB6C234493F8A1
:104FE80022010CF00CFDAB6C1C44D4F823010CF02E
:104FF80047FD082EC9D100F06EBC7020454C0CF05E
:1050080033FD04F1700594F8D4000CF0F8FC94F822
:10501800D5000CF0F4FC94F8D6000CF0F0FC94F8F1
:10502800D7000CF0ECFC94F8D8000CF0E8FC94F8ED
:10503800D9000CF0E4FC073494F8D3000CF0DFFC42
:10504800AC42E0D100F047BC10200CF00DFD00246C
:10505800334B185D01340CF0D2FC102CF8D100F061
:105068003ABC304D2878400000F0FE000CF0FCFC03
:1050780000242B789C4280F02E842B4B33F81400AC
:105088000CF0F5FC0134F4E7284C06200CF0ECFC9D
:1050980020880CF0ECFC60880CF0E9FC244B1888A4
:1050A800D6E204200CF0E0FC144B986E00F011BC22
:1050B80007200CF0D9FC1F4B1888FF28A8BFFF2039
:1050C800C0B20CF09CFC1C4B186880F3100080B236
:1050D8000CF0CDFCB5F86C000CF0C9FC0D4B93F846
:1050E8008721164B186822B10A23584380F3100011
:1050F80001E000F30F0080B2AAE200BF0010002018
:10510800005400400C110020D41100202A34002043
:1051180011100020202C0020DA1000203810002068
:105128004C1000200C23002038280020F4270020F1
:10513800E8100020FC1000200811002004110020B5
:10514800C44C02200CF090FC94F8DE010CF057FCE3
:1051580094F8DD01FBE20B200CF086FC2B6F18782D
:105168000CF04DFC2B6F58780CF049FC00262B6F87
:10517800B94C3344013618790CF041FC032EF6D1B2
:10518800236FD8790CF03BFC236F98780CF037FC30
:10519800236FD8780CF033FC236F58890CF067FC28
:1051A800236F187AD3E2AC4C1E200CF05DFCA36C84
:1051B8001B78022B4FF000056BD1A36C03EB850322
:1051C80093ED080AB2EE048A20EE080A11F03EF9BF
:1051D80080F30800C0B20CF012FCA36CDFED9F7ADC
:1051E80003EB850393ED0B0A20EE270A11F02EF945
:1051F80080F30800C0B20CF002FCA36CDFED987AD3
:1052080003EB850393ED0E0A20EE270A11F01EF931
:1052180080F30800C0B201350CF0F1FB032DCCD1AE
:10522800072DA36C23D193ED110A20EE080A11F083
:105238000DF980F30800C0B20CF0E1FBA36C93ED0C
:10524800120A20EE080A11F001F980F30800C0B232
:105258000CF0D5FBA36C93F84C3000EE103AB8EE86
:10526800400A11F0F3F880F30800C0B20BE02B44B9
:1052780058780CF0C4FBA36C2B44D87A0CF0BFFB15
:10528800A36C2B44587D01350CF0B9FB0A2DC7D10E
:1052980021E3A36C2B4458780CF0B1FBA36C2B448E
:1052A800D87A0CF0ACFBA36C2B440135587D0CF07C
:1052B800A6FB0A2DEDD10EE33C200CF0D5FB002413
:1052C800654D9FED678AAB6C03EB840393ED080A89
:1052D80020EE080A11F0BAF880B20CF0C8FBAB6CEB
:1052E80003EB840393ED0B0A20EE080A11F0AEF8E5
:1052F80080B20CF0BCFBAB6C03EB840393ED0E0A9D
:1053080020EE080A11F0A2F8013480B20CF0AFFBCD
:10531800032CD5D1072CAB6C16D193ED110A20EED6
:10532800080A11F093F880B20CF0A1FBAB6C93ED76
:10533800120A20EE080A11F089F880B20CF097FBE7
:10534800AB6C93F84C000BE0234458780CF08FFBBF
:10535800AB6C2344D87A0CF08AFBAB6C2344587DA1
:1053680001340CF084FB0A2CD4D1B4E214F8010FF8
:10537800002800F0B0820CF042FBF7E701200CF0A7
:1053880073FB354B9B6C1878E1E150200CF06CFBFB
:105398000025314B9C6C334B04EB85040C2194F8AD
:1053A800792001FB0233013593F838000CF027FB14
:1053B80094F87A000CF023FB94F87B000CF01FFBA8
:1053C80094F87C000CF01BFB142DE2D183E2224BF5
:1053D8009C6C062303FB0544013594F8CE000CF0C1
:1053E8000EFB94F8C9000CF00AFB94F8CA000CF004
:1053F80006FB94F8CB000CF002FB94F8CC000CF000
:10540800FEFA94F8CD000CF0FAFA0C2DDFD162E226
:105418004FF00008012600270F4B1A7C974232DA1A
:1054280011330024FA5C0F4D0C2305F1300163435E
:10543800595C914207D12B44586B10F03CFE8246D0
:105448002EB9B14610E001341B2CECD119E0804490
:1054580017E000BF202C0020001000200000C842E8
:1054680000007A44CC880108D1450ADA0C2303FBF2
:1054780004535B6B13F809000CF0C1FA09F1010938
:10548800F2E70137C8E7002E00F025825FFA88F0BE
:105498000CF0EAFA0026BEE7CD4D287C0CF0E4FAC1
:1054A80000242B7C9C4280F01682CA4BE65C0021CB
:1054B800C9480C2200F1300702FB01F3DA5DB24261
:1054C80005D1034493F838000CF099FA02E0013151
:1054D8001B29EDD10134E4E7C04C16200CF0C4FAC6
:1054E800B4F898010CF0C3FAB4F844010CF0BFFA10
:1054F800B4F846010CF0BBFAB4F848010CF0B7FA5E
:10550800B4F8DA010CF0B3FA94F8EB010CF077FA7E
:1055180000200CF074FA94F8EC010CF070FA94F88E
:1055280087010CF06CFA94F894010CF068FA0020EA
:105538000CF065FAA64B9B6C0A20B3F9563093FB26
:10554800F0F080B20CF093FA8BE0E0B201340CF08A
:1055580056FA092CF9D1BEE110200CF085FAA04BBF
:10556800A04C187800F002000CF049FA9E4B18780D
:105578000CF045FA20680CF083FA60680CF080FAA9
:105588009A4B18880CF073FA994B18880CF06FFA3C
:105598008F4BB3F874005BE00CF014FA0746122046
:1055A8000CF062FA8A4C17B9A66FE56F07E0102F66
:1055B80013BF0025D4F88060D4F884502E463846AE
:1055C8000CF01DFA30460CF05BFA28460CF058FA3D
:1055D800D4F888000CF054FA00200CF048FA0020A7
:1055E8000CF045FA0020B2E0794D95F88C00800067
:1055F8000130C0B20CF038FA95F88C000CF0FFF9C5
:1056080000242E4696F88C309C4280F06481794DB7
:10561800285D0CF0F4F905F11003185D0CF0EFF9B2
:1056280005F120033035185D0CF0E9F9285D0CF020
:10563800E6F90134E6E708200CF016FA00200CF031
:1056480016FA00200CF013FA00200CF010FA0020D3
:105658000CF00DFA3FE104200CF006FA5F4B986855
:1056680037E194F87C010CF0CAF994F880010CF049
:10567800C6F994F87F010CF0C2F994F8810166E04C
:10568800564C07200CF0F0F9B4F882010CF0EFF951
:10569800B4F884010CF0EBF994F886010CF0AFF93A
:1056A800B4F88801D4E74D4C0C200CF0DDF994F8DF
:1056B80092010CF0A4F9B4F89C010CF0D8F9B4F8F4
:1056C80098010CF0D4F9B4F89A010CF0D0F994F8D8
:1056D80093010CF094F9B4F89E010CF0C8F9B4F8F1
:1056E800A001B5E73D4C04200CF0BEF994F8D801B0
:1056F8000CF085F994F8D9010CF081F9B4F8DA01C5
:10570800A6E73D4C3D4D207800EB4000C0B20CF0C0
:10571800ABF9002623789E4205F1020580F0DB8074
:1057280015F8020C0CF06BF915F8010C00EB800071
:1057380000EB800000F2EE2080B20CF098F9013600
:10574800E8E701200CF090F9244B93F894010CF051
:1057580056F9C0E008200CF087F900241F4B2344B9
:10576800013493F88A010CF04AF9082CF6D1B2E01A
:10577800174B1A4C93F8CD00C0EBC000C0B20CF028
:1057880073F904F1280594F8F20100231C4AD25C4D
:10579800904200F0A4800C333C2BF7D10834AC4283
:1057A800F1D198E040200D4C0CF05EF904F1400571
:1057B800B4F8AC020CF05BF994F8AE020CF01FF9E7
:1057C800043494F8AB020CF01AF9AC42F0D182E040
:1057D8000010002011100020CC880108202C002087
:1057E800101100201811002016110020141100209B
:1057F800121100208D1000200C230020C22D002043
:1058080018230020E020444C0CF02EF904F1800508
:10581800B4F82E0200F03F000CF029F9B4F82E027B
:10582800C0F386100CF023F994F82C0200090CF050
:10583800E6F894F82C0200F00F000CF0E0F80434BD
:1058480094F829020CF0DBF8AC42E1D143E0334C88
:105858000D200CF009F905F07DF80CF0D0F820883F
:105868000CF00EF9E0680CF00BF902F0D1FE30E014
:105878000CF0BCF8054684200CF0F6F828460CF02D
:10588800FFF8264BDC6805F18003A3428CBF641B3C
:10589800802402F075FF28462246694605F08EF8F6
:1058A80000240546AC4216DA1DF804000CF0A7F8EF
:1058B8000134F7E713200CF0D7F80024184B185DD3
:1058C80001340CF09CF80B2CF8D100200CF0D8F81F
:1058D80000200CF0D5F8012018E0002016E00CF0AC
:1058E8008EF8B4F8F4010CF0C2F894F8F6010CF054
:1058F80086F894F8F7010CF082F894F8F9010CF0A6
:105908007EF894F8F8010CF07AF847E720B0BDEC7F
:10591800028BBDE8F08700BF202C0020100000207B
:10592800A8A701082DE9F047CB4CCC4F237886B0C7
:105938000646002B00F0EB813A686368D31A7C2B8B
:1059480040F2E581237A6260013323724FF0000848
:1059580008F12400C04DC0B208F014F805F10A039C
:1059680033F9183007EE903ABD4B1B88B8EEE77A4A
:1059780007EE903AF8EEE77A08F10108C7EE277AC1
:105988009FEDB87A67EE877AFDEEE77ACDED037A78
:10599800BDF90C0007F0E4FFB8F1030FD8D13020AF
:1059A80007F0F0FFB5F9100007F0DAFF07F0E2FFA3
:1059B8002B7A9A072CD16A6841F288339A4218D90F
:1059C800102007F0DFFF4FF06408686990FBF8F0DB
:1059D80000B207F0C5FF212007F0D4FF686990FBEB
:1059E800F8F308FB13000028B8BF404200B207F0E4
:1059F800B7FF142007F0C6FFB4F9180007F0B0FF8E
:105A08001C2007F0BFFF002007F0AAFF07F0B2FF35
:105A1800237ADFF844825B0740F05681022007F0C2
:105A2800B1FFD8F81C00DFF854926423323090FBA1
:105A3800F3F000B207F094FF0320B8F9265007F0FE
:105A4800A1FF894B1B7813F0040F4FF0050A95FB53
:105A5800FAF5ADB20BD030460DF0CAF928B9D9F82D
:105A6800003013F0100F18BF002528B205E0D8F851
:105A780028309889B0FBFAF000B207F071FFD9F826
:105A880000309E0765D5DFF8F891E68D99F800306B
:105A9800A28D714D36014FF06408B6B208FB023290
:105AA8005B00B2FBF3F346EA0326B6B2C3F3032363
:105AB8001E43062007F066FF30B207F051FFE38D62
:105AC80099F8001001339BB293FBF1F201FB1233FA
:105AD800E385236B9B7B012B05D1392007F052FF0F
:105AE800B5F92C0019E0AD8D6E233A205D431526DB
:105AF80007F048FF95FBF6F5AEB2B6FBF8F528B20D
:105B080007F02EFF08FB15653B2007F03BFFA8B206
:105B1800451D0A2095FBF0F000B207F021FF282070
:105B280007F030FF636B0A2093FBF0F000B207F038
:105B380017FF042007F026FFA36A9B8913B107F01B
:105B480053FB03E0444B986B80F3100000B207F05E
:105B580007FFE36B404E9D0640F1AB8096F840305E
:105B680098071DD5112007F00DFFB6F842003F4BEE
:105B78004FF4F365684390FBF3F000B207F0F0FED2
:105B8800192007F0FFFEB6F842004543642095FB54
:105B9800F0F595FBF0F300FB135000B207F0E0FEC0
:105BA80094F84030B4F8445013F0020F08BF0025B1
:105BB800012007F0E7FE28B207F0D2FE092007F01F
:105BC800E1FE002007F0CCFE294B94F846501A88D5
:105BD800B2F5967F0AD9204B1B7A03F00F03072BE7
:105BE80004D842F20F75954228BF1546052007F0E4
:105BF800C9FE236B5B7B0BB928B21CE0A5F120031F
:105C080007EE903A9FED1B7AF8EEE77AF6EE006A17
:105C1800C7EE877ABEEE007AF5EEC07AF1EE10FA9A
:105C280058BFB0EE667A77EE877AFDEEE77ACDED6B
:105C3800037ABDF90C0007F093FE94F84020064B58
:105C4800910703D493F84720012A1DD1012384F832
:105C58004730094834E000BFD01000202028002039
:105C68002000002000007A442A340020A086010089
:105C7800820000206666E63F18110020FC270020FD
:105C8800800000208096184B1B6B5FED026A93ED35
:105C9800017AD3ED027A27EE267A67EEA67ABDEE70
:105CA800C77AFDEEE77A8DED047ACDED057A04A882
:105CB80006E0B54A92E8030004AB83E803001846FF
:105CC80007F070FE07F056FE237A282B1FD1AF4B42
:105CD80000221A723C263B684FF47A70B3FBF0F846
:105CE800172007F04FFEB8FBF6F5B5FBF6F006FBFC
:105CF8001050000200B207F033FE182007F042FEF1
:105D080006FB158000B207F02BFE07F033FE94F86F
:105D180050309E4D002B00F0588105F069FE6B6DE8
:105D28009B4AC31A9342064640F2C180002385F875
:105D38005A3085F85C30AB8DDAB21B0A85F87620CC
:105D480085F8773085F86C2085F86D30D5F8842093
:105D58003B689A1AD5F88830D97B4FF47A734B434D
:105D68009A420ED38B4B1B68C5F8843095F88C305B
:105D7800013B012B9FBF102385F85A30022385F879
:105D88005C300A20626B92FBF0F284F874201212E5
:105D980084F8752094F84020A36B93FBF0F384F803
:105DA80078301B1284F87930920794F84630774996
:105DB80084F8A73003D42D2381F8A83076E0042B8B
:105DC800D4F84890E76CDFF8DC81734A8CBF332342
:105DD800322381F8A8304FF0060C704B99FBF3F092
:105DE80097FBF3F308FB009108FB037803EB8303AD
:105DF8000CFB01F103EB830391FBF2FE642502FB2C
:105E08001E119B0091FBF5F184F8991009120CFB07
:105E180008FC84F89A109CFBF2F143FA81F39BB2D8
:105E280002FB11C292FBF5F284F89E20121284F84C
:105E38009C3084F89F201B0AB4F8422084F89D30D7
:105E48002423534393FBF5F5B4F8BA3084F8A03013
:105E580000EB80001B0A00EB8000800084F8A13072
:105E68000A22B4F84430B3FBF2F303F5FA739BB299
:105E780040FA8EF080B284F8A2301B0A4FEAD97932
:105E880084F89700FF0F000A84F8945084F8A33030
:105E9800C5F30725B4F8BC3084F8969084F89800C8
:105EA80084F89B7084F8955084F8A930666594F856
:105EB800BE80364DB8F1000F0DD1D5F8C40005F0FD
:105EC8007DFE012807D90228354F00F0508207F0DF
:105ED80039FD0123BB70D4F8C8202C4D002A74D09A
:105EE80095F8BE703FB1D5F8D03040F6B731F31A07
:105EF8008B4219D869E00123D5F8C40085F8BE3073
:105F080001F0E3FCD5F8D43093F9000002238DE8C2
:105F1800880008213A464FF4964301F0E9FC85F8D9
:105F2800D870C5F8C4004EE095F8CC70CFB9D5F854
:105F3800C400C5F8C87085F8BE7001F0C6FCD5F875
:105F4800D43093F9000001238DE8880008213A46EF
:105F58004FF4964301F0CCFCC5F8C40007F0F2FCFE
:105F680031E0013FFFB285F8CC7095F8D81095F86C
:105F7800D930CFB94A1C013385F8D82085F8D930F3
:105F8800D5F8C4001DE000BF4C8A0108D0100020DD
:105F98003F0D03002028002040420F008096980003
:105FA80020000020806967FF12F8017BC5F8C8202F
:105FB800781885F8D8000133D5F8C40085F8D930A9
:105FC800394605F0FEFDC4F8D06094F8DA309C4DEF
:105FD800DBB1D5F8DC30C3B1D5F8E030ABB1C5F8EA
:105FE800E4301B68974AC5F8E830D5F8EC3013441C
:105FF800187AFEF72BFD0BF013FDD5F8EC300133C2
:10600800092B88BF0023C5F8EC308F4D94F8F02099
:106018002E688B4B002A00F0E481D3F8F420002A84
:1060280000F0DF8193F8F830013B012B00F2D981B1
:10603800D4F8F400824F05F0C1FDE0B1D7F8F400C0
:1060480005F0B9FD97F8F930D5F800907E2B804619
:106058000ED102231B2887F8F83009D1D7F8F400AD
:1060680005F0ACFD20B90123C7F8FC9087F8003192
:1060780084F8F980DCE7D7F8FC202B689B1A41F6F6
:10608800583293421DD9032387F8F830A9E16F4AA3
:1060980032F8130010B903464FF403600133B0F52A
:1060A800C06FDBB275D01DD9B0F5006F7AD031D989
:1060B800B0F5036F3ED184F80131E36B604F990668
:1060C8003FD494F8001194F80131002900F04C8174
:1060D8002A68921B012ADAD984F80131002384F84E
:1060E80000317EE1B0F5007F42D007D8B0F5807F5F
:1060F80047D0B0F5887F00F08580E6E7B0F5806F7F
:1061080000F0A880B0F5826F00F0ED80B0F5047F54
:10611800DBD123E0B0F5E26F00F08480B0F5E46FE6
:1061280000F08580B0F5E06FCFD184F80131B4F983
:106138000A1080E0B0F5046F6DD0B0F5026FC4D1DD
:10614800FCE097F840309A07BBD5B7F842102423F3
:106158004B431233642193FBF1F1FFE084F80131E2
:106168003B4B374F1B689B07ABD5BB8D0A21F4E02F
:1061780084F80131364B324F1B681905A1D5796B6C
:10618800ECE084F80131E36B2D4F5A0799D5796912
:10619800E4E084F801312E4B294F1B681B0590D58C
:1061A800B96BDBE0E16B264A84F801318F0688D5AC
:1061B80092F84010880784D5D90711D5D36C83EAA3
:1061C800E371002BA1EBE37101EB51014FF01902D0
:1061D800B1FBF2F1ACBF41F0004141F040410EE0AB
:1061E800936C83EAE371A1EBE371002B01EB51019E
:1061F8004FF01902B1FBF2F1B8BF41F080414FF402
:1062080000608AE084F80131E36B0D4F5B077FF58E
:1062180058AF3969A2E0B4F9181084F80131642341
:1062280059437AE084F80131B4F90C1003E0B4F969
:106238000E1084F801312C2391FBF3F16DE000BFBF
:10624800D01000204C8A010820280020C0AB01088B
:10625800FC27002084F8013194F80231624A0133A6
:10626800DBB2032B88BF012382F8023194F80211B4
:1062780042F2107359435D4B1B78D80748BF013170
:106288009A0748BF02315F07B4F8043148BF0431A8
:10629800D80748BF0A319A0748BF14311F0648BFBC
:1062A8002831D80548BF28315A0748BF64311F072D
:1062B80048BFC831980548BF01F5C8719A0648BF5C
:1062C80001F57A71DF0648BF01F5FA61580648BF43
:1062D80001F57A614FF4806000F0CCFD424B00225A
:1062E80083F80021EDE6E16BDFF8FC8084F80131EA
:1062F80011F0200717D098F8402012F0020F14BFB1
:106308004FF47A71002112F0010F14BF4FF4FA63B1
:1063180000230B4494F84610194400F0ABFD002309
:1063280084F80031CDE6324B1B6819067FF5C9AEFB
:10633800394600F09FFD88F80071C2E684F8013103
:10634800E36B294F9A067FF5BCAE97F840309B0760
:106358007FF5B7AEB7F844306421594300F08AFDA1
:10636800002387F80031ACE684F8013139E0BB78C6
:1063780023B1C5F8C06087F80280ACE5D5F8C03015
:10638800F31AB3F57A6FFFF4A6AD0123D5F8C4006C
:10639800BB7005F010FC0746D5F8C40005F00BFCEF
:1063A8007F067FF498AD8A2802D08E280CD092E51B
:1063B800EB6B98067FF58FAD95F8BE30002B7FF418
:1063C8008AAD05F18D0306E095F8BE30002B7FF409
:1063D80082AD05F15803C5F8C8302D2385F8CC30B7
:1063E80079E506B0BDE8F087D01000202A340020F7
:1063F800FC270020344B354A1B68126810B51A6018
:10640800334A1168596051689268DA60314A996074
:1064180011681961516892689A612F4A5961116827
:10642800D961516892685A622C4A19621188198593
:10643800518859859188D288DA85294A99851188A1
:1064480019865188598692889A86264A1188D9864B
:10645800518819871946928821F83A2F224A1078CC
:106468000022824206DA214C34F8124021F8024F09
:106478000132F6E71E4A1288A3F864201D4A1288E2
:10648800A3F866201C4A1188A3F86C1051889288DA
:10649800A3F87020194AA3F86E1012689A66184A71
:1064A8003B21126892FBF1F2B2F5967FC8BF4FF01C
:1064B800FF325A67134A1288A3F87820124A528981
:1064C800A3F85E2010BD00BFC828002008340020B3
:1064D800F0190020FC190020081A0020F0100020F4
:1064E8002C100020DA100020901F00204C100020F3
:1064F80098230020E40F002032100020E410002030
:10650800040000206C100020381000202DE9F8430A
:106518000E4B93E8800305460E460024B44213DA76
:106528007B1933F9140008EB050333F9142009EB40
:10653800050333F914301344022293FBF2F3C01A13
:106548000AF06AFD0134E9E7BDE8F883C8280020AD
:1065580010B5134B93F8DC37012B014619D1114BB9
:10656800114C1878421CD2B21A70120644BF00228D
:106578001A700E4A1B7812782154934236BFC2F122
:1065880080029B1A9B183F2B09D9BDE8104002F0E6
:1065980013B9074BBDE81040186805F012BB10BDD1
:1065A800202C0020682700206A2700206927002067
:1065B800B028002070B54720FFF7CAFF174B1B68AB
:1065C8001B0307D5164B174A5B6810681B68C01A6F
:1065D8000AF012FD144E154C154D30780AF00CFDDA
:1065E80023682868C01A0AF017FD63686868C01A2B
:1065F8000AF012FD0F4B18880AF0FEFC0E4B1888A3
:106608000AF0FAFC0D4B18880AF0F6FC337823746C
:106618002B68A3606B68E36070BD00BF4C2A002044
:10662800C82800200834002016110020B4280020B3
:1066380018110020141100201211002074100020DD
:106648007FB5254C254E264D2649274A274B20B194
:1066580027480088B0F5805F30D23088ADF8040054
:1066680028781D4D897912788DF806008DF8071065
:106678008DF808201B788DF8093001A829460622D4
:106688000FF0BAFC28B30198BDF808302860AB8039
:106698005320FFF75DFF20880AF0AEFCA0780AF0CF
:1066A800ABFCE37801932379029301A86379039300
:1066B8000AF006FC0E4B00221A800AE0308820807F
:1066C8008979287812781B78A070E170227163713B
:1066D800DEE704B070BD00BFD8110020D41100203F
:1066E80010110020340E0020630E0020C80E002078
:1066F8006C2A00200A4A138801331380094A136858
:1067080001331360084A138801339BB2202B01BF61
:1067180000231380054A138808BF0133138070478C
:106728006C2A0020542A0020582A00205A2A0020C7
:1067380038B5394B1B78083B012B05460C466AD8FF
:106748004520FFF705FF2846FFF702FF0C2D23D051
:1067580004D80A2D0AD014D835B138BD0E2D4BD027
:106768002ED3FF2D50D038BD206849E02078FFF7A0
:10677800EFFE62796378002A14BF80200020184356
:1067880000E02078FFF7E4FEA078FFF7E1FEE0786C
:10679800FFF7DEFE20793BE0B4F900000AF021FCA7
:1067A800A078FFF7D5FEE078FFF7D2FEB4F9040031
:1067B8000AF017FCB4F90600BDE838400AF011BC2D
:1067C800637820788BB180F08000FFF7C1FEA46861
:1067D800E0B2FFF7BDFEC4F30720FFF7B9FEC4F32C
:1067E8000740FFF7B5FE200E12E0FFF7B1FE606824
:1067F800BDE838400AF010BC20680AF0FDFB60686C
:10680800BDE838400AF0F8BB04480AF009FC00204B
:10681800BDE838409CE638BDA4280020E0AB01085C
:106828002DE9F04FBE4BBF4F1A888BB00193002A59
:1068380040F0A980B7F8DA07BB4E42F20103C21A4A
:1068480050425041FFF7FCFEFFF7D4FD3468492061
:10685800FFF77EFEB54B254618680AF0CDFB55F8C4
:10686800040B0AF0C9FB284605F0C6FF04F1100026
:1068780005F0C2FF04F11C094FF01008AC4D0123CC
:106888002A6803FA08F3134203D0D9F800000AF083
:10689800C3FB08F10108B8F1130F09F10409EDD1A0
:1068A80004F1280005F098FFB7F84431B4F92E0038
:1068B800C01A0AF0A1FB2B68DB0408D59D4BB4F87D
:1068C80064001B88181AC0F30D000AF095FB2B68AA
:1068D800980403D5B4F866000AF08EFB2B685905B6
:1068E80003D504F16C0005F077FF2B681A0502D573
:1068F800A06E0AF091FB2B685B0402D5606F0AF06A
:106908008BFB2B68180403D5B4F878000AF074FBE5
:1069180004F13000A04605F05FFF04F1360005F0F1
:106928005BFFB7F8443138F93C0FC01A0AF064FB32
:106938000127814B1B789F4208DA38F9020FB4F916
:106948003C30C01A0AF068FB0137F2E72B6899055A
:1069580005D5B4F95E00A0F2DC500AF05DFB3268A0
:1069680076487260B260121A9110754A4A43531CF5
:10697800032293FBF2F202EB42029A1A7C2303FBF6
:1069880002033360D6E16F4B6F4A1B6811688B4274
:1069980006D00AA9002041F8203D1360FFF7C8FE81
:1069A800019B97F8DA171B8897F8DB070B44013B24
:1069B800B3FBF0F200FB12338B4280F086815A4F12
:1069C8000120FFF73DFEFFF715FD50203E687D686A
:1069D800FFF7BEFDBA683B6810681B687A68034415
:1069E8001068A3EB40000AF017FB6A6873689B1AEB
:1069F8000293AA68B3689B1A0393EA68F36802A82B
:106A08009B1A049305F0F8FE2A6933699B1A0293CE
:106A18006A6973699B1A0393B369AA6902A89B1AE6
:106A280004930AF04DFA06F11C0B05F11C0810241A
:106A38003F4901220B68A2401A428A4606D0DBF879
:106A48000000D8F80030C01A0AF0E6FA0134132C16
:106A58000BF1040B08F10408EAD106F1260005F150
:106A68002601002331F9024F30F9022F121B02AC24
:106A780044F823200133042BF4D103214FF00009FB
:106A88004FEA89035FFA83F902AB53F821206AB110
:106A980002F108000F2802D849F0010906E0803207
:106AA800FF2A94BF49F0020949F0030911F1FF31A7
:106AB800E6D24846FFF74CFD00240DF1080BA0462E
:106AC80009F00302022A16D0032A1DD0012A4ED14A
:106AD800B8F1000F05D1DBF800402401E4B290467C
:106AE80045E0DBF8000000F00F002043FFF730FD21
:106AF8004FF000083BE0B8F1000F0CD0DBF80000C5
:106B0800C0F3031020432CE0B8F1000F1ED19BF80E
:106B18000100FFF71DFD9BF80000FFF719FD26E0B7
:106B2800582A0020202C0020C8280020542A0020A1
:106B38004C2A0020482A0020901F0020D42800203A
:106B4800DF7BEFBD602A00205C2A0020DBF8000014
:106B5800C0F303302043FFF7FBFCDBF80000C0F371
:106B68000710FFF7F5FCDBF800402401E4B20BF155
:106B7800040B06AB9B454FEA9909A1D1B8F1010F67
:106B880002D12046FFF7E4FCDAF8003013F4805411
:106B98001FBFB6F86420B5F86410521A029218BFE5
:106BA80001249A040AD50AAA02EB8401B5F8660002
:106BB800B6F86620121A41F8202C0134580513D56E
:106BC80002AA02EB840C06F16A0E05F16A000022A3
:106BD8003EF9021F30F9028FC8EB01014CF8221070
:106BE8000132032AF4D10334190508D50AAA02EBA5
:106BF8008400A96EB26E521A40F8202C01345A044F
:106C080008D50AAA02EB8400696F726F521A40F81D
:106C1800202C013418040BD50AAB03EB8402B5F819
:106C28007810B6F878305B1A42F8203C013400E05E
:106C3800FCB1012C03D102980AF0EEF919E0631EA9
:106C4800002002AA400052F82320C0B20AB140F046
:106C58000100013BF5D5FFF77BFC4FF0000802ABC4
:106C680053F8280008B10AF0D7F908F10108A0453F
:106C7800F5DB30200321FFF749FC36200321FFF71D
:106C880045FC2F4B3C201978FFF740FCDAF8003020
:106C9800990506D5B6F95E00B5F95E30C01A0AF056
:106CA800BBF93A6827487B687A60121A9110264A1D
:106CB800BB604A43531C032293FBF2F202EB4202ED
:106CC8009A1A7C2303FB02033B60204B1B681A06BD
:106CD80030D51F4C1F4D22682B689A420BD1626831
:106CE8006B689A4207D1019B1B88102B11D11A4B54
:106CF8001B885B060DD14820FFF72AFC20680AF0A4
:106D08008BF960680AF088F923682B6063686B6008
:106D18000EE0124A0F4B11782A7C914208D1104A92
:106D280099681068884203D15268DB689A4201D09A
:106D3800FFF740FC0AF0B2F80BB0BDE8F08F00BFD7
:106D4800901F0020D4280020DF7BEFBDFC27002007
:106D580078100020B42800205A2A0020161100209C
:106D6800181100202DE9F84F0C9E3A4CC2EB030B8A
:106D78000B9BF61A6368002914BF4FF0060A4FF000
:106D8800040A01330546904613D1236853455ED261
:106D9800314A324852F82320032B98BF29460AF07B
:106DA800A9F96368013363602D4B002205469A7187
:106DB80013E0002511E02B4A1278954240DA0B9B2C
:106DC800E3B109FB06F2995C01228A402649096869
:106DD8000A4213D1636801336360D4F804900A9BB4
:106DE8001C4F9945E7DB2BD10A20FFF7B1FB3B6825
:106DF80001333B604FF0FF337B6021E0184A917903
:106E080021B12C20FFF7A4FB013501E0012191718C
:106E1800226809FB0BF308EB030752B958F8030083
:106E28000AF0FEF897F904104B1C0544D2D00F481D
:106E380002E03A440E4811790AF05CF90544C9E7C2
:106E4800206850452CBF00200120BDE8F88F0020A5
:106E5800BDE8F88F642A0020608A0108EBAB0108BE
:106E6800D81100208C0000204C2A0020FAAB010821
:106E78006DAF010830B585B004AC002524F8025D7B
:106E88000091ADF806002146102006F03DFD9DF862
:106E98000600214606F038FD9DF80700214606F059
:106EA80033FD9DF80000214606F02EFD9DF80100F7
:106EB800214606F029FD9DF80200214606F024FD32
:106EC8009DF80300214606F01FFD9DF80E00C04303
:106ED800C0B2294606F018FD05B030BDF8B5044625
:106EE8000E4617460025204620210FF0D6F8044606
:106EF800D0B1013420460FF035F9B0F5617F05DBDC
:106F080040F634039842A8BF184601E04FF4617078
:106F1800A0F56170192390FBF3F00DB9307000E013
:106F280070703B7801333B700DB90125DBE72046D3
:106F3800F8BD30B505460C46134629462246024898
:106F4800BDE8304004F0D6B8F0AC01087FB504784D
:106F58000646E4B9354B1B6803EB8403192193F803
:106F68007B0093F87C6093F8792093F87A304FF49B
:106F7800617511FB005011FB0651009001912C48DE
:106F88002146013404F0B6F8142CE3D14BE00FF09D
:106F9800E9F81328054641DC244B701C1C682021A5
:106FA80000238DF80F300FF078F81E35064670B1C3
:106FB800013630460FF0D6F819289FBF04EB850339
:106FC80058709DF80F30013398BF8DF80F30304658
:106FD80020210FF062F8064670B1013630460FF0F6
:106FE800C1F80D289FBF04EB850398709DF80F30FA
:106FF800013398BF8DF80F3004EB85043046E11C4F
:107008000DF10F02FFF76AFF9DF80F30042B0AD02D
:10701800601C002104220FF00AF804E00548002152
:107028001322FFF786FF04B070BD00BF4810002090
:107038000FAD010824AD010801480AF09DBD00BF4D
:107048002AAD01082DE9F04304788FB00546002CDD
:1070580059D17B4B0021142209A807AED3F8008030
:107068000EF0E5FF0722304600210EF0E0FF05A8EC
:107078000023A700059308EB070583801A4671498A
:10708800B5F802E031F813C01CEA0E0F0AD00DF172
:10709800380C0E3102F1010E6244595C02F81C1CD6
:1070A8005FFA8EF20133072BE9D100210B46664ABD
:1070B800B5F802E011F802C01CEA0E0F0AD00DF173
:1070C800380C063203F1010E63448A5C03F8242C61
:1070D8005FFA8EF301310629E9D118F807305B49C8
:1070E8008DE841006A78029209A81A0903F00F0393
:1070F80003F0EBFF2146564809AA013403F0FAFFD2
:10710800202CA6D198E00FF02DF81F28044600F394
:10711800868028462021E4B20EF0BFFF1F2C02D93A
:10712800FFF78AFF88E0464B1B6803EB8404451C85
:107138000021204604220EF07AFF0027454B09AEB5
:10714800304600210A2217F803905FFA87F80EF0FC
:107158006EFF002315F8012B32B10A2B04D04A45E3
:1071680002D0F2540133F5E74A455ED108F1FF3306
:10717800032B09D8DFE803F01005023F0DF12301C6
:1071880034E00DF123011EE030460EF0EBFF2378CA
:10719800C0B243EA001006E030460EF0E3FF237861
:1071A80000F00F001843207031E00133062B0AD09D
:1071B800244800F11B069E5D9642F6D103445A7D91
:1071C80063881343638011F8012F02B30023EFE7AC
:1071D8000133072B0AD01B4800F10E069E5D96422C
:1071E800F6D130F8132063881343638011F8012F18
:1071F8006AB10023EFE730460EF0B4FF0F2804DC35
:1072080030460EF0AFFF607001E000236370013775
:10721800052F93D1012408F04BFF6CB980E70E4885
:1072280000211F22FFF785FE06E0204600210422E8
:107238000EF0FDFE0024EEE70FB0BDE8F08300BFBE
:10724800E0110020788A01088D8A010838AD01080C
:1072580047AD0108998A010824AD0108F8B50478FA
:10726800064674B9304DB5F8C621B5F8C8312F486F
:107278002146013403F03EFF042C05F10405F2D148
:10728800F8BD2B490EF0DCFEA8B9274B4FF47A71F4
:107298004FF4FA62A3F8C611A3F8C821A3F8CA11DB
:1072A800A3F8CC21A3F8CE11A3F8D021A3F8D211CA
:1072B800A3F8D421F8BD30460EF054FF0328054644
:1072C8002BD8304620210EF0E8FE044630B10134B8
:1072D80020460EF047FF0126074600E006462046F6
:1072E80020210EF0DAFE10B9BDE8F840A4E601301E
:1072F8000EF038FF012EF7D1A7F2EE2240F2DC5350
:107308009A42F1D8A0F2EE229A42EDD8064B703597
:1073180003EB8503DF801881F8BD064800210322AE
:10732800BDE8F84005E600BF202C002053AD010859
:1073380066AD010830BB01082DE9FF410478054618
:10734800002C39D17348744D0AF016FCD5ED057A36
:10735800F5EE407AF1EE10FA00F0D88021466F4839
:1073680003F0C8FE95ED050A684603F043FD0146A3
:107378006B4803F0BFFE95ED060A684603F03AFD38
:107388000146674803F0B6FE95ED070A684603F024
:1073980031FD0146624803F0ADFE95ED080A6846E6
:1073A80003F028FD013401465E4803F0A3FE0C2CCF
:1073B80005F11005CAD1A9E05B4905220EF084FE4B
:1073C80040B9554B03F1C002002159611033934273
:1073D800FAD19BE02846554904220EF075FE044672
:1073E8002846002C40D120210EF057FE002800F03E
:1073F8008D80451C28460EF05EFE07464C4B53F820
:1074080024601EB94B480AF0B7FB7FE02846314696
:10741800FAB20EF059FE01340028EFD13E4B03F1C9
:10742800C0029E460021596110339342FAD1424B63
:1074380003EBC4029846D2F804C0BCF1000F04D193
:1074480031463E4803F056FE57E0002718F834301E
:107458009F42F5DA3B010EEB030563440FCB14356D
:1074680085E80F000137F1E70EF07CFE0B28064691
:1074780047DC284620210EF010FE054650B10135A4
:10748800284603F02DFC244B03EB061383ED050A75
:10749800012400E00446284620210EF0FEFD0546A2
:1074A80048B10135284603F01BFC1B4B03EB0613C0
:1074B80083ED060A0134284620210EF0EEFD05462C
:1074C80048B10135284603F00BFC134B03EB0613B8
:1074D80083ED070A0134284620210EF0DEFD10B99D
:1074E800FFF7AAFD12E0013003F0FAFB0A4B032C68
:1074F80003EB061686ED080AF2D11148FFF71CFFC8
:1075080004E0104801210C22FFF713FD04B0BDE888
:10751800F08100BF6CAD0108202C002087AD010868
:107528008DAD01088CB8010866AD010891AD010860
:107538008094010896AD010820AC0108A5AD0108AA
:10754800ABAA010824AD0108F0B5047887B0064657
:107558001CBB514B1968062303FB0411192091F831
:10756800CA5091F8CB7091F8CE2091F8C9304FF4F9
:10757800617610FB056510FB07600095019091F896
:10758800CC000290C831454849790391214601341D
:1075980003F0B0FD0C2CDCD17CE00EF0E3FD0B28F1
:1075A800044672DC3C4B701C1D68202100238DF8BA
:1075B80017300EF072FD064680B1013630460EF0E7
:1075C800D1FD03289FBF062303FB045383F8CE0095
:1075D8009DF817309CBF01338DF8173030462021B5
:1075E8000EF05BFD074680B1013738460EF0BAFD54
:1075F8000D289FBF062303FB045383F8C9009DF899
:1076080017309CBF01338DF8173006266643A91939
:107618003846CA310DF11702FFF760FC20210EF041
:107628003CFD074670B1013738460EF09BFD142823
:107638009FBF9DF817307619013386F8CC0098BFA4
:107648008DF81730384620210EF027FD78B101302B
:107658000EF088FD0D289FBF062303FB045383F813
:10766800CD009DF817309CBF01338DF817309DF879
:107678001730062B0ED0062202FB04500021C93019
:107688000EF0D5FCFFF7D8FC04E0054800210B22DA
:10769800FFF74FFC07B0F0BD48100020B1AD01085E
:1076A80024AD01082DE9F341047880464CB9204601
:1076B80001A90AF055F80134FFF7F4FF122CF6D1AE
:1076C8006BE00EF04FFDC6B2112E61D8344C06F1B6
:1076D800D00704EB470308F1010020219D780EF044
:1076E800DCFC18B9AA1E5542554139E04378682B8D
:1076F80006D0732B07D0612B13D14FF0000804E09C
:107708004FF0010801E04FF00208A8F102035D42C2
:1077180000F101004FF020015D410EF0BEFCD8B130
:1077280015B9FFF789FC38E001300EF01BFD40F277
:10773800ED2380B2984205DD40F6CA039842A8BFFF
:10774800184601E040F2EE2004EB4703A0F2EE20D9
:10775800192290FBF2F0D87004EB470383F80280FB
:1077680004EB47040F4AA378134493F8262055B135
:10777800E3780D4840F2EE241925314605FB034312
:1077880003F0B8FC09E03146084803F0B3FC04E014
:10779800074800211122FFF7CCFB02B0BDE8F081B9
:1077A800202C0020788A0108D1AD0108E3AD01083A
:1077B80030BB010807B50123ADF8041001A98DF805
:1077C80006208DF8073007F035FE03B05DF804FB9E
:1077D8002DE9F843054672B64FF090464FF48061A4
:1077E8004FF40079318530460422A6F82890FFF737
:1077F800E1FF304601224946FFF7DCFF2B4850F8ED
:10780800354000EBC500236842680125570005FA9A
:1078180007F848EA030395402360A561C6F8189065
:107828004FF090431B8A5B05FAD4236848EA0303A8
:1078380023604FF090434FF40072A9B221851A8556
:107848000822C3F8182440F605534FF09040028AE6
:10785800560512D4013BF8D122680323BB4022EA23
:10786800030323604FF400710222FFF7A3FF62B6FF
:107878003220BDE8F84304F0E0B8A56120460422B0
:10788800FFF798FF4FF090431A8A5205CDD5228A08
:1078980092B21542064A4FF400704FF0080115BF26
:1078A8009861188591611185ECE700BF14AE010855
:1078B8000004004810B50446204604F076F918B9CB
:1078C8000A2004F0BAF8F7E710BD002207490C2394
:1078D80003FB02135968814204D10022C2621A7262
:1078E8005A6070470132052AF0D1704718230020EA
:1078F8002DE9F74389469DF8288011461A469DF8D8
:107908002C30064600250C2068431D4FC419C0576B
:10791800B04202D1207A20B12BE00135052DF2D1F9
:1079280027E0022E0FD005DC56B1012E21D100939D
:1079380014480AE01E2E0DD01F2E1AD1012009E08E
:107948000093114801E011480093434601F0D6F82E
:10795800044605E002F044FF4146044604F022F9DB
:107968004CB10C2303FB0575267185F808906C60F3
:1079780001E0002000E0204603B0BDE8F08300BF2E
:10798800182300200044004000380140004800400F
:1079980010B5084B1968002201EBC20393F90240A5
:1079A800844201D1981C10BD0132052AF4D100206F
:1079B80010BD00BF14230020F0B5027887B08AB943
:1079C8004A4C04F1280694F8F221002348495956F4
:1079D80050B281426ED00C333C2BF7D10834B442FC
:1079E800F1D181E0002204920592451C0EF0BAFB09
:1079F800C4B260B2FFF7CCFF074618B18DF810404B
:107A0800012400E00446284620210EF046FB0546E6
:107A180038B1013528460EF0A5FB0134ADF8120047
:107A2800E4B20026284620210EF037FBB0B3451CEF
:107A380028460EF097FB00222E4951F82230834247
:107A48005FFA82FE04D00132082AF5D1002300E053
:107A5800734651F82320824220D1022E0FD0032EE4
:107A680012D05A1E012ED2B204D0042A13D88DF88F
:107A780014300EE0042A0ED88DF8153009E0052BD5
:107A880009D88DF8173004E09A1E052A03D88DF816
:107A980016300134E4B20136042EC3D1052C04D8C3
:107AA80007B0BDE8F040FFF7C7BA04AB03CB3860B6
:107AB800796019E094F8F7010E4B94F8F65153F8F1
:107AC8002000B4F8F421009094F8F90153F820004C
:107AD800019094F8F80153F82000029053F82530EB
:107AE800054803F007FB79E707B0F0BD202C00201C
:107AF800182300203C920108F2AD010838B14388F0
:107B080011EA030003D08B420CBF0120022070470A
:107B180030B50A4B0A491C680A79042A0AD8134660
:107B280004EBC303551CEAB29D882842F5D00A71BC
:107B3800981C30BD0A71002030BD00BF14230020FE
:107B4800E0110020014B00221A71E1E7E01100204A
:107B58002DE9F047877890F803C0214DBBB2C7F1F3
:107B6800640E03EB83065C42C3F178005FFA8EFE75
:107B78007600CCF16408A4B280B2A3B20FFA83F9FC
:107B8800B9F1000F05DC002B14BFBA464FF0010A0B
:107B980000E0F24613FB03F303FB0CF21AFB0AF3B3
:107BA80092FBF3F3434403FB09F30A2293FBF2F33A
:107BB80033449BB225F8023FB1F800904A880A3452
:107BC800C9EB020AA4B21AB202FB0AF24FF47A73A2
:107BD800844292FBF3F34B442B80CED1BDE8F0876F
:107BE800E4110020426A806A131A584258417047CB
:107BF8004171704743799B070AD5436A8269D1541A
:107C0800436A01690133B3FBF1F201FB12334362AA
:107C1800704707EE900AF8EEE77ADFED0C6A9FED01
:107C28000C0AF5EEC07AF1EE10FAD4BFB1EE677A1D
:107C3800C7EEA67A08B5D8BFC7EE267A27EE800A1F
:107C480003F0EAFA034B83ED000A08BD8096184B4F
:107C580035FA8E3C7800002038B50D4B0D4D1A8A48
:107C68000D4B1968498811421C4603D003F0C0FE29
:107C7800286007E003F0BCFE2B68984282BFC01A58
:107C8800064B186023685868BDE8384004F0DABE2F
:107C98000004004800120020A00700200400002073
:107CA80003460A4690F84602D96A9B7902F098BDC5
:107CB800437913F0010310B504460DD002F066F9BC
:107CC80058B1236A6269E168D05C0133B3FBF1F211
:107CD80001FB1233236210BD184610BDF8B59B4B4B
:107CE8001B680446187818B1012800F068819BE2E7
:107CF800242C974D0CD006D80A2C00F0D9800D2CD6
:107D080000F0D68046E12A2C06D02C2C04D041E184
:107D180028716871A8714EE18E4B69792F798C4A68
:107D2800002058542FBB1978D771472921D1597889
:107D380050291ED19978472907D1D978472904D1E4
:107D48001979412901D10121D1719978814A5229A2
:107D580003D1D1784D2900F0918299787D4A47293D
:107D680007D1D178532904D11279562A04BF0322A6
:107D7800EA71EA79764E022A39D0032A4CD0012AD0
:107D880040F08580BA1E072A00F28180DFE802F001
:107D980004080F131A257F2A09F036FCA86076E03C
:107DA8001B78532B73D1AB685B42AB606FE009F073
:107DB8002BFCE8606BE01B78572B68D1EB685B42C3
:107DC800EB6064E01B78302B634B1A788CBF42F071
:107DD800020222F002021A7059E0002009F074FC35
:107DE800287454E0002009F06FFC68824FE0072FE8
:107DF80006D0082F4BD1012009F066FCF08246E03E
:107E0800012009F061FC41F2184358434FF47A739A
:107E1800B0FBF3F0B0823AE0022F07D0032F0AD16B
:107E2800002009F051FC4D4B187030E0002009F09B
:107E38004BFC30762BE02AD93A1F9210337E013260
:107E4800D2B2013B02EB8303DBB2102B1FD8F91E21
:107E5800C2F1010201EB8202D2B2012A0BD0042A3C
:107E680011D100205E1E09F02FFC3D4B98553D4B6B
:107E780000229A5507E05E1E3B4A0020935509F000
:107E880023FC3A4B98553A4A136801331360304B38
:107E98002A2C18BF9A7907F101074FF000000CBF90
:107EA800012254402F7168710CBF5A769C7182E090
:107EB800687E002847D02F4B13F8012D2E495A70A1
:107EC8008B42F9D1234A224C13785278402B85BF34
:107ED800373B1B011B01DBB298BF03F0F003402ABC
:107EE8008CBF373A303AD2B21344AA79DBB29A42FD
:107EF80026D121230B702149E0790B681E4A0133F2
:107F080001280B600AD002281CD1722313701C4B65
:107F1800A28A1A801B4BE28A1A8013E06723137027
:107F28000D4B1B789F070ED5174BA2681A60E268A5
:107F38005A60164B227C1A70154B628A1A8002E02E
:107F48003F230B70002000236B7634E0C407002029
:107F58000012002028280020101100208C1000207A
:107F6800BD100020AD1000208D1000209D100020B5
:107F780060240020D8020020C40200206C240020C5
:107F88001211002074100020181100201611002072
:107F9800141100206B79687E0E2B9FBFA34A591CD1
:107FA8005171A34A98BFD454A04A18B993795C4038
:107FB800947100E00020003018BF0120F8BD9B4BF1
:107FC800997E0022082900F22F81DFE801F0050BD5
:107FD8000F15202B48606A00B52C40F02581DA7611
:107FE80001223AE0622C08BF022236E003229A7688
:107FF8001C775C779C7717E104229A765A7F997FE1
:10800800DC772244D2B25A770A449A770CE10522E7
:108018009A765A7F997F1C842244D2B25A770A44AE
:108028009A7701E106229A765A7F997F2244D2B242
:108038005A770A449A771A8C02EB0424A4B2B4F54E
:10804800AC7F88BF794A1C8484BF0121D176002285
:108058005A84002C40F0E88007229A76E4E05A7FA0
:10806800997F2244D2B25A770A449A775A8CB2F549
:10807800AC7F3CBF6D49891802F1010238BF81F815
:108088002440198C92B291425A84E5D9CCE0082256
:108098009A765B7FA34200F0C780644B0122DA76B0
:1080A8000DE0644D9A7615F8012D6A70624A954282
:1080B800F9D1997F5D4AA14206D03F232B705F4AD0
:1080C800536801335360AFE05D48016801310160D6
:1080D800D07E10B13E232B70A6E021212970D17FDC
:1080E800062941D004D8022907D0032923D0F8BD96
:1080F800122959D0302967D0F8BD5021297051492B
:10810800946A4C60D46A0C60516B4FF47A7491FB9A
:10811800F4F14D4C218092F87C114C4A19B1117838
:1081280041F0020102E0117821F0020111700122F0
:1081380083F87D2169E05321297092F82910CE0730
:1081480005D592F82820D51E6A426A4100E0024609
:1081580002F0010183F87C11002A56D13B490A78C4
:1081680022F002020A7050E04F21297092F82F1075
:10817800CC0705D592F82E20D11E4A424A4100E08C
:10818800024602F0010183F87C1122B92F490A78CE
:1081980022F002020A702E4A93F8531011702D4AE9
:1081A800B3F85010118030E0562129702A49946B99
:1081B8000C8042F21074D16B91FBF4F1274C2180B2
:1081C800012182F87E1120E04921297092F82810B7
:1081D800234A102988BF10211170224914780022DF
:1081E800A2420ED2204D0E7A5655204D4E7A565543
:1081F8001F4DCE7A56551F4D11F80C6F565501324A
:10820800EEE71D490A6801320A6093F87D31074A92
:10821800002B3AD092F87E31BBB3002182F87D1151
:1082280082F87E111846F8BD0020F8BD0012002023
:1082380028280020D8020020C4020020A40700201B
:108248006C240020181100201411002010110020A7
:108258001611002082000020121100207410002046
:108268008C100020241200208D1000209D1000206A
:10827800AD100020BD100020602400201279432A90
:108288007FF46BAD0222EA7167E5F8BD0449054B3E
:108298000968187000225A6199611A77704700BFFF
:1082A80020280020A407002010B5121A07EE902AF3
:1082B8005B1A2DED028BF8EEE78A07EE903A184B21
:1082C800059CB8EEE78AD3ED007A28EE278A28EED7
:1082D800080AA8EEA80A0EF05FFBDFED127A049BED
:1082E80020EE270AF0EE480ABCEEC00A83ED000A29
:1082F800B1EE680A0EF0ACF9DFED0B7A9FED0B7A60
:10830800E0EE077ABDEC028BFDEEE77A17EE903AC5
:10831800002BBCBF03F50C43A033236010BD00BF86
:10832800780000202C7D8E3F00A00C46A00CB345A1
:1083380044F25063984203DDA0F50C40A038704722
:10834800034B9842BCBF00F50C40A030704700BFFB
:10835800B0B9FFFF73B51A4C036823600B686360FC
:10836800184D0068184EFFF754FC184B009395E819
:10837800030094E80C000196FFF796FF144B32684F
:108388001A606868636813491B1A07EE903A124B23
:10839800286893ED007A23681B1A0B600F4BF8EEE0
:1083A800E77A1A600E4B67EE877A1B68FDEEE77A6C
:1083B800DA880C4BC1ED017A1A8002B070BD00BF9B
:1083C800082700201811002014270020102700205B
:1083D8005027002018270020780000204827002078
:1083E800380F0020442700204279DFED2A5A2A4B13
:1083F8009FED2A5A07EE902AF8EE677AC27BC7EEFD
:10840800A57AB2EE047AC3ED007A07EE902AF8EE68
:10841800677A234ADA60C7EEA57AC3ED017A8179D3
:10842800204B07EE901AF8EE677A017CDA60C7EE07
:10843800877AC3ED007A07EE901A817E06EE101A4D
:10844800F8EE677AB8EE466AC7EEA57A86EE056A50
:10845800C3ED017A83ED026AC179134B06EE901AD7
:10846800417CDA60F8EE666AC6EE876A07EE101A93
:10847800C17EC3ED006A07EE901AB8EE477AF8EEAF
:10848800677A87EE257AC7EE857A83ED017AC3EDA0
:10849800027A70470000C8422027002000007A4472
:1084A8000000FA44302700205427002010B50C4C57
:1084B80023789B0713D50B4B1B78042B0FD90A4A3B
:1084C8000A4B106852685A601860FFF7A2FB084B05
:1084D8001A88084B1A80237843F00103237010BDD3
:1084E800101100201611002018110020781000200B
:1084F800E8100020642700201C4B1B681B0307B5ED
:1085080030D51B4A1B4BD2ED007A1B788DF8003012
:10851800B2EE047A67EE877A174B9FED187A1B78CC
:108528008DF80130FCEEE77A0A2017EE903AD2ED8A
:10853800017A8DF8023067EE877A6946FCEEE77AB1
:1085480017EE903AD2ED027A8DF80330FCEEE77A16
:1085580017EE903A8DF80430094B1B788DF80530EA
:10856800FEF7E6F803B05DF804FB00BFFC27002027
:1085780010280020EE2700200C28002000007A4454
:10858800F2270020054A137883F001031370044A88
:1085980000231360034A1360AEE700BFF2270020F0
:1085A8000828002004280020094A13781844C0B27B
:1085B80010F0800F18BF803810701346054A1978DC
:1085C8001378994201BF00231370014A1370704752
:1085D800692700206827002010B50A4B0A4A1B7833
:1085E80042609C18094A046012789A4225BFD31A3F
:1085F8000B60C3F1800300232EBF4B600B604A6001
:1086080010BD00BF692700206A27002068270020C6
:108618001FB5684602A9FFF7DFFF044B02981B68E5
:1086280003440398184405B05DF804FB28060020AD
:108638002DE9F04F89B082460193002302910392FD
:108648009946039A934205DA029A52F82320013395
:108658009144F6E7019B4D46002B56D102F07AF97A
:10866800002852D101987CE002223F4E8DF81C2050
:108678001A0C4FF480578DF81D2006201A0A8DF821
:108688001E208DF81F3002F089F93785062008F082
:1086980043FD364BB76101221A700020378507A9C0
:1086A800042208F061FD029FD04626464FF0000BD9
:1086B800039B9B451EDABC4657F8042B4FEA8B03F5
:1086C800002A47D0B24235D332465AF80310CDF8C3
:1086D80014C00020049308F047FD049BDDF814C083
:1086E8005AF8032032444AF80320DCF800309E1B75
:1086F800CCF800601C4B4FF480529A611C4A1368F6
:108708002D1B1C44019B14604BB345B3184B1B68CD
:10871800DCB22A19B2F5807F164AD2688CBFC4F53C
:1087280080742C4693429FD3134A00231370134A34
:10873800137014E00020D8F8001008F015FD57F861
:10874800043CD8F80020F61A1344C8F80030002377
:1087580047F8043C0BF1010B08F10408A8E7C5EB46
:10876800090009B0BDE8F08F000400482506002084
:108778002806002010000020682700206927002014
:1087880030B50B4C0B4D22782B789A4285B00CD023
:10879800684602A9FFF720FF0123684602A90222C2
:1087A800FFF746FF00232B70237005B030BD00BFD4
:1087B800692700206827002030B50E4D0E4C2A7816
:1087C80023789A4285B011D0684602A9FFF704FFC2
:1087D800002302A902226846FFF72AFFFFF7E4FEFA
:1087E80020782B781B1A5842584100E0012005B028
:1087F80030BD00BF692700206827002038B50E4C1F
:108808004FF4805545F2082002F0C8F82585062067
:1088180008F082FC094BA56101221A70C720258542
:1088280008F07AFC064AA56100231370054A137004
:10883800054A136038BD00BF000400482506002023
:10884800682700206927002028060020FFF704BABF
:10885800FFF702BAFFF700BA026BC168034610B50A
:10886800406942B11A6C8C1A013A005D08BF0A4689
:10887800C0B21A6410BD1A6A805C01328A4228BFED
:108888000022C0B21A6210BD436B13B190F84400C5
:108898007047836A406A1B1A584258417047036BF5
:1088A80013B15B68016C01E0C369016A8B423CBF8C
:1088B800C2689B18581AC0B27047836A8169426BB4
:1088C8001944D160416A99429DBF0169CB1A53602E
:1088D800CB1A96BF0023536083624FF0000380F8E1
:1088E8004430136888BF816243F001031360704706
:1088F800436A8269D154436A02690133934228BFAB
:1089080000234362436B1BB11B68DB0705D4D4E724
:10891800026D136843F0800313607047F0B5046D6F
:108928008668236823F0010323608379054613F0E2
:10893800020F40790CBF4FF0000E4FF4005E13F0A9
:10894800040F14BF4FF48067002710F0010F14BF05
:10895800042100218307206820F00100206062685C
:1089680022F440524EEA02026260226822F4B053B6
:1089780023F00C0348BF41F008013B430B4323603D
:10898800A36895B023F44073A360684604F0E2F945
:10899800284B9C4201D10C9B0EE0274B9C4201D1F5
:1089A8000D9B09E0254B9C4201D10E9B04E0244B12
:1089B8009C420CBF0F9B109B2268A879170448BFE4
:1089C8005B00B3FBF6F206FB1233B3EB560F2368DA
:1089D80028BF01321E0441BF4FF6F073C2F34201B3
:1089E800134041EA03026B7992B213F0020FA2819D
:1089F80000F0010114BF4FF400320022DC0748BF29
:108A080042F480322B6D11B159680A4302E059686B
:108A180021EA02025A609A6801074CBF42F0080234
:108A280022F008029A601A6842F001021A6015B032
:108A3800F0BD00BF0038014000440040004800403D
:108A4800004C0040417169E7816067E7026D036B84
:108A580070B50446D5699BB9A90611D5C36A1BB17F
:108A6800908C80B298470BE0E169928C40694E1C6B
:108A7800D2B2E6614254E169E268914228BFE361FB
:108A8800616BA1B92A0612D5636AA26A9A42236D5C
:108A980009D0501CA669A062B25C1A852369984265
:108AA80005D3A16203E01A6822F080021A602B073E
:108AB80042BF236D08221A6270BD0D4B0D484FF45A
:108AC80000525A600C4A11684FF6FE730B4013604F
:108AD800426B11684FF6FE730B401360426A836A5B
:108AE8009A4200D0E9E6012380F84430704700BF7D
:108AF8000000024048260020440002402DE9F047CB
:108B08001E46A64B8CB09842894690469DF8505018
:108B180040F08580A24BA34A1A60A34A5A6102F525
:108B280080729A614FF48072DA601A619F4A1A6300
:108B3800143A5A63A2F54842203ADA6404329A6435
:108B4800C3F8088018659A4B9A6942F480429A6182
:108B58005A6942F001025A6102238DF80830032352
:108B680015F0010A8DF809304FF000038DF80A302E
:108B780014BF022301232C078DF80B3019D54FF0B1
:108B880090444FF4007701978AF001038DF80A307A
:108B9800636A23F0F0036362636A43F070036362FD
:108BA800204601A904F048FABAF1000F27D1A761BD
:108BB80025E0B00710D50CA94FF4007341F82C3DFF
:108BC8004FF09040436A23F0F0034362436A43F056
:108BD8007003436204F030FAF10710D50CA94FF482
:108BE800806341F82C3D4FF09040436A23F4706352
:108BF8004362436A43F4E063436204F01DFA0E23C0
:108C08008DF800300022012368468DF801308DF878
:108C180002208DF80330624C08F0DCFA0BE1654B5A
:108C2800984276D1644B5F4A1A604FF48072DA60DA
:108C38001A61624A5A6102F580729A615C4AC3F805
:108C480008801865D36943F40033D36102238DF893
:108C58000830032315F0010A8DF809304FF000039E
:108C68008DF80A3014BF022301232A078DF80B3030
:108C780019D54FF090444FF4804701978AF00103CB
:108C88008DF80A30636A23F070636362636A43F0A5
:108C9800E0636362204601A904F0CEF9BAF1000F3F
:108CA80027D1A76125E0B30710D50CA94FF480435D
:108CB80041F82C3D4FF09040436A23F070634362C3
:108CC800436A43F0E063436204F0B6F9F70710D54E
:108CD8000CA94FF4004341F82C3D4FF09040436AF3
:108CE80023F070434362436A43F0E043436204F075
:108CF800A3F926238DF800300022012368468DF859
:108D080001308DF802208DF803302B4C08F062FA00
:108D180091E02B4B984240F00F812A4B214A1A6070
:108D28004FF48072DA601A61274A5A6102F580723C
:108D38009A611F4AC3F808801865D36943F48023F1
:108D4800D36102238DF80830032315F0010A8DF84A
:108D580009304FF000038DF80A3014BF02230123B5
:108D68002C078DF80B3033D5184C4FF480670197DA
:108D78008AF001038DF80A30636A23F47063636232
:108D8800636A43F4E0636362204601A904F054F97E
:108D9800BAF1000F40D1A7613EE000BF00380140A2
:108DA80048260020648F01088013002058000240E4
:108DB8000010024000440040F425002080150020E7
:108DC80000480040A025002080170020000400482B
:108DD800B0070FD50CA94FF4806341F82C3D5848D3
:108DE800436A23F470634362436A43F4E063436273
:108DF80004F022F9F1070FD50CA94FF4006341F8EC
:108E08002C3D4F48436A23F470434362436A43F45A
:108E1800E043436204F010F927238DF80030002264
:108E2800012368468DF801308DF802208DF8033053
:108E380008F0D0F9434CC4F82C900027012384F89B
:108E480044302762E761A76267626671C4F80880E8
:108E5800A5712046FFF762FDF20734D5236B002B7E
:108E68002AD001A803F0FAFDE36C01934FF4805374
:108E78000A9380230693E368ADF810302023099302
:108E8800206B636902930B970597079708970397D9
:108E980003F00FFE01A9206B03F0EDFD236B216D9C
:108EA8001A6842F001021A608A6842F040028A6039
:108EB8005B689BB2236406E0236D20221A621A685D
:108EC80042F020021A60B3072FD5636B43B301A8A1
:108ED80003F0C4FDA36C01934FF480530A938023DD
:108EE80006932369ADF8103000251023606B0393B7
:108EF8000B95059507950895099503F0DAFD606BC4
:108F080001A903F0B8FD636B1A6842F002021A6007
:108F1800226D5D605D60936843F08003936004E0B8
:108F2800226D136843F080031360226D136843F0C9
:108F380001031360204600E000200CB0BDE8F08774
:108F480000040048A02500201FB50123ADF8083013
:108F58000023ADF80C30ADF80A30094BADF8041019
:108F68001B78ADF80620012B08BF032301A908BF11
:108F7800ADF80C3003F02BFE05B05DF804FB00BF24
:108F88002C0100202DE9F04F2DED028B85B007460E
:108F98000293A04B1B889807934636D5109B9E4892
:108FA800DC89B0F900301B1B03F2F31540F2E632FE
:108FB800954203D8002BB8BF5B4201E04FF4FA7327
:108FC800B0F90220121B02F2F31440F2E630844298
:108FD80003D8002AB8BF524201E04FF4FA72934214
:108FE800B8BF1346C3F5FA73052293FBF2F30A22BE
:108FF800643B53433A7FD2105343642293FBF2F30A
:10900800134423EAE373DBB200E064230093CB1C30
:109018000193B8460024019BDFF824A213F8016FDE
:109028000193022C4FEA440905D1BAF904301B36E2
:109038005E43761146E079493AF8142031F9141064
:10904800022012FB0011CBF10002914203DB5945CB
:109058000A46A8BF5A467249029B31F90950551B66
:1090680033F91420154409F03DF988B107EE905AF8
:109078006C4AB8EEE70AB2EE048A105D80EE080A80
:1090880008F034F920EE080AFDEEC07A17EE905A7F
:10909800604A1288D10712D43AF909301B365E4368
:1090A80093074FEA26160DD5BB7C5D439DF900302A
:1090B8005D43642395FBF3F506EB251602E03E7A43
:1090C80075432E11584B042533F9093093FBF5F5F8
:1090D800564BE25C924698F80120751B51466A434C
:1090E8004A43642192FBF1F297F85110D21108EE2D
:1090F800102AA9B1022CB8EEC80A08D14A0803D030
:109108009142A8BF114600E00121494802E0181D1C
:1091180000EBC400D3ED070A01F0B8FDBDEEC08A2C
:10912800DFF808E1434B98F80B6018880EF120032C
:1091380000FB05F253F82410D21206FB0216B6F50E
:10914800001F3D4AA8BF4FF400169642B8BF164606
:109158000EF12C0243F8246052F8243042F82450CF
:10916800EB1A0EF138014FF6FF720009B2FBF0F06E
:1091780043430EF1440051F8245050F8242040F89D
:1091880024509B112A4441F8243097F850101A446F
:109198004FEA840C761300EE102A79B10EF15000D4
:1091A800B8EEC00A00EBC400DEED070ACDF80CC02B
:1091B80001F06CFDDDF80CC0BDEEC00A98F8153062
:1091C80010EE102A18EE101A5A43534653431A4603
:1091D8003144642392FBF3F3184A1B12194422F812
:1091E800091018EE100A02F1080101344CF80100C8
:1091F80002F114012032032C4CF801604CF80230C3
:1092080008F101087FF407AF05B0BDEC028BBDE89B
:10921800F08F00BFD411002038280020223400200D
:10922800F42700207C8F01082C10002080190020D2
:1092380094190020001000200000E0FFE819002029
:10924800F01000202DE9F04F2DED028B85B08046FF
:109258000393BC4B02911C88019204F00204A4B24F
:1092680094B1B94BB3F90240B3F90030002CB8BF40
:109278006442002BB8BF5B429C42B8BF1C46B4F5A1
:10928800007FA8BF4FF40074C2460025AF4AAE4B1A
:1092980032F9152033F81510AD4882EAE27EAEEBBC
:1092A800E27E0BB2BEF5206F4FEA45094FEA430351
:1092B8004FEA850750F8256012DC4FF0040E92FB48
:1092C800FEF29A1A1644B6F57A5FA8BF4FF47A569A
:1092D800A04A9642ACBF40F8256040F8252002E03D
:1092E800002240F82520C6599AF80B20F61156435B
:1092F8009AF801205343934A12884FEAA31B930715
:109308004FEAA61654D0944A019B32F9092002204C
:1093180011FB00215A42914203DB8B42A8BF0B4646
:109328001A468E49039B39F90110511A33F9152051
:109338008B1808EE103A08F0D5FF68B1B8EEC80AE5
:10934800874AB2EE048A80EE080A505D07F0CEFF25
:1093580020EE080ABDEEC08A824883493A5818EEC2
:10936800103A42F2107E1A447245A8BF72468A42E9
:10937800B8BF0A463A5098F8081098F81C005943A4
:1093880000EB8000C911C0F1000E714503DB81427A
:10939800A8BF01468E4698F812104A431213CEEB26
:1093A8000B03B61A6643634302EB66260EEB632B88
:1093B800664A39F90210042291FBF2F16B4A02F174
:1093C8009C00405D4143ABEBA11398F8511008EEA7
:1093D800103A51B1101DB8EEC80A00EBC500D2ED25
:1093E800070A01F053FCBDEEC08ADFF880E1574B55
:1093F8000EF1A00139F8030039F9012029F801001C
:109408000FFA80FC0EF1A4010EF1AC00C2EB0C02C5
:109418003B584FF0040C92FBFCF257F801C07A500D
:10942800634498F8501047F800C0134400EE103A0F
:1094380059B10EF15000B8EEC00A00EBC500DEEDE0
:10944800070A01F023FCBDEEC00A484901F1B40245
:1094580010EE103A525D53435A1118EE103A01F1CA
:10946800680E9819801A01F1700329F80E0018EE99
:10947800100AF85001F17C035242FE5001F18803B2
:109488000AF1010AFA500B460DB90125FEE62E4AEB
:109498009C6AB2F90410029A92790F3252004A4338
:1094A80052112A49002AB1F904104FF0040091FB27
:1094B800F0F0A2EB0000B8BF5242322A98F80D1023
:1094C8000BDC2B4A01FB00418A42A8BF0A46294906
:1094D8008A42ACBF9A62996201E000229A6298F8C7
:1094E800031001FB00F22449097803294FEAA2126C
:1094F8000CD9B8F84E10B1F5FA7F07D2484282422B
:1095080003DB8A42A8BF0A4600E00246996A9A67C6
:1095180041F34F31B1F5807FA8BF4FF480716FF0F0
:10952800FF008142B8BF014650180022A3F86C0022
:10953800C3F88410C3F8902005B0BDEC028BBDE8D9
:10954800F08F00BFD4110020F01000202C10002054
:10955800A019002080C1FFFF22340020F42700203A
:109568007C8F0108141A0020F0D8FFFF8019002012
:10957800FEFFFF0F020000F0901F00202DE9F04FC2
:109588002DED028B87B000260593C54B0491B3F9E6
:109598000280B3F900300392B8F1000FB8BFC8F1E8
:1095A8000008002BB8BF5B429845B8BF9846B8F58D
:1095B800FA7F0746A8BF4FF4FA780090B1460196A3
:1095C800B3463446B74D2B88990758D0B44BB64AA2
:1095D80033F8143032F91420022013FB0022039BC5
:1095E8005B429A424FEA440103DB039B9342A8BFC4
:1095F8001346AE4A31F902A0059A32F91420CAEB93
:10960800030303EB020A08F06DFE88B107EE90AA87
:10961800A74BB8EEE70AB2EE048A185D80EE080A96
:1096280007F064FE20EE080AFDEEC07A17EE90AA55
:109638003B7A642203FB0AF393FBF2F33A7F6FF061
:10964800040101FB02FB5B4505DB02EB820293424E
:10965800A8BF13469B46974A52F824100AEB010309
:1096680042F210718B42A8BF0B4693498B42B8BF98
:109678000B4642F82430BA7C53431B1301932D88C0
:1096880005F00303012B38D0854B8C4933F914902E
:10969800009B51F824E093F801C0894B33F914007A
:1096A80080EAE073A3EBE073B3F5206F4FEA84061A
:1096B80016DC09EB89031A0192FBFCF3042290FBE8
:1096C800F2F0181A8644BEF57A5FA8BF4FF47A5EA6
:1096D8007C4B9E45ACBF41F824E041F8243002E0C1
:1096E800002341F824308B597D2693FBF6F6009B26
:1096F800DB7A7343402693FBF6F6AA0711D5019B44
:10970800C8F5FA7208FB09F008FB06F54FF4FA7180
:1097180002FB0B0002FB035590FBF1F095FBF1F502
:1097280005E0EB074DBF019D354648465846644B5A
:1097380033F91420042392FBF3F3634A02F19C01EA
:109748004FEA440A615C4B436FF04F0193FBF1F31E
:1097580097F85110C31808EE103A51B1101DB8EE21
:10976800C80A00EBC400D2ED070A01F08FFABDEE7B
:10977800C08ADFF854E1524B0EF1B8013AF8030001
:109788003AF901302AF8010002B20EF1BC010EF1DB
:10979800C400D31A042293FBF2F2A30051F824C0A8
:1097A800029350F8243041F82420634497F850106D
:1097B80040F824C0134400EE103A59B10EF150009D
:1097C800B8EEC00A00EBC400DEED070A01F05EFA4D
:1097D800BDEEC00A3C4A02F1B40110EE103A095D30
:1097E80001FB03FE18EE101A02F1680029444FF03D
:1097F800200C9EFBFCF3C91A2AF80010029902F10A
:10980800700E084618EE101A40F80E1002F17C018E
:109818005B42455002F188014350009B013300939D
:109828000CB90124CEE61E4B946AB3F90410049BCC
:109838009B790F335B004B435B112149002BB1F936
:1098480004104FF0040091FBF0F0A3EB0000B8BF48
:109858005B42322B797B0BDC1C4B01FB00418B42BA
:10986800A8BF0B461A498B42ACBF9362916201E0D4
:1098780000239362F97801FB00F31649097803295C
:109888004FEAA31329D9B7F84E10B1F5FA7F24D2BD
:109898004842834220DB8B42A8BF0B461DE000BF35
:1098A800F0100020D411002022340020F4270020DA
:1098B8007C8F0108141A0020F0D8FFFFA01900209F
:1098C8002C10002080C1FFFF80190020FEFFFF0F31
:1098D800020000F0901F00200346916A936741F34D
:1098E8004F31B1F5807FA8BF4FF480716FF0FF0052
:1098F8008142B8BF014658180023A2F86C00C2F88C
:109908008410C2F8903007B0BDEC028BBDE8F08F30
:109918002DE9F04F2DED0A8B85B08346039390F81F
:109928005030029101921BB1322BA8BF322300E0C4
:10993800012307EE903AF8EEE7BADFEDDE7ADE4B68
:109948009FEDDECA1B88C7EEABBA002B08BF012308
:1099580007EE903AB8EEE7AAD94B2AEE0CCA1B8854
:109968007BEE8CBA9807CCEE2BBA27D5D54AB2F93C
:109978000030B2F9022083EAE37182EAE270A1EBD7
:10998800E371A0EBE27088420446B8BF0C46B4F518
:10999800E17F16DA88429FEDCCBA05DD002AD8BFF0
:1099A800524207EE902A04E0002BD8BF5B4207EE34
:1099B800903AF8EEE77A87EE8BBA04E09FEDC3BAE7
:1099C80001E0B7EE00BAC24EDFEDC09ACDF800B0A4
:1099D80006F1080806F1100906F11C050024F0EE4E
:1099E80069AABC49DFF8D8A231F91430B54909EEA3
:1099F800103AB8EEC99AF5EE047A29EE279A31F9A9
:109A08001430BAF80010BDEEC99A08EE103AF8EE14
:109A1800C97A9FEDB19A89074FEA440727EE899AD8
:109A2800B8EEC88A00F08180AC4931F9143007EEED
:109A3800903AF8EEE77AB0EE007AE8EE077A019B02
:109A48005842FDEEE77A17EE901A814203DB8B420B
:109A5800A8BF0B461846A249039B795E401A33F902
:109A68001410084407EE900AF8EEE78A08F03AFC6A
:109A780048B19C49F2EE049A88EEA90A085D07F0FD
:109A880035FC60EE298A9BF81C30DFED976A0AEEF8
:109A9800903A9BF8083007EE903AF8EE677AF8EEBD
:109AA8006AAA68EEA77AB1EE047A67EEA67A2AEE79
:109AB800877AFDEEE77A17EE901AF1EE477AFDEE17
:109AC800E7AA1AEE903A994208DBFDEEC7AA1AEE09
:109AD800903A8B42A8BF0B460AEE903AD5ED007A31
:109AE800E8EE8C7ABBEE0E7AF4EEC77AF1EE10FA55
:109AF800F8EEEAAA09D4B3EE0E7AF4EE477AF1EE5C
:109B080010FAC8BFF0EE477A01E0F0EE477AC5EDEB
:109B1800007A9BF8123009EE903AF8EE699A67EEEF
:109B2800A97ADFED729A67EEA99ABAF80010CA0707
:109B380053D46848385E0028B8BF4042B0F5206F5B
:109B480003DD0020C9F8000026E0009B9FED687A3D
:109B58005B7868EE077A07EE103AB8EE477A87EE38
:109B6800877AD9ED007A37EE497AE7EE0C7A9FEDDD
:109B7800617AF4EEC77AF1EE10FA09D49FED5E7AB5
:109B8800F4EE477AF1EE10FAC8BFF0EE477A01E03A
:109B9800F0EE477AC9ED007A009BD9ED007ADB7ABE
:109BA80008EE903AF8EE688A8B0768EEA77ADFED40
:109BB800538A67EEA88A14D538EE6A8AF0EE6A7A74
:109BC800EBEE087A78EEE98AB0EE678AF0EE697A09
:109BD800EBEE287AF0EE678A03E0F0EE698AB0EEE1
:109BE8006A8A474B9FED477A03F19C01625C9BF8B8
:109BF800511007EE902AF8EEE77A67EEC97AA7EED9
:109C0800878A51B1181DB0EE480A00EBC400D3EDA5
:109C1800070A01F03BF8B0EE408A96ED007ADFF8CB
:109C2800E0A0D8ED007AA6EC019A39EE477A0AF15D
:109C3800B40187EE0C7A635C09F10409043509EE76
:109C4800103A37EE677AB8EEC99AEBEE877A38EEB3
:109C5800280AE8EC017A67EE897A9FED2B9A27EEBD
:109C6800899A30EE490A0CF0F1FB0AF16801BDEE61
:109C7800C88AC85318EE103A0AF17001FDEEE88A56
:109C8800B1EE499A41F82430BDEEC99A0AF17C0137
:109C980018EE903A41F8243019EE103A0AF188018A
:109CA800574641F82430009B0133009374BB0124CC
:109CB80097E600BF83F9223E00100020BD378635A5
:109CC800D4110020F01000200000E1430000000043
:109CD8004C1A00202C100020CDCC4C4022340020FF
:109CE800F42700207C8F01086F12033C0AD7A33D9C
:109CF8000000A043000040C3000040430AD7233CB3
:109D080080190020A69B443BF7CC9238029A584B06
:109D18009479B3F90430640028345C43554BB3F9A3
:109D2800043000EE103ABAEECF0A0CF08FFB641143
:109D3800201A002C07EE900AB8BF6442322CF8EEC5
:109D4800E76A03DD0023CAF8283029E0BDEECAAA75
:109D58001AEE103A23F0030307EE903AB8EEE7AA9A
:109D6800DFED457A9BF80D30CAEE277A07EE103AF8
:109D7800B8EE477ADAF8283026EE877A67EE277A3F
:109D8800FDEEE77A17EE902A13443C4A9342A8BFA7
:109D980013463B4A9342ACBFCAF82830CAF8282079
:109DA800BB6A5B13B3F5807FA8BF4FF480736FF075
:109DB800FF029342B8BF134607EE903AF8EEE78ADF
:109DC800FDEEE67A9BF8032017EE903A53439B1179
:109DD80007EE903A2B4B1B78032BB8EEE78A14D981
:109DE800BBF84E20B2F5FA7F0FD2FDEEC87A534287
:109DF80017EE901A994204DB914217EE903AA8BFE9
:109E0800134607EE903AB8EEE78A9BF8511079B1FD
:109E18004B0803D09942A8BF194600E00121B0EED3
:109E2800480A1948D7ED070A00F030FFB0EE408A1B
:109E380038EE280ABDEEC00A8DED000ABDF90030E3
:109E480000EE103AB8EEC00A0CF000FBBDEEC88A6E
:109E5800FDEEE88A0023A7F86C0087ED1E8AC7ED9F
:109E6800218AC7F8903005B0BDEC0A8BBDE8F08FA9
:109E7800F01000202C10002000803B45FEFFFF0F53
:109E8800020000F0901F00209419002038B5294DD9
:109E98002DED048B95ED008AB0EE480A044601F0DA
:109EA800BBF9F0EE408AB0EE480A01F052F995EDA0
:109EB800019AB0EE408AB0EE490A01F0ADF9F0EE31
:109EC800409AB0EE490A01F044F994ED017AD4EDD4
:109ED800027A94ED006A68EE676A27EE088AE7EE70
:109EE800286A68EE000A67EE807AE6EE290AB0EE84
:109EF800660AE7EEA80A0CF0ABFBDFED0F7A0F4B12
:109F080020EE270ADFED0E7A80EE270AD3ED3C7AA1
:109F180030EE270AF2EE047A80EE270A0CF096FA61
:109F2800BDEC048B83B21A0444BF00F5B47083B24D
:109F380018B238BDF42100200000E1448019002047
:109F4800DB0F494001380A4B042804D8DFE800F049
:109F58000507090B0D00074A08E0074A06E0074A0B
:109F680004E0074A02E0074A00E0074A1A6070471F
:109F780084000020112301088D8F00083D26010868
:109F88004D9200088595000819990008437913F047
:109F980001031FBFC36803F1FF32C369006A1DBF15
:109FA800181A1040C0B21846704790F83B3210B5E6
:109FB8007BB990F83A3290F83942A34209D2B0F806
:109FC800401201229A400A430133A0F84022DBB232
:109FD800F3E710BD8379DB07D0F8343144BFB1FA19
:109FE80081F149095A681B8909B193617047138542
:109FF80070476E4B6E4A9FED6F7AD2ED007ADFEDB7
:10A008006E4ADFED6E3A30B51C88B3F90AE01D8A56
:10A0180006EE904AB8EEE76AF8EE666ADFED687A0F
:10A02800B3F9044067EEE67AB7EE004AE6EE077A3F
:10A038009FED647A67EE666A9FED637AE6EE076ADB
:10A0480027EEA77A07EE904AB3F902409FED5F6AC0
:10A05800F8EEE77A67EE277A07EE104AB8EEC77A85
:10A06800DC89E6EE877AB6EE007AFDEEE76A87EEDF
:10A07800866AC3ED066AF8EEE66AD2ED017A9A8935
:10A08800E6EE874A06EE90EAB3F908E09FED507ACB
:10A0980005EE90EAF8EEE66AF8EEE55A66EEA46A8E
:10A0A80065EEA45A66EEA46AB3F806E0E6EE875AAF
:10A0B80065EE875AA5EEA34AF0EE445A04EE10EA7C
:10A0C800B8EE444A25EE844AB5EE404AF1EE10FA5D
:10A0D8005BD02DB205EE905A24B224EEA45A07EEB6
:10A0E800104AF8EEE55A12B265EE255AB8EEC75A8C
:10A0F80065EEA35A64EE854AB0EE007AE4EE875A1C
:10A10800B5EE007A65EE875A07EE102AB8EEC75A00
:10A118009FED307ADFED306AB3F91620E5EE075A85
:10A12800F8EEE77A9FED2D7A76EEE77ADFED2C6A86
:10A13800E5EEC77A05EE902AB0EE677ADFED297A68
:10A14800B3F91420B3F9123067EE277A07EE102A14
:10A15800C7EE847AF8EEE55AB8EEC77A65EEA75AE4
:10A1680027EE877A65EEA75A27EE237AA5EEA67A18
:10A17800F0EE476A07EE103AB8EEC77A36EE877AFD
:10A18800DFED196AE7EE267A01E0DFED187A18B1FB
:10A19800FDEEE77AC0ED007A31B1FDEEC67A6422B1
:10A1A80017EE903A53430B6030BD00BF9802002071
:10A1B800741A00200000003700007AC70000003839
:10A1C800000000390000803A000080380000A045F7
:10A1D80000000036000080470000804900008039F8
:10A1E800000000300050C3450000803D0000000022
:10A1F800704770471FB50123ADF80830ADF804105B
:10A20800002301A9ADF80A30ADF80C30ADF80620EE
:10A2180002F0DDFC05B05DF804FB38B5A0F5137459
:10A228006379A579DB0744D594F8383205F0010540
:10A23800EBB1226B1068C36A5B08436294F83C3246
:10A2480023B1B4F842320133A4F84232917A6A0059
:10A25800FFF7D0FF012384F83B32002384F839321A
:10A2680084F83A3284F83832A4F8403238BD94F889
:10A278003B32012B04BF94F8393284F83A32204635
:10A28800FFF793FE94F83B22236B3AB9012284F836
:10A298003B221868997A05FA02F207E0002284F84E
:10A2A8003B2295421868997A08BF0222BDE83840D7
:10A2B800A0E738BD10B5A0F5127494F83C22BAB9DD
:10A2C800A36A616A994228D0591CA069A162C35C3B
:10A2D8002069DBB25B0043F400738142A4F83E328C
:10A2E8004FF00A0384F83D3228BFA262012312E02E
:10A2F80094F93D327BB1B4F83E124B08A4F83E32D3
:10A30800204601F00101FFF765FE94F83D32013B5C
:10A3180084F83D3201E084F83C3294F83832002B5E
:10A328004ED194F839320133DBB2092B84F8393233
:10A3380003D12046BDE8104037E60A2B40D194F8F7
:10A348003B322BB9B4F8403243F00103A4F8403251
:10A358006379D9071CD5B4F84002820501D4C30734
:10A3680005D4B4F844320133A4F8443210E0E36A67
:10A37800C0F347000BB198470AE0E3696269D0541B
:10A38800E369E1680133B3FBF1F201FB1233E361E6
:10A39800012284F8382294F83B220023012A84F809
:10A3A80039320DD1A27984F83B32236B12F0010FB8
:10A3B8001868997A0CBF02220022BDE8104019E7FC
:10A3C80010BD7620F421312205F0C6B913B5062256
:10A3D80004466B4603211E2005F042F99DF8002033
:10A3E8009DF801309DF8021043EA02231BB21B4A74
:10A3F80007EE903A92ED007AF8EEE77A67EE877A00
:10A4080092ED027AFDEEE77A17EE903A23809DF8F6
:10A41800033043EA01231BB207EE903AF8EEE77ADD
:10A428009DF8041067EE877A92ED017AFDEEE77ADF
:10A4380017EE903AA3809DF8053043EA01231BB23A
:10A4480007EE903AF8EEE77A67EE877AFDEEE77A5C
:10A4580017EE903A638002B010BD00BF24000020C0
:10A4680007B5F7216B460622762005F0F9F89DF826
:10A4780000309DF801100C4A1B0343EA01139DF8B4
:10A48800021043EA111353609DF803309DF804103D
:10A498001B0343EA01139DF8051043EA11131360E7
:10A4A80003B05DF804FB00BF741A00201FB5044612
:10A4B80002210C2001220DF1070305F0D1F8C8B3E1
:10A4C8009DF80730DB0735D50321062202AB0C20A7
:10A4D80005F0C6F80C20092101220DF1070305F04B
:10A4E800BFF838B39DF8073013F00C0F22D19DF850
:10A4F80009209DF8083043EA0223C3EB83339B000D
:10A508009DF80B2023809DF80A3043EA0223C3EB11
:10A5180083339B009DF80D2063809DF80C3043EA3F
:10A528000223C3EB83339B00A3800C200A21012262
:10A5380005F012F904B010BD07B50A2100220C205D
:10A5480005F00AF9142001F078FA0A210F220C20EC
:10A5580005F002F90A2001F070FA01AB102103227C
:10A568000C2005F07DF80A2001F067FA0A21002284
:10A578000C2005F0F1F80A2001F05FFA0DF1030351
:10A58800022101220C2005F06BF80DF103030921CB
:10A5980001220C2005F064F80A2101220C2005F0A4
:10A5A800DBF803B05DF804FB074B1B681869074B21
:10A5B80020F01F0200F01F01D25801238B401A42DD
:10A5C80001D002F03FBA7047B802002014040140DD
:10A5D8002DE9F0437C4A136887B0904693B11A6816
:10A5E8001AB17A49486902434A619A88ADF800204D
:10A5F80002228DF803209868002269468DF802200F
:10A6080004F018FF322001F018FA002111221E2050
:10A6180005F0A2F8012160221E2005F09DF86420B3
:10A6280001F00BFA02A8FFF7D1FE00240A272646FC
:10A638002546022101221E2005F08EF8322001F065
:10A64800FCF902A8FFF7C2FEBDF90820BDF90A10FF
:10A65800BDF90C308A421444A8BF0A4693421D44EF
:10A66800A8BF134613F5805F0E4404DD013FE0D117
:10A678004FF0010901E04FF000091E2000211222CD
:10A6880005F06AF80A27022101221E2005F064F865
:10A69800322001F0D2F902A8FFF798FEBDF9082090
:10A6A800BDF90A10BDF90C308A42A4EB0204A8BF18
:10A6B8000A469342A5EB0305A8BF134613F5805F2E
:10A6C800A6EB010602DD013FDDD101E04FF00009F4
:10A6D80007EE904A9FED3E7A3E4FF8EEE77A00216A
:10A6E800C7EE277A70221E20F0EEE77AC7ED007ACF
:10A6F80007EE906AF8EEE77AC7EE277A9FED367A8A
:10A70800F0EEE77AC7ED017A07EE905AF8EEE77AAD
:10A71800C7EE277AF0EEE77AC7ED027A05F01CF863
:10A72800012120221E2005F017F81E2002210022F8
:10A7380005F012F8642001F080F9B9F1000F04D196
:10A748004FF07E533B607B60BB60D8F800301E4CF6
:10A758001A7B002A35D01A7D002A32D01B498A6913
:10A7680042F001028A61187B197D02F01BFA236806
:10A778009A689B88128A134223D0184801F002FA7B
:10A788002368186902F05EF923681B6904930026A0
:10A798000C23012504A88DF815308DF814608DF868
:10A7A800165006F035FD23688DF806605B7D8DF840
:10A7B800043001A803238DF805308DF8075006F002
:10A7C80009FD07B0BDE8F083B80200200010024080
:10A7D80000406F462400002001C05E46B1A5000875
:10A7E8002DE9F04F544D1E464FF4147305F108043B
:10A7F800434385B080469146E718A24610B92B44DA
:10A808004E4A03E0012805D14D4A2B449A63103281
:10A81800C3F83C214FF4147303FB08F3EC180AEB5C
:10A82800030203F59C734748A060343253446163C4
:10A83800E261236200224FF0010B4FF48071D4F8DB
:10A848003C3161610320A2626262A1612263E2621B
:10A8580084F8442284F840B284F84122A4F84A22B9
:10A86800A4F84C22C4F810906073A67384F84E8242
:10A8780004F59C7258681B8901924FF0020C03A9D9
:10A88800ADF80C308DF80EB08DF80FC0CDF800C0C3
:10A8980004F0D0FDA36BDDF800C0597B58681B8914
:10A8A8008DF80E1003A9ADF80C308DF80FC004F028
:10A8B800C1FD59463846FFF78DFB322001F0BDF83F
:10A8C800019A214BD2F804B0B3FBF9F1B1F5803FFE
:10A8D80003D3012BF8D95B08F6E74FF4147404FB93
:10A8E80008F805EB0809584689B2482208F5127895
:10A8F80005F0ACFA0AEB0804144BC9F850320022F0
:10A908005846214605F0F8FAD9F8385016F0010FE4
:10A918000CBF022200222868A97AFFF76BFC0C4BB7
:10A92800C9F854322846211D002205F0E5FA3846B8
:10A9380005B0BDE8F08F00BF741A002080A601089A
:10A94800A0A60108808F010800A24A04BDA2000841
:10A9580023A200080F4B73B518781C4698B105233D
:10A968000D4D8DF800304FF4805600238DF80130DE
:10A9780001A82E856946022206F0F6FBAE619DF815
:10A98800050000F0010000F00100207080F00100D7
:10A9980002B070BD2506002000040048064B70B5C3
:10A9A8001D6806461C46FFF7D5FF18B923685B1BD0
:10A9B800B342F8D970BD00BF20280020F7B50323A3
:10A9C8008DF80430030C8DF805308DF80700030A64
:10A9D80006200F4614468DF80630FFF7DFFF78B1E2
:10A9E800084D4FF4805601A904222E85002006F058
:10A9F800BBFB38460021224606F0B6FBAE61204676
:10AA080003B0F0BD00040048024640213C2004F099
:10AA1800A3BE70B500EB8000094CA0F1A1059C38DD
:10AA280025440444074B15F8010F1E787040FFF7C2
:10AA3800EBFFA542F6D13046BDE87040E4E700BF21
:10AA4800988F01082B34002010B5441E14F8010F0C
:10AA580010B1FFF7DEFFF9E710BD024680213C2068
:10AA680004F07ABE10B5D420FFF7F7FF8020FFF777
:10AA7800F4FFA820FFF7F1FF3F20FFF7EEFFD320F8
:10AA8800FFF7EBFF0020FFF7E8FF4020FFF7E5FFA7
:10AA98008D20FFF7E2FF1420FFF7DFFFA120FFF76B
:10AAA800DCFFC820FFF7D9FFDA20FFF7D6FF122016
:10AAB800FFF7D3FF8120FFF7D0FFCF20FFF7CDFFAF
:10AAC800D920FFF7CAFFF120FFF7C7FFDB20FFF708
:10AAD800C4FF4020FFF7C1FFA420FFF7BEFFA62058
:10AAE800FFF7BBFFAF20FFF7B8FFA620FFF7B5FFC2
:10AAF800AE20FFF7B2FF2020FFF7AFFF0020FFF7DF
:10AB0800ACFFB020FFF7A9FF4020FFF7A6FF002009
:10AB1800FFF7A3FF1020FFF7A0FF4FF48064013C6C
:10AB28000020A4B2FFF770FF002CF8D18120FFF7B6
:10AB380094FFC820FFF791FFAF20FFF78EFF012099
:10AB480010BD08B55038C0B2FFF787FF0020FFF7E7
:10AB580084FF1020BDE808407FE7503910B504464F
:10AB6800C8B2FFF77AFF04EB4400400004EB44044A
:10AB780000F00E00FFF771FFC4F3C3001030BDE80A
:10AB880010406AE7F0B50124B0FBF4F58D4201D31B
:10AB98004C43F9E70026D4B1B0FBF4F504FB1500EB
:10ABA800B4FBF1F41EB9002D01DC002CF3D1092D02
:10ABB80003F1010EEFB204DD002A14BF3725572533
:10ABC80000E030253D441D7001367346E3E71C70F4
:10ABD800F0BDF0B50124B0FBF4F58D4201D34C4330
:10ABE800F9E70026D4B1B0FBF4F504FB1500B4FB7B
:10ABF800F1F41EB9002D01DC002CF3D1092D03F16D
:10AC0800010EEFB204DD002A14BF3725572500E0F6
:10AC180030253D441D7001367346E3E71C70F0BDD6
:10AC280003685A1C0260197070472DE9F843089EA2
:10AC3800002B07468846144614BF4FF030094FF0E2
:10AC48002009334613F8012B0AB9254603E0002CE6
:10AC5800FBDD013CF6E7002D04DD38464946C047D8
:10AC6800013DF8E724EAE4743546A01B284415F8AA
:10AC7800011B11B13846C047F7E7BDE8F883024B1E
:10AC8800186800F09EBF00BFF00F002090ED017A19
:10AC980007EE901AB5EE407AF1EE10FA01BFF8EE21
:10ACA800E77A9FED0E7A67EE877AB7EE007A04BFEF
:10ACB800C7EE277AC0ED017A90ED017AD0ED007ADF
:10ACC80030EE877A30EE670AC0EE870AE0EE807AC7
:10ACD800B0EE670AC0ED007A704700BFDB0FC940CD
:10ACE80010B50278202A034600F10100F9D0092A9C
:10ACF800F7D02D2A03D10346BFEE000A04E02B2A21
:10AD080008BF0346B7EE000ADFED387A1A46134645
:10AD180012F8010BA0F13001CCB2092C0AD807EEC9
:10AD2800101AB8EEC77AF2EE046AA7EEA67AF0EE29
:10AD3800477AECE72E2816D1F2EE046A1146B0EEF7
:10AD4800666A0B4611F8012B303AD0B209280AD8A6
:10AD580007EE102AB8EEC77A87EE267A66EE866A7C
:10AD680077EE877AEDE71A7802F0DF02452A35D1C7
:10AD78005A782D2A02D10233012004E02B2A14BF6D
:10AD8800013302330020013B002213F8011F303940
:10AD9800CCB2092C03D80A2404FB0212F5E7B2F559
:10ADA8009A7F28BF4FF49A721346B7EE007A072BA2
:10ADB80005D9DFED0F6A083B27EE267AF7E702F0A0
:10ADC80007032BB1F2EE046A27EE267A013BF8E777
:10ADD800F0EE476A20B1C7EE877A03E0F7EE006A23
:10ADE80067EEA67A20EE270A10BD00BF000000001B
:10ADF80020BCBE4C30B52DED028B87B0B0EE408A3A
:10AE08000C220021054603A80BF011F9B5EEC08A03
:10AE1800DFED2A7AF1EE10FACCBF38EE278A38EE49
:10AE2800678ADFED277A28EE278A6946FDEEC87A19
:10AE380017EE904A84EAE470A0EBE47006F090FC08
:10AE4800002CACBF20232D2368468DF80C300BF066
:10AE580032F9012807D130238DF80D308DF80E30E6
:10AE68008DF80F300CE0022805D130238DF80D3015
:10AE78008DF80E3004E0032804BF30238DF80D3020
:10AE8800694603A80BF0FAF803A80BF014F9033885
:10AE9800C4B2224603A928460BF03AF900232B55E1
:10AEA800284608490BF0EAF803AB284619190BF0B5
:10AEB800E5F8284607B0BDEC028B30BD6F12033AA7
:10AEC80000007A4454AE010870B506461546084697
:10AED800B6FBF2F414B12046FFF7F6FF05FB146445
:10AEE800024B1B5D00F8013B70BD00BF56AE010868
:10AEF8002DE9F04F814689B08A4616461C46002542
:10AF08003178002900F0DD80252902D00136484635
:10AF180075E07278302A08BFB278A2F1300319BF01
:10AF2800B71C4FF0000BF71C4FF0010B092B4FF02B
:10AF3800000819D8A2F13003D9B2092905D80A2284
:10AF480002FB083817F8012BF4E7A2F16103052B7F
:10AF580002D8A2F1570305E0A2F14103052B03D85B
:10AF6800A2F137030A2BEADD6C2A31D13A78642A38
:10AF780007F1010600F083800BD8252A3DD003D8BD
:10AF8800002A00F09E80BBE7582A0CD0632A19D00B
:10AF9800B6E7732A22D002D86E2A37D0B0E7752ACE
:10AFA8005CD0782AACD1271D2068A2F158046242EF
:10AFB8004FF01001624155E02CD9582A32D0632A4B
:10AFC8002AD13E4648462178271DD04701350FE053
:10AFD800642A64D00ED9732A14D13E46236800939C
:10AFE8004846514642460023FFF71FFE271D0544E9
:10AFF8003C4685E7252ADFD13E4648462521D047ED
:10B0080001357DE70AD86E2A06D13E462368043406
:10B018001D6075E7002A54D03E4671E7752A26D090
:10B02800782AF9D1A2F1580304F1040C5A42206895
:10B03800CDF80CC04FF010015A4105ABFFF7A2FD47
:10B04800DDF80CC03E46644605AB009348465146C1
:10B0580042465B46FFF7E9FD054451E72068271D96
:10B068000A21002205ABFFF7B4FD3C46ECE704F1EA
:10B07800040CCDF80CC020680A210022DDE7206806
:10B08800002804F1040708DA2D238DF81430404213
:10B098000DF115030A210022E5E705ABFAE7206860
:10B0A800002804F1040C0ADA2D238DF814304042EC
:10B0B8000DF11503CDF80CC00A210022BEE705AB3F
:10B0C800F8E7284609B0BDE8F08F0EB40FB505AB18
:10B0D800019053F8042B0649039301A8FFF708FFD2
:10B0E800019B00221A7004B05DF804EB03B07047AE
:10B0F80029AC00080FB413B50B4904AB08680B4919
:10B1080053F8042B09680193FFF7F2FE0446084B35
:10B11800186800F04AFD0028F9D0204602B0BDE8C2
:10B12800104004B0704700BF040100200001002057
:10B13800F00F002080EAE073A3EBE0738B4206DB9C
:10B14800002801DD401A704702D0084470470020EB
:10B158007047FDEEC07A17EE903A2033402B43D863
:10B16800DFED237AB4EEE70AF1EE10FA04DDDFED45
:10B17800217A30EE670AF3E7DFED1F7AB4EEE70ACB
:10B18800F1EE10FA04D5DFED1B7A30EE270AF3E76B
:10B19800DFED1A7AB4EEE70AF1EE10FA04DD30EECC
:10B1A800670A37EEC00A0AE09FED157AB4EEC70ABF
:10B1B800F1EE10FA44BF30EE270A37EE400A60EE8F
:10B1C800007ADFED106A9FED107AA7EEA67ADFED20
:10B1D8000F6AE7EE876A9FED0E7AA7EEA67A20EE51
:10B1E800276AA6EE070A70479FED0A0A704700BF54
:10B1F800DB0F4940DB0FC940DB0F49C0DB0FC93FFC
:10B20800DB0FC9BF9A7C2E36FAAF4FB93587083C99
:10B21800A4AA2ABE00000000DFED027A30EE270A59
:10B2280097E700BFDB0FC93F38B52DED068B90EDD2
:10B23800008AB0EE480A0C460546FFF7EDFFB0EE6F
:10B2480040AAB0EE480AFFF784FFD5ED018AB0EEB8
:10B25800409AB0EE680AFFF7DFFFB0EE408AB0EE22
:10B26800680AFFF776FFD5ED02AAF0EE408AB0EE45
:10B278006A0AFFF7D1FFF0EE409AB0EE6A0AFFF7CC
:10B2880068FF60EE0A6A69EE297AF0EE665AE7EE20
:10B29800A85A29EE8A6A29EE007A69EE889A29EE78
:10B2A800489A28EE400A28EE0A8AC4ED035AF0EEBE
:10B2B800465AE7EE685AE6EEA87AA6EE687AC4ED32
:10B2C800009AC4ED028A84ED059A84ED088ABDECE3
:10B2D800068B84ED010AC4ED045A84ED067AC4EDA8
:10B2E800077A38BD10B52DED048B8AB090ED009A21
:10B2F800D0ED028A90ED018A0446084601A9FFF7BD
:10B3080093FFDDED047A9DED017A68EE277AE9EE88
:10B31800077A9DED077AE8EE877A9DED027AC4ED0B
:10B32800007ADDED057A68EE277AE9EE077A9DED79
:10B33800087AE8EE877AC4ED017ADDED067A28EE20
:10B34800278ADDED037AA9EE278ADDED097AA8EED2
:10B35800A78A84ED028A0AB0BDEC048B10BD074BA6
:10B368001A8822EA0000904210B518801C4602D0C4
:10B37800012000F0BDFB208810BD00BFD4110020C3
:10B38800064B1A881043904210B518801C4602D00C
:10B39800012000F0ADFB208810BD00BFD4110020B3
:10B3A800024A936823EA000090607047202C00202E
:10B3B800024A936818439060704700BF202C002011
:10B3C80008B5104B1A780023D9B2914207D20E491A
:10B3D80051F823100968002008600133F4E732208F
:10B3E80000F02BFB094B1B685A0309D5084B9B68D7
:10B3F8005B0305D440F2DC50BDE8084000F01DBBFB
:10B4080008BD00BF901F0020601F0020FC270020FF
:10B41800202C0020454A69232DE9F34113704FF48D
:10B42800FC635380BE231371EF2382F8DD370023BA
:10B4380082F8DE3719461646F25C0133B3F5FC6F25
:10B4480081EA0201F8D1394B83F8DE17384B1A69C3
:10B45800120604D5374A5A6002F188325A60042726
:10B468000020013F17F0FF074FD0314B3422DA603C
:10B47800002444B1002356F80480019301F036FA01
:10B488000428EED117E001F031FA0428E9D1284D5B
:10B498002B6943F002032B61274B6B612B6943F047
:10B4A80040032B6101F022FA2B69042823F00203E0
:10B4B8002B61DFD0D5E71E4D2B6943F001032B61CB
:10B4C80004F1006303F57E331FFA88F21A8001F055
:10B4D8000DFA042810D1194B23440193019B4FEA1C
:10B4E8001848A3F8008001F001FA2B69042823F01A
:10B4F80001032B6105D0B4E72B6923F001032B610D
:10B50800AFE70434B4F5FC6FB3D1094A13690428D2
:10B5180043F08003136102D105F0A1F910B90A20A4
:10B5280000F0FEFA02B0BDE8F08100BF202C002038
:10B53800002002402301674500F8030802F80308C9
:10B5480010B50E4C206800F0D9F92068047A002262
:10B5580002FB02F3193B634303F6C4135343192157
:10B5680093FBF1F3064921F812300132072AEFD193
:10B578000449BDE81040FCF7EBBA00BF701000208A
:10B58800C00F0020642D00202DE9F04105F067F977
:10B5980010B90A2000F0C4FAA44CA549A54D4FF4EF
:10B5A800FC6220460AF038FD94F8B437022B84BFB9
:10B5B800002384F8B43794F8B4274FF4CC7101FB16
:10B5C80002F3E018234400F53B70286093F8400329
:10B5D80003F54E73022801FB024284BF0020187253
:10B5E80092F84033944A13700C2202FB0343934AA7
:10B5F80003F2B6731360A26846F2090313401BB93D
:10B608004FF40050FFF7D4FEA368D80703D54FF4D2
:10B618000050FFF7C5FEA368590409D50820FFF7B5
:10B62800BFFE4FF40050FFF7BBFE0120FFF7B8FE46
:10B63800A3681A0706D54FF40050FFF7B1FE0120A2
:10B64800FFF7AEFEA3689B0402D54020FFF7A8FED3
:10B6580094F8DC21754B2AB193F8E02112B100224D
:10B6680083F8E021764B774E1E604FF0000C67465A
:10B6780004EB0C03B3F8F4E14FEA5E0101F0773113
:10B688004FEA9E0303F03333C1EB0E00C11A4FEAB1
:10B69800DE0303F01133CB1A03EB23131EF001086A
:10B6A80003F00F324FF0FF0392FBF3F3C3EB0323D6
:10B6B80018BF0137A2EB030318BFFFB2012B0ADD45
:10B6C800022B40F0B080B8F1000F00F0AC801EF003
:10B6D800BC0F00F0A8800CF1080CBCF1280FC7D1F2
:10B6E800013F012F00F29F80FFF72AFF302200213F
:10B6F8005548564F0AF09BFC554BD5F800801F6003
:10B70800544B002108F17900C3F8008000F036F9A5
:10B71800514B80F001001870504B07F126021A6057
:10B728004F4B07F1D8021A6098F80000FEF70AFCA0
:10B7380028684C4B00F5C5721A60FCF755FE4A4B59
:10B74800DFED4A6A07F194021A60494B00221A8019
:10B758009A71484B07F12C021A602B68464A93ED00
:10B76800187A03F219111160444A03F28911116021
:10B77800434A07F108011160424A1760424A07F13B
:10B788009C011160414A07F1A601116040495361CB
:10B7980067EE266A0E60B6EE007AB4F8661187EE98
:10B7A800267A101D07EE901AB4F86811F8EE677A39
:10B7B800C2ED027A07EE901A93F85C10117193F8B3
:10B7C8007810517194F8DF111174F8EE677AB3F8B4
:10B7D8001611C2ED037A07EE901A2E492E4A086018
:10B7E80003F1640111602D4A2D4982ED007AF8EECB
:10B7F800E77A9FED2C7A2C4A0B60C7EE277A2B4903
:10B808009FED2B7A67EE877AC2ED007A03F1680222
:10B818000A60284903F211130B60274B1F60274B5E
:10B828001A60BDE8F08101F035F85DE7202C0020B2
:10B8380000F803084810002060280020701000203D
:10B84800142C0020AA2D0020F40E0020642D0020C6
:10B85800280F00202C0F00200C000020442100207D
:10B8680004060020380F0020E80E0020DB0F4940B6
:10B87800340E0020A0210020BC24002064090020F0
:10B88800AC200020B0200020780800201C1F0020D9
:10B898003C090020D421002014220020102200207E
:10B8A8009807002000006144740800208C070020DD
:10B8B8004C3D0F44640800206C08002094060020CA
:10B8C80008B5FFF7A7FDFFF75FFE0120BDE80840B8
:10B8D80000F00EB9034B4FF4004208B19A6170476B
:10B8E8001A85704700080048034B4FF4004208B11E
:10B8F8001A8570479A6170470008004810B5447867
:10B908000078002202FB02F3193B634303F6C413D9
:10B91800534340F6C411434393FBF1F3034921F821
:10B9280012300132072AEDD110BD00BF341F0020AC
:10B938000430114B33F91000B0F5617F10B506DB08
:10B9480040F6330398420246A8BF1A4601E04FF476
:10B9580061720C78192340F2833013FB040494427B
:10B9680007DA497813FB01039342B4BF0020012092
:10B9780010BD002010BD00BF3828002010B500F110
:10B98800500302788A4203D18478C278944204D35F
:10B9980004309842F5D1002010BD012010BD1FB51C
:10B9A800084B1B681B030AD58DF8040001230D20E2
:10B9B80001A98DED030A8DF80530FAF7B9FE05B037
:10B9C8005DF804FBFC2700201FB5084B1B681B0310
:10B9D80009D58DF80400029100230D2001A98DF8E6
:10B9E8000530FAF7A5FE05B05DF804FBFC2700203A
:10B9F80010B5094A094B11689B6812689142F8D141
:10BA0800074A14694FF47A7000FB04F2D31AB3FBA7
:10BA1800F4F300FB013010BD2028002010E000E006
:10BA2800341F002038B50446FFF7E2FF0546FFF74C
:10BA3800DFFF401BA042FAD338BD10B504462CB135
:10BA48004FF47A70FFF7EEFF013CF8E710BD024AA9
:10BA5800136801331360704720280020054B5A698A
:10BA680010B51C4602B19047A36913B1BDE8104058
:10BA7800184710BD341F0020014B1B68184700BF32
:10BA88001034002010B50020FFF7F6FF054B002406
:10BA98001C7007F087F9044B1C771C629C849C621D
:10BAA80010BD00BF182C0020341F002010B510B99D
:10BAB800BDE81040E6E700230C225A430A4C11194E
:10BAC800125D824203D00133102BF5D110BD074B14
:10BAD800986A18B14A784078824203D20022996263
:10BAE8009A841A6210BD00BFAC970108341F002069
:10BAF80010B540001428A8BF14200023074A0221CB
:10BB080099540B4499181424834201F8014CF5DB2D
:10BB1800FF21D1540F20BDE81040C7E78C28002032
:10BB280038B540F2DB15124B082268439A61851E2E
:10BB38000B24013C14F0FF0412D00D4A938A9BB2E7
:10BB480083F0080393822846FFF777FF0120FFF769
:10BB580093FF1920FFF771FF0020FFF78DFFE8E73B
:10BB6800044B054A1A60054B054ADA6038BD00BF28
:10BB780000040048FC9F0020EFBEADDE00ED00E0B1
:10BB88000400FA0506494B690A4623B18B690BB1D3
:10BB98000F20C5E7012302EB83035861704700BFFC
:10BBA800341F002003685B69184703681B6918473E
:10BBB8000368DB68184703689B68184703685B6875
:10BBC800184703681B6818472DE9F84FB0F9023089
:10BBD800934218BF00232DED028B18BF0370057820
:10BBE80004460E469146002D40F08B8007EE902AC1
:10BBF8009FED770AF8EEE77AB6EE008A27EE800A1C
:10BC0800DFED747A20EE270AA04620EE080A0AF033
:10BC180093FCDFED716A60EE266AB7EE006AB0EE5B
:10BC2800667AA0EE007A40F2DC536365D0EE006AD3
:10BC38001023A4F8523037EE067A76EE866AC6EEFE
:10BC4800077A1823A4F85030274684ED046A27EEB3
:10BC5800807A27EE007A77EE075A84ED017AC4EDF0
:10BC6800025A70EE005A84ED037AB8EE007AA5EE17
:10BC7800807A27EE877A67EEA67A84ED057AC4ED96
:10BC8800067ADFED567A98ED047A27EE277AF0EEF9
:10BC9800678AB5EEC07AF1EE10FA4CBF77EE487AB3
:10BCA80077EE087A013517EE900A07F0F7F8D8ED25
:10BCB800017A67EEA87AC7E90E01F5EEC07AF1EECF
:10BCC80010FA4CBF77EEC87A77EE887A08F1040844
:10BCD80017EE900A07F0E2F8032DC7E9080107F10B
:10BCE8000807CED1A6F2DC531B042367E36763671A
:10BCF800C4F88030A367C4F884300123A4F8029004
:10BD08002370D4F85490B4F95280636A276A206F7C
:10BD1800E26FD4F840C0D4F88010C4F88020C9EB92
:10BD2800060606FA08F64FEAE67B734307FB0B3371
:10BD38002667A7FB06671F44636C656F60674FEA59
:10BD4800E27B53430CFB0B3EACFB02237344B61A55
:10BD580067EB0307E36AA26AC4F884104FEAE07B42
:10BD6800434302FB0B3EA2FB00237344B6185F411A
:10BD7800E36CA06CB4F95020A5674FEAE17B4B4314
:10BD880000FB0B33A0FB01011944636B361A206BCF
:10BD98004FEAE57B05FB03F300FB0B3367EB010779
:10BDA800A0FB050119448019794107F04DF808F105
:10BDB800FF3201239340E067C01841EBE37142462C
:10BDC80007F042F8BDEC028B4844BDE8F88F00BF8D
:10BDD8006F12833ADB0F4940F404B53F0000804BF3
:10BDE8002DE9F8430024234B93F85C60E0B2B0429D
:10BDF8000CD203EB8003204ADB6A32F810101BB127
:10BE08000B2801D8DB6898470134ECE71B4B1B680B
:10BE18005B032DD500242346E2B2B24228D2DFF8D4
:10BE2800549009F12C074FEA840857F824205568E4
:10BE38009D4215D0284604F033F8EFF312835022C0
:10BE480082F3128828216A6A01FB00900132C0F847
:10BE580084206A6942F001026A61DBB283F31188C7
:10BE680057F808301B6800221A6001342B46D3E7C4
:10BE7800BDE8F883341F00204C100020FC27002068
:10BE880008B50E4B1B6813F4805F0D4B14BFD3F835
:10BE98007821D3F87C2193F85C1092880023D8B2DB
:10BEA800884204D2074820F813200133F7E7FFF748
:10BEB80097FF3220BDE80840BFE500BFFC270020FF
:10BEC800341F00204C1000200A4B1A680A4B30B56A
:10BED80002F48052D3F87841D3F87C5100230AB198
:10BEE800A18800E0A988054820F8131001330C2B1D
:10BEF800F5D130BDFC270020341F00206228002027
:10BF080070B5124D0024214605F28110702285F883
:10BF180080410AF08CF82146D5F8F4310B4A0B44DD
:10BF280093F9020080B102F281141E680E510819BB
:10BF38009C8884809B79837192F880310731013322
:10BF4800702982F88031E7D170BD00BF341F00200E
:10BF5800094B1A680E2303FB0020437AFF2B07D0F6
:10BF6800064A12789A4203D9054A32F8130000E0CB
:10BF7800808800B2704700BFBC2400200C2300203A
:10BF8800382800202DE9F04F2DED048B944C954F67
:10BF9800D4F8FC31DFF850828DB0064692489847B5
:10BFA800914894F80C22014601F082F83B8804F588
:10BFB8001772002B73D0D4F810321B7808EE103AA1
:10BFC80004F5057904F508754FF0000AB7F800B0D4
:10BFD80038F91A00BBF57A7F02BF0023C9F8003090
:10BFE8002B61D9F800300344C9F800302B6907EEFB
:10BFF800900A0133012B4FEA4A01F8EEE77A2B61E8
:10C0080006D10023C5ED017AC5ED007AAB601BE0CF
:10C01800D5ED006A07EE103A37EEE66AB8EEC77A51
:10C0280086EE077A36EE877AD5ED026A85ED017AD3
:10C0380077EEC77A85ED007AE6EE276AF0EE667A43
:10C04800C5ED036AC5ED026A0023BBF1010F28F8AC
:10C05800013053522ED12B69012BC3BF03F1FF339B
:10C0680000EE103AD5ED037A9FED600AC8BFB8EE2E
:10C07800C00A8DE80600C8BF87EE800A0AF08CFC6B
:10C088009DE8060018EE103A5BB1F8EEC87AB4EEF7
:10C09800E70AF1EE10FA04DD4FF47A733B800023CF
:10C0A8001CE0D9F800304FF47A7003F5FA7393FB6B
:10C0B800F0F353520AF1010ABAF1030F09F1040926
:10C0C80005F1140582D1BBF1010F04D15846009245
:10C0D800FFF7ECFC009A3B88013BDFE738F81310C8
:10C0E80032F813003E4D091A28F813100133032BB8
:10C0F800F4D13F4F3B6813F0020300F0C9823D4B77
:10C1080005F262205B6898473B4B05F262201A787B
:10C11800014600F0CDFFB5F8683205F26229002B20
:10C1280041D0D5F86C020023B4F86822334939F9B4
:10C1380013E02B4DB2F5C87F04BF002241F823203D
:10C148004FEA830C51F80C20724441F80C2000216E
:10C1580029F8131020F813100133032BE4D1B5F894
:10C168006832012B1AD1D5F870324FF4C87EC83323
:10C1780093FBFEF30380D5F87422C83292FBFEF2DB
:10C1880042801F4AD5F878321288C83393FBFEF3F1
:10C198009B1A838031807180FFF792FBB4F8683274
:10C1A800013BA4F86832174B1B68590740F18D8092
:10C1B800B4F87C220A4B322A26D1D3F86C22118893
:10C1C800A3F87E1251889288A3F882223288A3F8B5
:10C1D80084227288A3F88012A3F8862216E000BF92
:10C1E800341F0020263400202C10002000000000FE
:10C1F8000C110020802800202C340020A4210020CD
:10C2080020000020FC270020002A3DD0D4F86CC272
:10C218000023B4F87C22AA4939F91300A94D322A1F
:10C2280004BF002241F823204FEA830E51F80E2064
:10C23800024441F80E20002229F813202CF813207C
:10C248000133032BE5D1B5F87C32012B17D10C2033
:10C2580085F8942285F89532FFF728FCD5F86C32DA
:10C26800B5F87E221A80B5F880225A80B5F8822265
:10C278009A80B5F884323380B5F886327380B4F882
:10C288007C32013BA4F87C3294F896328D4AE3B1B3
:10C29800D2F86C52D2F88802002182F896124FF038
:10C2A800320E90FBFEF02880D2F88C0290FBFEF054
:10C2B8006880D2F89032844A93FBFEF312889B1A66
:10C2C800AB8031807180FFF7FBFAD4F86C22B4F8A8
:10C2D800623211885B1AA4F862325188B4F8643269
:10C2E8005B1AA4F864329288B4F866329B1AA4F8F0
:10C2F8006632FFF77DFBD4F8983294EDA76AD4F83C
:10C30800A062C4F89802C3EB000A07EE90AAB8EE40
:10C31800678A002528EE066A96F800C06B486C49C3
:10C328000DF10C0E2A4638F9123007EE903AF8EE65
:10C33800E77A67EE867AEEEC017ABCF1000F1CD042
:10C3480007EE90CAF8EEE76AB7EE007AC7EE266AFB
:10C3580039F9123007EE903AF8EEE77A37EE667A56
:10C3680067EEA67AD1ED006AE6EE877AC1ED007A2B
:10C37800FDEEE77A17EE903A01E039F81230438083
:10C3880030F8023F0132032A13FB035501F104017F
:10C39800C9D1DFF834814F4864236B43B8F80050A3
:10C3A8006D4393FBF5F5493D03A9ADB2FEF79AFF3E
:10C3B8003B2DD6ED016A11D9B4F9BC32D4EDAE0AE1
:10C3C80007EE903AF8EEE77A434BF4EEE70AF1EE1F
:10C3D80010FA1EDD1A7842F008021DE0F7EE007A26
:10C3E80036EEA77A3B4A87EE877A00233B4931F934
:10C3F80013100133032B07EE901A92ED006AF8EE42
:10C40800E77AE6EE267A67EE877AE2EC017AEDD1F2
:10C41800D2E71A7822F0080294EDAD0A1A700AF0F1
:10C4280017F9B0EE409A84EDB00A94EDAE0AD4ED57
:10C43800AD7AD4EDAC8ADFED2A9A2A4D20EE000AB7
:10C44800F1EE688AA7EEA70A0AF0A6FAF0EE400A0B
:10C45800B0EE680A0AF0FCF8F0EE408A84EDB10A02
:10C4680029EE290A09F0F2FF28EEA90A288009F026
:10C47800EDFF3B6868801A073AD51B4803A9FEF709
:10C4880031FFD6ED026A184AF7EE007A36EEA77A3F
:10C49800002387EE877A154931F913100133032BEE
:10C4A80007EE901A92ED006AF8EEE77AE6EE267A41
:10C4B80067EE877AE2EC017AEDD10B4843E000BFE2
:10C4C800BC210020341F002020000020D8100020AC
:10C4D800D8210020E421002010110020DA100020CB
:10C4E8004C3D0F44F4270020FC210020321000208E
:10C4F8006D4D03A92846FEF7F5FE95ED010A95ED69
:10C50800007AD5ED027A20EE000AA7EE070AA7EE18
:10C51800A70A0AF041FAB5EE400AF1EE10FA11D076
:10C52800D5ED007AC7EE807AC5ED007AD5ED017AAF
:10C53800C7EE807AC5ED017AD5ED027A87EE800ADA
:10C5480085ED020A5848FDF7A1FC584BDFED587AF3
:10C558001880564B9FED577AB3F9003028EE278A9A
:10C5680007EE903A544BF8EEE77AB3F9002067EEFD
:10C57800C77AB1EE499ACDED087A07EE902AB3F959
:10C588000220B3F904308DED069AF8EEE77AF1EE61
:10C59800688ACDED097A07EE902AF8EEE77A09A8BD
:10C5A800CDED0A7A07EE903AF8EEE77A06A9CDEDD6
:10C5B800078ACDED0B7AFEF795FE73789DED0B7A21
:10C5C800012B19D13D4B1B785B070FD4D4F8D4321B
:10C5D800402293FBF2F29B1A07EE903AF8EEE77AC4
:10C5E80077EE877AFDEEE77AC4EDB57AD4F8D432DF
:10C5F800402293FBF2F301E0B8F800309DED090A00
:10C6080007EE903AF8EEE77A37EE677AD4EDB67A25
:10C618008DED0B7A94EDB77A38EE077A88EE078AB3
:10C628009DED0B7A37EE677AE8EE077AB0EE678A07
:10C63800C4EDB67A09F00AFFD4F8E0522978FEF77B
:10C6480079FDD4F8E4329DED0A0A1844C4F8E402EE
:10C6580009F0FCFE2978FEF76DFDD4F8E832B0EE5B
:10C66800480A1844C4F8E80209F0F0FE6978FEF7B1
:10C6780061FDD4F8EC32124A18441368C4F8EC028D
:10C6880053441360D4F8F0320133C4F8F03205E0B3
:10C69800A5F86232A5F86432A5F866320DB0BDEC93
:10C6A800048BBDE8F08F00BF30000020E8100020A8
:10C6B800BD37863535FA8E3CDA1000202A34002042
:10C6C8000C340020084BDA68D10709D4DA68D2069E
:10C6D80008D4DB6813F0040F14BF0320042070474C
:10C6E80001207047022070470020024003788B42E7
:10C6F80086BF024B33F81100002070472822002023
:10C7080070B5344C0546FFF773F9A369A061C31AE5
:10C71800B3F5FA5FE36182BF002384F8203084F820
:10C72800213094F820302BB9A12D02BF294A0121CC
:10C7380082F8211094F82110264A31B1D118EDB2AF
:10C74800013381F8225082F8203094F8205094F870
:10C758004330AB423CD11F4B93F84430052B02D0F9
:10C76800062B03D02FE0002006F09AFA94F8233025
:10C778001E2B28D100200246C1B26B1E99421ADA3C
:10C78800214491F822300821DBB283EA0206F60739
:10C7980044BF83F01803C3F3460301F1FF3154BFCC
:10C7A8005B0843F0800311F0FF01C2F34702ECD1AC
:10C7B80001301A46E0E7234493F822309A4202D126
:10C7C800032006F06DFA002384F8213084F8203025
:10C7D80070BD00BF2822002010B50446B0F9000043
:10C7E80004F01AFCB4F9020004F016FCB4F90400D1
:10C7F800BDE8104004F010BC10B50446006804F011
:10C808000BFC606804F008FCA068BDE8104004F068
:10C8180003BC2DE9F74F0120FBF794F9002488B3F6
:10C82800012C2FD8194E4FF04C0909FB04FA06EBDE
:10C838000A0808F19007BD7815B10134E4B2EEE7B3
:10C8480090F9003090F804E01846114B03228DE867
:10C85800240001212A4653F82E30FBF749F8834675
:10C8680060B106F14800504429464A4609F0DFFB0A
:10C8780001231C44C8F848B0BB70E4B20120FBF7A0
:10C8880047F9CCE703B0BDE8F08F00BF28220020AD
:10C898003C92010800212A2210B5114809F0C7FB73
:10C8A800104B002219461048105C83F8F20104244A
:10C8B8000520013283F8F74182424FF0000483F8E3
:10C8C800F60183F8F94183F8F80103F10803EAD186
:10C8D8000123A1F8F431522381F8F03110BD00BFD3
:10C8E800102E0020202C00207BAE010810B5FFF789
:10C8F800E9FE4FF43024012806D11CB1FFF7E2FE0F
:10C90800013CF8E7052010BD002C08BF052010BD2C
:10C9180070B50646441E14F8011F89B1094D284612
:10C9280009F0BBFB0028F6D005F1080398423FBF89
:10C93800054B401BC018A31B38BF80F88A31EAE7B3
:10C9480070BD00BF06B80108202C002007B51C4B9D
:10C9580003F1E402C3F8E0201A4A92F892215AB18E
:10C96800012A14D1032183F8E610072183F8E8206F
:10C9780083F8E7100C2208E0022183F8E61003216F
:10C9880083F8E82083F8E710072283F8E4200E4BA9
:10C998000E4A1A604020FBF7D5F870B10122002337
:10C9A80090F9000040218DE80C00094A4FF4E1336A
:10C9B800FAF79EFF003018BF012003B05DF804FBB2
:10C9C80028220020202C00203C000020612A010899
:10C9D800152B01080120002105F028B8F0B5184AE8
:10C9E80092F8E930D2F8EC701546042B11D807EB11
:10C9F800C3025E1C941CF6B209D013469288D10774
:10CA080005D5104203D008E00131052908D1334685
:10CA1800EBE785F8E9300020F0BD93F802E000214B
:10CA2800074C0C2204F1F00C02FB01F31CF8032064
:10CA38009645E9D1234484F8E960D3F8F400F0BDC1
:10CA48002822002020F01F01012300F01F00024AC5
:10CA580083408B50704700BF1404014000230360DB
:10CA6800436083608381036143618361C3610362BF
:10CA78004362836270478A68036810B50C6A14437E
:10CA88000A6914434A6914438A691443CA691443F6
:10CA98004A6A14438A6A23F4FF4323F0700322434B
:10CAA800134303608B8943600B6883604B68C360E2
:10CAB80010BD02684FF6FE73134003600023036045
:10CAC80043608360C360294B984201D1284A27E01C
:10CAD800284B984201D1264A2AE0274B984201D197
:10CAE800234A2DE0254B984201D1214A30E0244BBE
:10CAF800984201D11E4A33E0224B984204D11C4A85
:10CB0800536843F470032EE01F4B984204D1184A2F
:10CB1800536843F0706326E01C4B984204D11C4ACA
:10CB2800536843F00F031EE01A4B984204D1184A89
:10CB3800536843F0F00316E0174B984204D1144AA7
:10CB4800536843F470630EE0144B984204D1104AC2
:10CB5800536843F4704306E0114B984204D10C4AE1
:10CB6800536843F470235360704700BF08000240C5
:10CB7800000002401C000240300002404400024015
:10CB8800580002406C000240800002400804024045
:10CB9800000402401C0402403004024044040240E5
:10CBA8005804024001F0030301F0FC0101F1804147
:10CBB80001F5803110B59B008C680F229A4024EA59
:10CBC80002028A608A68984002438A6010BD0A8817
:10CBD8008B88F0B54C880E89CD88C2B9026A22F0DC
:10CBE800010202628269016A22F0F3021A4342EAF0
:10CBF800061344F0010421F00A021443836104621D
:10CC0800836923F00C03836183691D431FE0042AB1
:10CC1800016A1ED14FF6EF720A4002628269016A08
:10CC28001B0222F4734243EA06332401134344F0FF
:10CC380010044FF65F720A40A4B222438361026275
:10CC4800836923F440638361836943EA0525856129
:10CC5800F0BD082A1DD14FF6FF620A400262C26980
:10CC6800076A4FF60C7111404FF2FF523A4042EA00
:10CC7800042443EA06130B4344F480749BB2A4B221
:10CC8800C3610462C2694FF6F3731340C361C36999
:10CC98001FE04EF6FF720A400262C169026A40F65E
:10CCA800FF470F4045F6FF7111401A0242EA06336A
:10CCB80041EA04343B4344F480549BB2A4B2C361B8
:10CCC8000462C2694FF2FF331340C3612D02C36986
:10CCD800ADB21D43C561F0BD036A23F001030362D1
:10CCE800036A70B5446882690D6822F4803222F0C4
:10CCF800730215438A8923F0020313438A88134376
:10CD0800134A90420FD002F5006290420BD002F510
:10CD18004062904207D002F58062904203D002F54B
:10CD2800806290420DD1CA89CE8823F0080313434C
:10CD38000A8A24F4407414434A8A23F004033343D0
:10CD480014438A68446085614263036270BD00BF12
:10CD5800002C01409B4A536803F00C03042B2DE977
:10CD6800F04105D0082B06D097490160B3B916E009
:10CD7800954B036012E053685468C3F38343991CCE
:10CD8800E30349BFD36A914B8F4C03F00F0344BFB1
:10CD98000133B4FBF3F34B43036000E00023516815
:10CDA8008B4FC1F3031139440D790168EDB221FAB3
:10CDB80005F444605668C6F302263E44367924FAE0
:10CDC80006FEC0F808E05668C6F3C2263E44367927
:10CDD800F6B2F440C460D2F82C80C8F3041808F006
:10CDE8000F0C07EB4C0C18F0100FBCF814C01FFA0E
:10CDF8008CFC07D0BCF1000F04D0B3FBFCFCC0F8DE
:10CE080010C000E00161D2F82CC0CCF3442C0CF027
:10CE18000F0807EB48071CF0100FBF8ABFB204D0F9
:10CE28001FB1B3FBF7F7476100E04161176BFF06DD
:10CE38005ABF654F87618161176BBF065ABF624F42
:10CE4800C761C161176B7F065ABF5F4F07620162F6
:10CE5800176BFF0506D5994204D1AE4202D14F00A7
:10CE6800476200E04462176BFF0406D5994204D17B
:10CE7800AE4202D14F00876200E08462176BBF05A3
:10CE880006D5994204D1AE4202D14F00C76200E0F4
:10CE9800C462176B7F0506D5994204D1AE4202D110
:10CEA8004F00476400E04464176B3F0506D599427C
:10CEB80004D1AE4202D14F00876400E08464176B4E
:10CEC800BF0406D5994204D1AE4202D14B00C364D7
:10CED80000E08464156B3B4BAD0701D1046315E09A
:10CEE8001C6B04F00304012C01D101630EE01C6BE0
:10CEF80004F00304022C02D14FF4004305E01B6B3D
:10CF080003F00303032B01D12F4B0363146B2D4B49
:10CF180014F4403F02D1C0F834E018E01C6B04F46C
:10CF28004034B4F5803F01D1416310E01C6B04F438
:10CF38004034B4F5003F02D14FF4004306E01B6BC8
:10CF480003F44033B3F5403F01D11F4B4363146BE7
:10CF58001C4B14F4402F02D1C0F838E018E01C6BC9
:10CF680004F44024B4F5802F01D1816310E01C6BD8
:10CF780004F44024B4F5002F02D14FF4004306E036
:10CF88001B6B03F44023B3F5402F01D10E4B836391
:10CF9800146B0C4B14F4401F02D1C0F83CE021E0A4
:10CFA8001C6B04F44014B4F5801F01D1C16319E06F
:10CFB8001C6B04F44014B4F5001F0BD14FF400436C
:10CFC8000FE000BF0010024000127A0000093D0087
:10CFD8003C0000201B6B03F44013B3F5401F01D144
:10CFE800134BC363126B134B12F4400F03D1C0F8F9
:10CFF80040E0BDE8F0811A6B02F44002B2F5800F00
:10D0080002D10164BDE8F0811A6B02F44002B2F566
:10D01800000F02D14FF4004306E01B6B03F44003FA
:10D02800B3F5400F01D1024B0364BDE8F08100BFA6
:10D0380000127A0000100240F0B500230E681C466A
:10D048000125A54005EA060EAE452BD10F797A1EBB
:10D05800012A15D8856803229A4025EA02028260CF
:10D068004D7982689D4015438560828892B222EA94
:10D078000E0282808A798588A2402A4392B28280F1
:10D08800032205689A40D2431540056005689F4011
:10D098002F430760C7681740CA7902FA03F547EAC1
:10D0A8000502C2600134102C03F10203C8D1F0BD9F
:10D0B80038B52DED048B4A4C0368C4F82C318388AD
:10D0C800A4F83031013A0D46072A42D8DFE802F0C9
:10D0D800040A101822292F35B4F82C310B80B4F823
:10D0E8002E3113E0B4F82E310B80B4F82C3105E062
:10D0F800B4F82C315B420B80B4F82E315B4205E06A
:10D10800B4F82E315B420B80B4F82C316B80B4F844
:10D1180030311DE0B4F82C315B420B80B4F82E316D
:10D1280012E0B4F82E310B80B4F82C310CE0B4F8CE
:10D138002C310B80B4F82E3105E0B4F82E315B4267
:10D148000B80B4F82C315B426B80B4F830315B4211
:10D15800AB80244B93F83430002B3ED1B5F9003026
:10D1680094ED500AD4ED4D7A09EE103AB5F9023033
:10D1780008EE103AB8EEC88AB5F90430B8EEC99A84
:10D1880028EE000A08EE903AA7EE890AF8EEE88A37
:10D19800D4ED537AA7EEA80A09F058F994ED510A8C
:10D1A800D4ED4E7A288028EE000AA7EE890AD4ED3D
:10D1B800547AA7EEA80A09F049F994ED520AD4ED79
:10D1C8004F7A688028EE000AA7EE890AD4ED557ACE
:10D1D800A7EEA80A09F03AF9A880BDEC048B38BD7F
:10D1E800282200203C000020104BDFED117A1B683C
:10D1F8009A89104B1B6883F31003D31A07EE103A71
:10D20800B8EEC77A27EE277A07EE902AF8EEE77A83
:10D21800C7EE277AFDEEE77A17EE900A6428A8BFD2
:10D22800642020EAE070C0B2704700BFF810002008
:10D238000000C84208110020094B1A68137844F608
:10D24800FB7103EB431300FB03135078C0EB003072
:10D25800B3FBF0F39078B3FBF0F080B2704700BFF7
:10D26800F810002008B50A4890F8593100EB43033C
:10D278000A22B3F8681189B2A0F8701100F5BC70E1
:10D28800FEF7A2FC80B2FFF7D7FF024B188008BD5B
:10D2980028220020FC10002008B5084808F00BFFE1
:10D2A800C0B209280246054B04DC01302021C0B277
:10D2B8009954F6E700221A5408BD00BF49240020FB
:10D2C80008B5074808F0F7FEC0B21428044B04D884
:10D2D800421C20211954D0B2F7E700221A5408BD85
:10D2E800492400202DE9F74FA74CFEF781FB26685B
:10D2F8006568A768861BF643451BC71BED43FF43BC
:10D30800F60F8046ED0FFF0F2EB93FB9002D00F044
:10D318008682B9462CE04FF0000929E0B14627E0A3
:10D3280003EB8A0BBBF802301A050ED413F4805FA6
:10D338001DBF964A9BF801101268954A954B14BF79
:10D3480052F82120126843F82A20BBF80230D80589
:10D3580016D499050AD5904B1B7813F0040F0CBF0F
:10D368008E4A8F4A8B4B126843F82A2009F101092B
:10D37800207B8C495FFA89FA82450B68D0D326E076
:10D38800894A5046594602F023FE884B1B885A06A4
:10D3980003D550465946864A16E0580703D55046E5
:10D3A8005946844A10E0190703D550465946824A1F
:10D3B8000AE09A0703D550465946804A04E0DB073D
:10D3C800D4D57F4A5046594602F002FECEE7DFF830
:10D3D80008E20093BEF906307822A3F57A73534326
:10D3E8004FF47A7293FBF2F303F22B1301930022AA
:10D3F800F3465FFA82FE864517D2009B03EB820E46
:10D40800BEF802E01EF4806F0DD0DFF88891019B12
:10D4180039F822E040F2671A9E449EFBFAFC0AFBA8
:10D428001CEE29F822E00132E3E74DB308F5C333D7
:10D43800A0336360637B544A13BB9373614B1B68CF
:10D4480013F0020F0AD0DFF894E19EF800E0BEF175
:10D45800000F03D04FF0010E82F80EE0DA0506D572
:10D46800594B5B791BB1A37B43F00203A3734A4B6F
:10D478001B7813F0050F02BFA37B43F00403A373CB
:10D4880094F80EE0BEF1000F03D13F4B5B7B002BFD
:10D498004FD094F80DC01CF0010FACF10C031DD156
:10D4A800BCF1030F07D8DFF8E8903C4A1EF0040FE0
:10D4B80008BF4A4600E0364AACF1040CBCF1070F3D
:10D4C80005D8DFF81CC11EF0010F18BF6246DBB299
:10D4D800032B0ED81EF0020F3C4B06E0DBB2032BE9
:10D4E80006D82F4B2A4A1EF0020F18BF1A4600E032
:10D4F800274A4FF0000C5FFA8CF383420DD20B6879
:10D5080003EB8C035B881B0642BF224BD2F80090CA
:10D5180043F82C900CF1010CEDE785B1BEF1000F3A
:10D5280008D0637B184A0133DBB2142B06D10023E1
:10D5380004E025B1637B002BF3D100E05373002E88
:10D5480052D0234AB2F90250B2F90020002DB8BFD8
:10D558006D42002A4FF03203B8BF524295FBF3F5F3
:10D5680092FBF3F2EDB2D3B2AB4238BF2B46194A65
:10D5780013B192FBF3F300E0134643442360E37BCB
:10D58800014A7BBB01232EE028240020B824002078
:10D5980050A70108AA0D00202A34002094970108FA
:10D5A80084970108E01100205C920108D411002042
:10D5B80062920108689201086E920108749201084B
:10D5C8007A920108FC270020340E00209C9701085D
:10D5D800F0100020400D0300382800205C110020C6
:10D5E800A49701080023D3738E4D8F4B2D78E27BCF
:10D5F800ADB9002F00F00E818C4B267B1A788C4B2E
:10D608008C4D93F800C08C4BD3F800E00B6802F007
:10D6180004020021D2B203EB86060F46B5E01AB920
:10D62800864A1A61002508E0854AFAE70A68AB00CD
:10D63800D6187688760604D40135EBB28342F5D342
:10D64800D7E7804EB6F90060192E25DD12F803E001
:10D6580094F814C026690EF00F09E1450CDCDFF8D8
:10D66800C8C19CF815C0BCEB1E1FDEBFDFF8D8E1AF
:10D67800D6F800C043F80EC012F803E094F816C0BC
:10D688000EF00F09E14533DBDFF89CC19CF815C0AB
:10D69800BCEB1E1F2CDC26E0193629DA12F803E051
:10D6A80094F814C026690EF00F09E1450CDCDFF888
:10D6B80078C19CF817C0BCEB1E1FA2BFDFF888E139
:10D6C800D6F800C043F80EC012F803E094F816C06C
:10D6D8000EF00F09E1450BDBDFF84CC19CF817C0D1
:10D6E800BCEB1E1F04DBD6F800E0574E43F806E0FB
:10D6F800544EB6F90260192E1BDD12F803C094F8D7
:10D7080014E026690CF00F09F1450CDCDFF81891DC
:10D7180099F81590B9EB1C1FDEBFDFF82CC1D6F8BD
:10D72800009043F80C90D25C02F00F0CF4451EDD1B
:10D7380082E7193680DA12F803C094F816E02669F1
:10D748000CF00F09F1450CDBDFF8DC9099F8159027
:10D75800B9EB1C1FDEBFDFF8F0C0D6F8009043F825
:10D768000C90D25C02F00F0CF445FFF665AF94F80C
:10D7780017E0BEEB121FA2BF334A36689E505BE724
:10D788005888000504D404330435B342F8D122E0A4
:10D798004AB101EB0C0A06209AFBF0F900FB19A02C
:10D7A80001280DDC01E057B9012793F801900EEB31
:10D7B80089003EF829A090F80290C07803E0174647
:10D7C800002081468246013125F802AC85F8009098
:10D7D8006870C9B2D7E7164A1378013B13F0FF0304
:10D7E80008BF06231370114B1B785B0741BFBBF9B9
:10D7F8000630A3F57A7303EBC3034FF47A7243BF81
:10D8080093FBF2F30133DBB20123104A92FBF3F3EB
:10D818004344A36003B0BDE8F04F01F02DBD03B051
:10D82800BDE8F08F630E0020282400202A34002051
:10D8380074000020AC0D0020B8240020A097010837
:10D8480050A70108F0100020AA0D0020400D030089
:10D8580030B50028104C114AB8BF40423C2590FB17
:10D86800F2F304FB030068430D4D90FBF2F22D68C0
:10D878002D7B25B903EB830303EB830301E0C3EBA3
:10D88800031302EB83030B8004FB02024FF47A7349
:10D8980092FBF3F24A8030BD806967FF809698005A
:10D8A80000110020022803D0431E584258417047F7
:10D8B800064B1B681B7823B1054B1868C0F3C040A2
:10D8C8007047044B1878C0F38000704704060020A6
:10D8D8000C1000202A34002010B50A4C5E2801469E
:10D8E800206805D15D21FEF76CF920683E2105E02E
:10D8F8005D2903D1FEF765F920683D21BDE8104098
:10D90800FEF75FB940240020A0F17D03012B70B51C
:10D9180004460D460A4E05D830687D21FEF751F9B8
:10D9280084F0200430682146FEF74BF935B12B8886
:10D938001C4404EB142404F0FF042C8070BD00BFC9
:10D94800C411002010B5054C2068FEF737F918B14E
:10D958002068FEF730F9F6E710BD00BF94110020EB
:10D9680010B50446C0B2FFF7B7FFC4F30720BDE8FF
:10D978001040B1E7024B5E211868FEF722B900BFDC
:10D988004024002038B5064C05465E212068FEF785
:10D9980018F920682946BDE83840FEF712B900BFDB
:10D9A8004024002013B5044601A90068FFF750FF82
:10D9B8001320FFF7E7FFBDF90400FFF7D1FF1B2095
:10D9C800FFF7E0FFBDF90600FFF7CAFF2320FFF7C6
:10D9D800D9FF2368002BB4BF53204E20FFF7C0FFA8
:10D9E80001A96068FFF734FF1220FFF7CBFFBDF9EC
:10D9F8000400FFF7B5FF1A20FFF7C4FFBDF90600C2
:10DA0800FFF7AEFF2220FFF7BDFF6368002BB4BF0E
:10DA180057204520FFF7A4FF02B010BD674B73B530
:10DA28001878674DFFF73EFF2B788342044620D0D5
:10DA3800C8B1644B1B68E3B193F90000022300935B
:10DA4800614B1B685B78003318BF012301930421E5
:10DA58004FF416530022F9F74BFF5C4B186040B1A6
:10DA680001232B7005E0594E3068F9F72EFF34601A
:10DA78002C70574B574D1878FFF714FF2B788342BB
:10DA8800044618D088B1544B1B68A3B10022012466
:10DA980093F9000000944FF4964301920821F9F796
:10DAA80027FF4E4B186028B905E04C4E3068F9F74F
:10DAB8000CFF34602C704A4B4A4D1878FFF7F2FE81
:10DAC8002B78834204462E4642D0002837D0464B56
:10DAD8001A68002A3CD0D37992F90000434C002BF5
:10DAE80008BF022302220092002254F82330019238
:10DAF8001021F9F7FDFE3E4B0546186040B33D4C3A
:10DB080094F84A30022B0BD094F89620022A01D1BF
:10DB18004C3405E023B1002A04F14C0418BF00245A
:10DB2800354B1C6044B1204600214C2208F07FFA96
:10DB38000223256084F84A300123337008E02C4E14
:10DB4800306803F01FFF3068F9F7BFFE34602C70AF
:10DB58002A4B2B4D1878FFF7A5FE2B7883420446F5
:10DB680029D000B3274B1B682BB3274A93F9000031
:10DB780012685278002A0CBF082209220323009356
:10DB880001924FF4614320210022F9F7B1FE1F4BA7
:10DB9800186080B11E4A012313702B701D4B1A6840
:10DBA8001D4B1A6007E0194E3068F9F78EFE184BC6
:10DBB80034601C702C7002B070BD00BF0C060020D1
:10DBC800D01000200806002000110020402400206A
:10DBD8000D06002020110020A4110020941100201F
:10DBE80018060020AA110020140600203C92010803
:10DBF800AC11002070220020B01100202406002063
:10DC0800C0110020200600201C060020C41100209E
:10DC1800C811002020280020CC110020642928BF2A
:10DC28006421F8B510FB01F56424064695FBF4F46D
:10DC38000027E4B2FBB2A34204D29F20FCF7E9FE1E
:10DC48000137F7E7B4420BD2C4EB84101421C4EBBC
:10DC5800800095FBF1F5663D2844C0B2FCF7D9FE7B
:10DC68000134E4B2B44201D29A20F7E7F8BD2DE9B5
:10DC7800F743934CFDF7BCFE6368C31A002BC0F250
:10DC8800678300F5433303F5A07363608D4B1D78FC
:10DC9800237AC5F38005EB1A18BF012325724DB10D
:10DCA800002B00F05583884B5A789A7001225A70DD
:10DCB8001A702BE0844A2BB1D37843F00203D37057
:10DCC80093785370D67806F0020101F0FF0339B952
:10DCD8007D498968411A002903DB06F0010300E049
:10DCE800012303F00107784917707BB1F2070DD5BE
:10DCF8000A790132D2B20523B2FBF3F303EB8303B3
:10DD0800D31ADBB2714A0B71D35C4B706E4EDFF8DD
:10DD1800088233787BB3F37823F00203F3706C4BFB
:10DD28000344AE20B360FCF798FE08B1FCF79AFEF6
:10DD380088F80000002800F00B83B020FCF78DFE67
:10DD48004020FCF78AFE0020FCF787FE1020FCF735
:10DD580084FE4FF48067013F0020BFB2FCF754FEF9
:10DD6800002FF8D13846FCF7ECFE7278594B53F87F
:10DD78002200FCF769FE98F80030002B00F0E882DA
:10DD88007378062B00F2B382DFE813F00700B102C4
:10DD9800180078006C018901EE014F494F4A504B39
:10DDA8005048FDF792F90120FCF7CBFE4D48FCF7EF
:10DDB8004BFE0220FCF7C5FE4B48AEE14B4F3B68DB
:10DDC8009B0735D5DFF85481DFF85491B8F8001077
:10DDD80044480A23B1FBF3F203FB121399F800102D
:10DDE800009192B242499BB2FDF76FF9FFF768FACA
:10DDF8000120FCF7A6FE3B48FCF726FE3D4B99F8B0
:10DE080000201868B8F80030067906FB1231642340
:10DE18004B43C1788E1B56430220B3FBF6F6F6B28D
:10DE2800FCF78FFE31461520FFF7F8FE032600E0C9
:10DE380001263B681F0540F15A822F4B2F491F6866
:10DE48000968009164232E4997FBF3F2254803FBE8
:10DE58001273FDF73AF9FFF733FA3046FCF771FE13
:10DE68002048FCF7F1FDFFF7BFF90746701CFCF7E7
:10DE780068FE15203946FFF7D1FE38E20120214F10
:10DE8800FCF75FFE2048FCF7DFFD3B68980749D5A3
:10DE98001E4A1448B2F90210B2F900300091B2F9E2
:10DEA80004201B4901921B4AFDF70FF9FFF708FAF6
:10DEB8000220FCF746FE0B48FCF7C6FD032632E0BD
:10DEC800402400202A3400207824002080AE010855
:10DED800404B4C008092010885AE01088EAE0108C7
:10DEE80089A701084924002095AE0108FC270020D5
:10DEF800A0AE0108F810002004110020081100202D
:10DF0800B8AE01080C110020CDAE0108DA100020CF
:10DF1800E3AE0108F2AE010879020020FC100020EF
:10DF28008000002002263B68D9071AD57C4A7D4824
:10DF3800B2F90210B2F900300091B2F904207A491E
:10DF480001927A4AFDF7C1F8FFF7BAF93046FCF7B3
:10DF5800F8FD744806F10108FCF776FD5FFA88F8C9
:10DF680046463B681A0718D5714A6E48B2F902103E
:10DF7800B2F900300091B2F904206B4901926D4A60
:10DF8800FDF7A3F8FFF79CF93046FCF7DAFD654882
:10DF9800771CFCF759FDFFB23E46674A6249B2F961
:10DFA8000030B2F902200092644A5E48B2F90020BB
:10DFB8000192634A634FFDF788F8FFF781F930460D
:10DFC800FCF7BFFD5748FCF73FFD97ED000A5548A1
:10DFD800FCF710FF534808F06EF806F101085FFAE5
:10DFE80088F8C0B2B946092809D8431C2044DBB2D6
:10DFF80020224272E218002191721846F3E7494F35
:10E0080099ED010A3844FCF7F5FEFFF759F9404647
:10E01800FCF797FD3846FCF717FD99ED020A3846DC
:10E02800FCF7E8FE384608F046F80236F6B2C0B209
:10E03800092809D82318421CD2B220215972A318E2
:10E04800002199721046F3E73F4AB2F9003000EE1A
:10E05800103A3844B8EEC00AFCF7CCFEFFF730F9A6
:10E06800304657E00026394F3B78B34240F23F81B3
:10E078000E2E00F03C8170080130FCF762FD30463E
:10E0880003F048FB3B78B34206D92020FCF7C1FCDB
:10E09800701CC0B203F03EFB0236F6B2E3E72C4E2A
:10E0A8002C4996F8B4271F48FDF70FF80120FCF714
:10E0B80048FD1C48FCF7C8FC274B28491F7819481D
:10E0C8003A46FDF702F80220FCF73BFD1548FCF73D
:10E0D800BBFC0C2303FB0766214996F8B72796F883
:10E0E800B6371048FCF7F1FFFFF7EAF80320FCF712
:10E0F80028FD0C48FCF7A8FC96F8BC1796F8BA2738
:10E1080096F8BB37074800911649FCF7DEFFFFF782
:10E11800D7F80420FCF715FD0248FCF795FCE6E06B
:10E128002C10002049240020E3AE0108F6AE0108B7
:10E13800321000201EC40108F4270020E810002037
:10E14800FAAE0108E4210020F02100200C23002071
:10E15800202C0020FEAE0108602800200AAF01082C
:10E168001BAF01082CAF01087B4B1B681B0640F155
:10E17800BA80236A616A794A8B421FBF536292F858
:10E188002830013303F003034FF001014FF0000082
:10E1980018BF82F82830FCF7E0FC94F82830704A61
:10E1A800D05CFCF736FC02200121FCF7D6FC0026E7
:10E1B8006C4B9B5D3620C3EBC30393FBF0F0C0B2FE
:10E1C800062828BF06206038C0B20136FCF721FCBB
:10E1D800102EEDD1644B65491B78654813F0020F8A
:10E1E800644B1A7814BF59234E23FCF76EFFFFF7D0
:10E1F80067F80220FCF7A5FC5D48FCF725FC5E49A2
:10E208005E4B4E680A685A4892FBF3F25C4996FBEB
:10E21800F3F3FCF75AFFFFF753F80320FCF791FCE0
:10E228005348584EFCF710FC574B58491A88504829
:10E23800FCF74BFFFFF730F80420FCF782FC4C4852
:10E24800FCF702FC524B53491A884948FCF73DFF3A
:10E25800FFF722F804210A20FCF77FFC4448FCF76A
:10E26800F3FB4D49E26A4248FCF72FFFFFF714F829
:10E278000520FCF766FC3E48FCF7E6FB7268B368CD
:10E2880046493B48FCF721FFFFF706F805210A201D
:10E29800FCF763FC3648FCF7D7FB3369F268404962
:10E2A8003348D21AFCF711FFFEF7F6FF0620FCF7F9
:10E2B80048FC2F48FCF7C8FBB2683A492C48FCF7E1
:10E2C80004FFFEF7E9FF06210A20FCF746FC284870
:10E2D800FCF7BAFB34492648152207F019FFFEF768
:10E2E800DBFF072016E7F37843F00203F370002DF5
:10E2F8002ED12E4B9B79032B9BBF2D4A9B183F2574
:10E308001D7F00211220FCF728FC2846FCF781FB22
:10E3180013200021FCF721FC264B1B78002B264BF1
:10E328001B7814BF72202120002B18BF5220FCF745
:10E3380070FB14200021FCF710FC94F83050084BB7
:10E34800585D013505F00305FCF763FB84F8305090
:10E3580003B0BDE8F08300BFFC2700204024002064
:10E368003EAF0108BD1000201011002043AF010886
:10E3780049240020161100201811002080969800CA
:10E3880054AF0108A40700201211002061AF010852
:10E398007410002069AF010870AF010877AF010859
:10E3A80080AF010887AF0108C4020020340E0020A6
:10E3B80080920108630E0020C80E002038B50024A2
:10E3C8000B4D6059254403F0D7FB696811B1094822
:10E3D800FCF790FEA96811B10748FCF78BFE0748C7
:10E3E800103403F0C9FBB4F5F07FE9D138BD00BFA4
:10E3F800A0920108C0AF0108C6AF0108E8B901083A
:10E4080070B50546284607F056FE064658B91A4B19
:10E418001A485A791A4B03EB8203BDE87040D3F8C7
:10E42800DC11FCF767BE28461649324607F04CFE59
:10E4380060B91548154C03F09FFB54F8041F19B137
:10E448001348FCF757FEF8E7124805E00024124B82
:10E4580053F8241021B91148BDE8704003F08CBB73
:10E468002846324607F030FE01340028EFD1024B2F
:10E478000B4D5C71C6E700BF202C0020CCAF010813
:10E48800A0920108D8AF0108DDAF01087C9401080B
:10E49800F0AF0108E8B901088094010896AD0108B9
:10E4A800ABAA0108F0B585B0044607F004FE0828B9
:10E4B80026D1621EE01D1F4912F8013F0968194460
:10E4C800497801F00301022908BF203B82421370FA
:10E4D800F1D1254604F1080715F8016B16483146B5
:10E4E80007F0DBFD20B12846314607F0D6FD10B114
:10E4F800F8F7A2FD1CE0BD42EED12046FEF708FA6F
:10E508000E4803F039FB00230D4A1A4404A992F877
:10E518008A210A440849595C02F80C1C0133082B6B
:10E52800F2D1002307488DF80C3001A9FCF7E2FD71
:10E5380005B0F0BD9000002006B80108F4AF01084E
:10E54800202C00208CB80108264B274C1D68206819
:10E5580080B5F9F7AFF92846F9F7ACF920684179A1
:10E568008A0703D441F00201FDF71CFB1F4B082268
:10E578009A611F4B1A6812F4003F1F461FBF0623FB
:10E588006371E37923F001031CBF43F00203E371D5
:10E598002068FDF713FB90B1144E08233385124B06
:10E5A8001868FDF708FB8046F9F798FB08B101F0F9
:10E5B800D9FD28464146FDF704FB0823B3612846E8
:10E5C800FDF7FCFA38B128462668FDF7F4FA01464B
:10E5D8003046FDF7F6FA3B689B03D9D5FFF747FBB2
:10E5E800D6E700BF7C2800207424002000040048DF
:10E5F800FC2700202DE9F041054607F05CFD2C4B77
:10E6080004469E6888B92B4803F0B6FA2A4B53F89B
:10E61800241041B10123A340334202D02748FCF71C
:10E6280069FD0134F2E7264821E0284625492246BB
:10E6380007F04AFD58B92448244C03F09DFA54F8D1
:10E64800041F0029EFD01D48FCF754FDF7E72B788D
:10E658002D2B03BF013504F1FF344FF001084FF0B3
:10E6680000080026144B53F8267027B91848BDE84F
:10E67800F04103F081BA28463946224607F024FDC6
:10E6880098B90120B040B8F1000F03D0FCF788FE1C
:10E69800104802E0FCF78CFE0F4803F06DFA39468B
:10E6A8000E48BDE8F041FCF725BD0136DAE700BFAA
:10E6B800202C0020FAAF0108E8940108F0AF010807
:10E6C800E8B90108D8AF010804B00108E4940108CA
:10E6D80096AD010810B0010819B001088BB80108FF
:10E6E80010B5084803F048FA074B00241C741C6452
:10E6F800064B1C70FDF7E8FB03F0F0FB044B1C60B5
:10E7080010BD00BF21B00108742400202D34002062
:10E718007C28002070B5064600240B4BE518AA8813
:10E7280016420AD0E1580948FCF7E4FC28460021C3
:10E7380003F0AFF9064803F01FFA143440F6944387
:10E748009C42EAD170BD00BF4C9901084DB0010848
:10E75800E8B9010808B50848FCF7CCFCFAF74EF808
:10E76800FCF7F8F818B96420FDF767F9F8E70348EB
:10E77800BDE80840FCF7BEBC57B0010864B001080A
:10E788002DE9FF410A48068885684488B0F8048066
:10E79800C768F9F73DFFCDF8008002900197314630
:10E7A8002A4623460348FCF7A5FC04B0BDE8F081DF
:10E7B800100000206CB00108F0B504788BB0054655
:10E7C8000CB1002436E04A4B19680E2303FB0411F0
:10E7D80001F58C70B1F91D51B1F91921B1F91B314D
:10E7E800009591F82051019591F82151029590F9E1
:10E7F8000700039001F590713E4891F902100491C9
:10E8080021460134FCF776FC082CDCD16DE02D2B79
:10E8180014D1072C1BDC284607F0A4FC0AAB661CA5
:10E8280003EB440424F8100C15F8013F303B092B86
:10E83800FAD934462B78002BE9D104E0A3F1300251
:10E84800092A09D8E5E7082CBDF8182009D00BB02B
:10E85800BDE8F040F8F7F0BB202BF8D1013526468B
:10E86800E7E7072AF3D8BDF81A00214BA0F2EE21FA
:10E8780089B240F2DC55A9421B68E8D8BDF81C10E3
:10E88800A1F2EE24A4B2AC42E1D8BDF81E7004B2E5
:10E898003EB2A642DBDB0DB2AE42D8DCA542D6DBE7
:10E8A800BDF92440642CD2D1BDF8266034B2112CB5
:10E8B800CDDCBDF82050B42DC9D8BDF82240B42C09
:10E8C800C5D812B24FF00E0E0EFB0233A3F81B117F
:10E8D8006421A3F81901A3F81D7183F8205183F866
:10E8E800214183F81F1183F822610BB0F0BD00BFEE
:10E8F80048100020C9B00108F0B504468FB0204682
:10E9080007F0D9FBC5B225BBAC48AD4C03F034F9D0
:10E9180094F8D61009B9AB4854E049B294F8D42019
:10E9280094F8D530009194F8D710019194F9D81043
:10E93800029194F9D910039194F8DA100491A2483D
:10E9480029460135FCF7D6FB102D04F10704DFD169
:10E95800E1E720469D49052207F0B6FB0546B8B910
:10E9680029469B48702207F062FB9A4B1968284693
:10E978000E2303FB001301300022082883F823210B
:10E9880083F8242183F8252183F82621F0D113E187
:10E9980020469149042207F097FB05462046002DA2
:10E9A8004AD1202107F079FB002800F00581461C98
:10E9B800304607F080FB2C460746884B53F8245016
:10E9C8002DB987480FB0BDE8F040FCF793BB30463F
:10E9D8002946FAB207F078FB01340028EDD1784ACD
:10E9E80002F170011646002382F8DA3082F8D63038
:10E9F80082F8D53082F8D43007328A42F3D1794987
:10EA080001EBC40191F8A022934210DAD1F8A47264
:10EA1800C3EBC302B0183A4400F1D4011768C0F838
:10EA2800D4709088888092798A710133E7E7294603
:10EA38006D48FCF75FFB90E06C49072207F044FB48
:10EA480005462046002D4AD1202107F026FB064620
:10EA580007F031FBC4B274BB6548FCF74BFB214699
:10EA680064480134FCF746FB0E2CF8D15548FCF7F6
:10EA780041FB002460482146FCF73CFB0025554A31
:10EA88005E4811680E2202FB04120123D2F82321EA
:10EA98005B49AB4013425B4B05F1010508BF1946C2
:10EAA800FCF728FB0E2DEAD146480134FCF722FB7F
:10EAB800082CDFD180E03046534907F057FB2C463D
:10EAC80000284CD0022C4FD007F04CFB06AB4E4927
:10EAD80043F82400002007F049FB0134F0E74A49D5
:10EAE80007F044FB002460B1082C38D007F03AFB4B
:10EAF80006AB454943F82400002007F037FB0134F2
:10EB0800F1E7082C2BD1069B0F2B28D8DDF81CE049
:10EB1800BEF1070F23D8089F0D2F20D8099E06F1B4
:10EB28006402C82A1BD80A9DFF2D18D80B986428A0
:10EB380015D80C99642912D8884210DA0D9C032C38
:10EB48000DD8324AC3EBC303134483F804E05F7162
:10EB58009E71DD71187259729C722D4CCFE60FB000
:10EB6800BDE8F040F8F768BA069B072B20D807994C
:10EB78000D291DD80278722A0DD06E2A18D1154A8F
:10EB880012680E2000FB032301228A40D3F82311C8
:10EB980021EA020209E00F4A12680E2000FB032353
:10EBA80001228A40D3F823110A43C3F8232101E044
:10EBB800F8F742FA0D4CA2E60FB0F0BDF1B001082B
:10EBC800202C0020E8B901081CB1010866AD010835
:10EBD800F42C00204810002091AD01088094010811
:10EBE80096AD0108A0920108A5AD0108E9B0010899
:10EBF800CAAF010838B101086DAF01083DB101087D
:10EC080063BC01081DBD010841B10108F02C0020BA
:10EC1800ABAA01082DE9F743047805468CB9324DB3
:10EC280095F8AF12B5F8AC2295F8AE322F4800919E
:10EC380021460134FCF75EFA102C05F10405EFD1EA
:10EC48004EE007F08FFA0F28044636DC28462021CC
:10EC580007F023FA264EE4B2D6F84480451CA400F7
:10EC68000027284607F07EFA5FFA87F9B9F1010F05
:10EC780083B208D0B9F1020F0BD0B3F5B47F24D218
:10EC8800726C13530AE0FF2B1FD8736C23449870DF
:10EC980004E0FF2B19D8736C2344D87028462C2124
:10ECA80007F0FBF9054608B1013502E0B9F1020F9A
:10ECB8000BD10137032FD4D112E00E4800210F22C7
:10ECC80003B0BDE8F043F8F734B908EB04000021BD
:10ECD800042207F0ACF903B0BDE8F043F8F7ACB98B
:10ECE80003B0BDE8F08300BF202C002043B1010829
:10ECF8007424002024AD01082DE9F0412DED048B8A
:10ED0800B3498AB0044607F09BF9B2490028204667
:10ED18000CBF0126072607F093F9AF4900282046C3
:10ED280008BF022607F08CF9002808BF0426F1075F
:10ED380040F10681A948AA4C02F01EFF002002F00B
:10ED480021FDA84802F018FFA74802F015FF6279D4
:10ED5800A64BA74803EB82032546D3F8DC11FCF742
:10ED6800C9F9A448FCF7C6F94FF00008274695ED05
:10ED7800058AB5EE408AF1EE10FA04D19E48FCF7F8
:10ED8800B9F9002570E09D48D5ED069A95ED079AEA
:10ED9800D5ED088A4146FCF7ADF9B5EEC08AF1EE2B
:10EDA80010FA02D5202002F0DFFEB0EE480A06A8CD
:10EDB800FCF720F801469248FCF79CF9F5EEC09A5A
:10EDC800F1EE10FA02D5202002F0CEFEB0EE690A6C
:10EDD80006A8FCF70FF801468948FCF78BF9B5EE51
:10EDE800C09AF1EE10FA02D5202002F0BDFEB0EE76
:10EDF800490A06A8FBF7FEFF01468148FCF77AF9A5
:10EE0800F5EEC08AF1EE10FA02D5202002F0ACFE31
:10EE1800B0EE680A06A8FBF7EDFF08F10108014605
:10EE28007848FCF767F9B8F10C0F05F110059ED189
:10EE3800A4E749B294F8D42094F8D530009194F816
:10EE4800D710019194F9D810029194F9D91003912F
:10EE580094F8DA1004916C4829460135FCF74AF910
:10EE6800102D04F1070403D094F8D6100029E0D13E
:10EE780000254FF00E0808FB05F80024634A926C41
:10EE880042440123D2F80A20A340134240F0948060
:10EE980001340E2CF2D10135082DEAD15C485D4CC5
:10EEA80002F06AFED7F8088054F8041F19B15A48CE
:10EEB800FCF720F9F8E70D46584B53F8254054B1B4
:10EEC8000123AB4013EA080F03D055482146FCF74D
:10EED80011F90135F0E7534802F04EFE21467B1840
:10EEE8000AAA93F88A3113444F4A8A5C03F8102C13
:10EEF80001310829F3D1002306A94C488DF82030A8
:10EF0800FCF7F8F84A4802F037FE4A48F8F754FD8B
:10EF1800494802F031FE4748F8F794F8474802F0AC
:10EF28002BFE4448FFF776FE4548FCF7E3F84020FF
:10EF3800FFF7F0FB434802F01FFE3E48F8F7B2FB2C
:10EF4800B20726D5404802F017FE404802F014FEEA
:10EF5800384802F057FC3E4802F00EFE3548F7F7F5
:10EF6800F5FF3C4802F008FE3248F8F7EDFA3A4857
:10EF7800FCF7C0F82F48F8F771F9384802F0FCFDA3
:10EF88002C48FFF719FC2E48FCF7B4F88020FFF74F
:10EF9800C1FB730716D5324802F0EEFD314802F086
:10EFA800EBFD244802F008FC2548FCF7A3F84FF4D1
:10EFB8008070FFF7AFFB05E0294622462A48FCF798
:10EFC80099F865E70AB0BDEC048BBDE8F08100BF95
:10EFD80057B10108CBB501085EB1010864B1010859
:10EFE800202C002072B1010884B10108A092010808
:10EFF80090B101089BB10108A8B10108B5B1010899
:10F00800C9AF01088CB80108BDB1010874240020FB
:10F01800DCB10108E4940108ECB10108E8940108A6
:10F02800FAB1010807B2010806B8010813B20108CD
:10F038001CB20108ABAA01082BB2010837B20108BB
:10F04800E8B9010845B2010852B2010865B20108E1
:10F0580073B201087DB201088CB201089AB20108A6
:10F06800A6B20108B7B20108C9B2010810F80A3CF3
:10F078000133DBB20A2B84BF10F8131C044A00F8D2
:10F088000A3C82BF002322F8113000F80A3C70477E
:10F098006C2B0020334A136C90681944081A40F608
:10F0A8008C23984270B513469160D06051603BD96B
:10F0B800127893F945108A4210460BD1111F08297E
:10F0C80008D893F84610182901D8013103E083F8CD
:10F0D800442002E0002183F8461093F94440214976
:10F0E800A24219D191F84740B4B10C31002494429E
:10F0F80006DA1D4D51F8046F25F814600134F6E75F
:10F108000C2805D01849002421F810400130F7E7F1
:10F11800164801780131017083F845200022012149
:10F128001A7083F8471070BD92F84710C9B1A0F261
:10F13800EF2440F2DA518C4208D811780B2905D80F
:10F148000B1D0131117042F8230070BD002283F8B5
:10F158004720074B03F13002002143F8041F934274
:10F16800FAD170BD300100206C2B0020340600203D
:10F178003C010020024A136C0133194411647047A2
:10F1880030010020024B53F820301B68196070478B
:10F19800601F0020064B53F820301A681B89A1F520
:10F1A8007A7159434FF47A7391FBF3F11160704708
:10F1B800601F0020054B98420CBF054A054A13887A
:10F1C80001339BB213800020704700BF00540040F9
:10F1D800081000200A10002038B510F80E2C50F83E
:10F1E800043C04465AB9012200F80E2C20F80C1CE5
:10F1F800997A18680222BDE83840F9F7A5BE30F8B8
:10F208000C2C20F80A1C891A89B220F8081C084A14
:10F2180010F80F0C002522F8101004F80E5C18687E
:10F22800997A2A46F9F790FE04F8065C38BD00BFC3
:10F238006C2B0020044B53F820301BB107289CBFCF
:10F248001B681960704700BF58020020074A1368FE
:10F258009B060AD5064B00211970064908684FF627
:10F26800FE7303400B602023536070470000024088
:10F27800293400201C0002402DE9F047664D2B6818
:10F2880066490A78581C02F0FF068E460AB1034602
:10F29800F6E72B60687BAB6895F80C80AA7B37464D
:10F2A80039B2202900F09B80DFF880C10CEB810384
:10F2B8003CF82110DC789B78C3F1FF039BB2002B4C
:10F2C80065D0C3F1FF0363434FF03C0C1B12B1FB45
:10F2D800FCF9B9F1050F5DD8DFE809F0030B1A292D
:10F2E8003A4AE01ADAB24143B1FBFCF01044C0B22A
:10F2F80051E0B1FBFCF00CFB101189B2DAB2C1F19C
:10F308003C01E31A4B432046B3FBFCFC94442CE03D
:10F31800B1FBFCF00CFB10115FFA83F8E21A89B21A
:10F328004A43B2FBFCF24244D2B2204632E0B1FB7F
:10F33800FCF90CFB191189B25FFA83F8E01AC1F1E4
:10F348003C014843B0FBFCF04044C0B2224621E0F7
:10F35800B1FBFCF80CFB1811D8B289B2E31A01FB17
:10F3680003F2B2FBFCFC224684445FFA8CF412E000
:10F37800B1FBFCF80CFB181189B2D8B2C1F13C0101
:10F38800E31A4B43B3FBFCF20244D2B203E0224639
:10F39800204600E044464FEA042C4CEA004C4CEA74
:10F3A800020C172306F117014FF0010808FA03F8B9
:10F3B800C91A18EA0C0F89B2DFF8748014BF4FF02D
:10F3C80011094FF0090913F1FF3308F80190E9D248
:10F3D80018360137B6B2BFB2114BA04660E7AA7320
:10F3E800AB60104AE98001238EF800300E4985F899
:10F3F8000C8040F22A336873AE80536000234B625E
:10F408000B889BB243F001030B80136843F00103A0
:10F418001360BDE8F08700BFC02400202934002015
:10F42800CC2400201C000240002C0140AA0D002022
:10F43800D902002073B506460D46002401232A8808
:10F44800A34013421AD0AA78009302F003038DF860
:10F458000430EB78022B03D0032B0CBF03230123CA
:10F468008DF805303046C2F301136946C2F38102B4
:10F478008DF806308DF80720FDF7DEFD0134102CDD
:10F48800DCD102B070BD2DE9F04F734EF57B074615
:10F498000C4687B011469A4600686B1C9146224676
:10F4A8004FF0020BF37300F083FC3B897868ADF8EA
:10F4B800043001A98DF806B08DF807B0FFF7BAFF40
:10F4C8000023ADF80A30ADF81230ADF816307023CD
:10F4D8000193BA7A3C68CDF80CA0012306F1100814
:10F4E8002D01ADF808304FF48073A844ADF810B082
:10F4F800ADF814300C2A7ED8DFE802F0077D7D7D58
:10F508000F7D7D7D387D7D7D5E00204601A9FDF75C
:10F51800E3FBA36943F0080326E0236A4F4823F07E
:10F5280010032362236A6168A26922F0807222F4C0
:10F53800E642844242F4E04206D000F5006084428C
:10F5480002D043F0300307E023F0E00321F44061E8
:10F5580043F0300341F480616160A261C4F838A0CF
:10F568002362A36943F40063A36144E0236A3B4830
:10F5780023F480732362226A6168E369844223F07A
:10F58800730343F0700306D000F50060844202D094
:10F5980042F4407207E022F4606221F4405142F4E0
:10F5A800407241F480516160E361C4F83CA022627A
:10F5B800E36943F008031DE0236A284823F48053D5
:10F5C8002362226A6168E369844223F4E64343F4D0
:10F5D800E04342F4405203D000F50060844201D178
:10F5E80041F480416160E361C4F840A02262E369AC
:10F5F80043F40063E3613A7B3B681AB15A6C42F406
:10F6080000425A641A8892B242F001021A80BA7A09
:10F618000C2A18D8DFE802F0071717170B17171767
:10F628000F1717171300721903F134010AE0721942
:10F6380003F1380106E0721903F13C0102E0721986
:10F6480003F14001116135444046A5F818906B61FB
:10F6580007B0BDE8F08F00BFC0240020002C014097
:10F66800F8B53A4E3A4C4000C7B24FF420453068DE
:10F67800C4F8D050D0F818E01EF4004F05D0AE46BC
:10F68800013DBEF1000FF5D116E0D0F804E0314D90
:10F698000EEA050545F490353D4345604FF4204595
:10F6A800C4F8D050D0F818E01EF0020F2DD1AE46A5
:10F6B800013DBEF1000FF5D1C4F8D0501FE0294636
:10F6C800013D0029F8D081694906F8D5C4F8D05021
:10F6D80020494568294041F0007141F4105141EA40
:10F6E8000241394341604FF42041A2B13068856935
:10F6F8006D071ED411F1FF31F9D2C4F8D010FFF70D
:10F7080059FD003018BF0120F8BD4FF42045816233
:10F71800C4F8D050D7E73068C4F8D0100B468269D7
:10F7280092060CD41A46013B002AF8D1C4F8D0300E
:10F73800E5E7416A03F8011B013AD2B2D3E7C4F8FE
:10F74800D0302023C3610120F8BD00BF0410002081
:10F75800C0240020009800FC400070B5C5B23248B3
:10F76800324B00684FF42044C3F8D0408669360411
:10F7780004D52646013C002EF8D113E046682C4CEF
:10F78800344044F0807444F490342C4344604FF483
:10F798002044C3F8D0408669B60729D42646013CE0
:10F7A800002EF8D1C3F8D0401CE02146013C0029C6
:10F7B800F8D081690E06F8D544681D49214041F00A
:10F7C800007141F48031294341604FF42041C3F86E
:10F7D800D0108469A40711D40C460139002CF8D143
:10F7E800C3F8D010FFF7E6FC003018BF012070BD49
:10F7F8004FF420448162C3F8D040DAE782624FF4C4
:10F808002042C3F8D0208169890606D41146013AFE
:10F818000029F8D1C3F8D020E4E7C3F8D02020238A
:10F82800C361012070BD00BF04100020C024002067
:10F83800009800FC6C4B6D4A2DE9F04F5E89146806
:10F848004FEA062AB4EB0A0A9C884FEA04481C8946
:10F858004FF000054FF0000B65EB0B0BA4FB0A679C
:10F8680004FB0B77F40944EA476418EB04065C8848
:10F878004FF000094FEAE7154FEAC438DC8849EB36
:10F88800050787B0CDE90467A4FB0A6704FB0B777B
:10F89800340A44EA076418EB04064FEA27259C89D2
:10F8A8004FF0000949EB0507CDE90067AAFB04679B
:10F8B80004FB0B77F40D44EA472414F5FA664FEA83
:10F8C800E75545F10007B6F5FA6F77F10003CDE982
:10F8D8000267964667DAA4FB046704FB05F34FF05A
:10F8E800050C07EB4307DDE90489A6FB0C230CFB99
:10F8F80007335F104FEA3206B8EB06084FEA920664
:10F9080069EB070946EA83769F10DDE90023921B1D
:10F9180063EB0703DDE90267CDE90023344A4FF0C2
:10F92800FF33964277EB0303CDE9048928DA40F6E2
:10F93800AC52A4184FF000035D4104FB05F3A4FB8F
:10F94800044505EB43056FF00602664202FB0566B7
:10F95800A4FB0223334418EB020649EB0307CDE965
:10F9680004670B26A4FB062306FB0533DDE90045E7
:10F978005B104FEA3202A41A65EB0305CDE9004596
:10F988000AFB0BF3DDE90245AAFB0AAB0BEB430BC1
:10F998004FEADA7242EA4B02A41A4FEAEB7365EBBC
:10F9A8000305CDE90245DEF80440009B019DA4FB58
:10F9B800032304FB05334FEA52584FEA635948EAD8
:10F9C800C328DDE90423B8EB020269EB0303994677
:10F9D800D30B43EA494300B1036009B1029B0B60B2
:10F9E80007B0BDE8F08F00BF8602002094250020F4
:10F9F80024FAFFFF772048210122FFF7ADBE7720C8
:10FA080058210122FFF7A8BE07B5002101AB032248
:10FA18007720FFF725FE9DF805309DF804001B02AE
:10FA280043EA00439DF80600184303B05DF804FB61
:10FA380008B5FFF7E9FF014B586008BD9425002081
:10FA480008B5FFF7E1FF014B186008BD94250020B9
:10FA580013B506220446432168206B46FFF700FED3
:10FA6800A0B19DF800209DF8013043EA02232380CD
:10FA78009DF802209DF8033043EA022363809DF835
:10FA880004209DF8053043EA0223A38002B010BD8C
:10FA980013B5062204463B2168206B46FFF7E0FDBC
:10FAA800A0B19DF800209DF8013043EA022323808D
:10FAB8009DF802209DF8033043EA022363809DF8F5
:10FAC80004209DF8053043EA0223A38002B010BD4C
:10FAD80013B501220DF107033A2104466820FFF708
:10FAE800BFFD0520FBF79EFF9DF8073003B10123FA
:10FAF800237002B010BD084B1B681869074B20F033
:10FB08001F0200F01F01D25801238B401A4201D076
:10FB1800FCF798BF704700BF800200201404014022
:10FB2800F0B52B4D2B7A85B0002B4ED1294C23688C
:10FB3800002B4AD01A68284E12B171690A437261C3
:10FB48009A88ADF80020022298688DF8032069464B
:10FB580000228DF80220FFF76DFCB3691D4F43F0BA
:10FB68000103B3612368187B197DFDF71BF8226830
:10FB7800936894881B8A1C4002D001232B7224E0CE
:10FB88001648FBF7FFFF3B681869FCF75BFF3B680B
:10FB98008DF80C401B69029308230DEB0300012626
:10FBA8008DF80D308DF80E6001F032FB3B688DF852
:10FBB80006405B7D8DF8043001A803238DF80530DD
:10FBC8008DF8076001F006FBD7E705B0F0BD00BF70
:10FBD800942500208002002000100240FFFA00084F
:10FBE80008B5FFF79DFF6B2180226820FFF7B4FD61
:10FBF8006420FBF722FF6B2103226820FFF7ACFD8E
:10FC08000F20FBF71AFF124B19211A786820FFF70B
:10FC1800A3FD0F20FBF711FF0E4B1A211A7868205D
:10FC2800FFF79AFD1B2118226820FFF795FD1C217C
:10FC380010226820FFF790FD372102226820FFF785
:10FC48008BFD682038210122BDE80840FFF784BDFC
:10FC5800B40200200000002008B5FFF761FF074B41
:10FC68001B7813B1012B03D008BD4FF4006201E0EB
:10FC78004FF48052024B1A8008BD00BF8402002056
:10FC8800200000202DE9F0410369C76805460E46AB
:10FC98001F40002F35D0B7FA87F24FF00043D3400A
:10FCA800DB432B611F40A2F11B03042BF1D8DFE8D3
:10FCB80003F0221F1C190300746A24B1013C0023BD
:10FCC800A4B2736201E0EC6AA4B2D6F82080B8F15D
:10FCD800000FDED0D8F80030404621469847D8F8C3
:10FCE8000480F4E73068696B07E07068A96B04E08A
:10FCF800B068E96B01E0F068296C036889B298473D
:10FD0800C7E7BDE8F08107B52320FBF796FE68201A
:10FD1800752101220DF10703FFF7A2FC28B19DF818
:10FD28000700A0F168035842584103B05DF804FB8E
:10FD380001480249A6E700BF00480140842000208E
:10FD4800014802499EE700BF0040014034200020DE
:10FD58000148024996E700BF000800400C20002037
:10FD6800014802498EE700BF00040040E41F00205C
:10FD78004FF08040004985E7BC1F002010B5054CB6
:10FD880005482146FFF77EFF04F1C8010348BDE896
:10FD9800104077E7941F0020002C014000440140E8
:10FDA800014802496EE700BF002C0140941F002063
:10FDB800224B10B5224C5A43224BB3FBF2F2038874
:10FDC8000139013AA04289B292B29BB20ED004F531
:10FDD8000064A0420AD0B0F1804F07D0A4F598344F
:10FDE800A04203D004F58064A04202D123F070033E
:10FDF8009BB2154CA04206D004F58064A0421CBFFB
:10FE080023F440739BB203800D4BC1629842028574
:10FE18000FD003F5006398420BD003F54063984276
:10FE280007D003F58063984203D003F580639842B6
:10FE380001D1002303860123436110BD40420F0016
:10FE4800002C014000A24A040010004073B505468A
:10FE58000068FFF7ADFF2A6813889BB243F00103DF
:10FE68001380EB7A8DF804300124002601A88DF860
:10FE780005408DF806608DF8074001F0ABF9EB7A84
:10FE88001B2B0BD1192301A88DF804308DF80540E0
:10FE98008DF806608DF8074001F09CF902B070BD3E
:10FEA800134B800A984220D00AD84A3B984212D075
:10FEB8000133984211D0B0F5801F14D1012070474A
:10FEC8000C4B98420BD0013398420AD0023B98421F
:10FED80009D104207047022070470320704705208D
:10FEE800704706207047FE2070470020704700BF0B
:10FEF8004B00100051001000F8B504680646204673
:10FF08000F461546FFF7CCFF06284BD8B27A910862
:10FF180047B902238B40D4F80CE0DB439BB203EAD9
:10FF28000E03E3600A23204A03FB001342F8237000
:10FF3800043342F8235015463FB1B17AE268890884
:10FF480002238B409BB21343E360282202FB00523A
:10FF58002032EFF31286502383F3128803B203EBA7
:10FF68008303DB0003F10C011C3329442B4451F8B3
:10FF7800047F17B117600A6804329942F7D1002349
:10FF88001360F3B283F31188282303FB0050036A3C
:10FF98001BB1E36843F0010303E0E2684FF6FE7328
:10FFA8001340E360F8BD00BF941F00200148F8F734
:10FFB8004DBD00BFA02500200148F8F747BD00BF90
:10FFC800F42500200148F8F741BD00BF482600206D
:10FFD80010B54B88DC0641BF2F4B14791B6853F8CA
:10FFE800244044BF2D4B43F820404B889B0641BF1B
:08FFF800294B54791B6853F8F2
:020000040801F1
:10000000244044BF274B43F820404B881C070ED5A3
:10001000254B0C781B78B3EB141FA1BF204BD47871
:100020001B6853F82440A4BF1E4B43F820404B8864
:100030009B070ED51D4B0C781B78B3EB141FDFBF4D
:10004000174B54781B6853F82440DCBF154B43F81A
:1000500020404B88DC070FD5154C0B78247803F033
:100060000F03A342DFBF0E4B14781B6853F82440E4
:10007000DCBF0C4B43F820404B885B070FD50B7857
:100080000C49097803F00F038B42A1BF044B92780F
:100090001B6853F82220A4BF024B43F8202010BD58
:1000A000B8240020AA0D00203F2400203D24002079
:1000B0003C2400203E240020254A264826490023CF
:1000C000F0B5156803700B701C461A462E19768819
:1000D0004EB92F5D3FB9037000230A704B7007784B
:1000E0001C461A460CE0360548BF013204F10404F0
:1000F00003F1010348BFD2B2802CDBB2E6D1EAE7BC
:10010000E0B2B8420CD215F8240006099E4200F075
:100110000F00A8BF731C9042A8BF421C0134EFE738
:100120008A704B70C2F3470102F001020A444C1E70
:100130000A490B480A70C3F3470203F00103134452
:1001400004700849501E084A08701370F0BD00BFC3
:10015000E0110020342400209C2600203E240020B2
:100160003C2400203F2400203D2400202DE9F04FB6
:10017000C24BDA682DED028B1A61C14A1168D96051
:10018000C0490B6843F020030B60BF4B197801296D
:1001900090460CBF002201221A70BC4B1A789107BE
:1001A00089B040F13D83BA490978042940F2388387
:1001B000B849097801F0040101F0FF0011B922F0FB
:1001C00001021A701B78DB0702D408B1F8F772F944
:1001D000B149CA78531C052293FBF2F202EB82026A
:1001E0009A1AAE4BCA701B78039392000023AC4C52
:1001F000DFF8CCC2DFF8D8925CF8231091FBF9F558
:1002000004F1080004F1100640F82350A54844F812
:10021000231000FB051142F2107091FBF0F080B248
:1002200026F813004FF0140E04F1140604F13C0AF2
:100230000EFB036E5AF823605EF802704EF802104F
:10024000F61B314444344AF82310052691FBF6F19D
:1002500009FB051144F82310039C012C4FEA830B82
:10026000E24605D10238B0F5797F98BF4BF80C1003
:100270000BB90123BBE7884CD8F80030226D9FED05
:100280008A7A8A4E8A4D9B1A07EE903AF8EE677A80
:10029000D8F800302365C7EE877A7C4B1B78B7EE21
:1002A000008AF4EEC87AF1EE10FA58BFF0EE487A00
:1002B00013F00103C4ED157A12D005AA00927D4B0C
:1002C00006AA01920CCB9AE80300F7F7F1FF64212C
:1002D000059A069BB2FBF1F293FBF1F3328000E04A
:1002E00033802B8094F858306B48002B3BD0D0EDF6
:1002F000157AC26DDAF80030C8EE276A9B1A026ED2
:10030000022507EE103AB8EEC77ADAF8043027EE85
:10031000267A9B1AFDEEC77AB0F9662017EE901A7E
:1003200007EE903A644BB8EEE77AD3ED007A67EEC9
:10033000277A67EEA67AFDEEE77A17EE903A02FA90
:1003400083F3B0F9642093FBF5F302FA81F29BB2D8
:1003500092FBF5F292B2A0F86A30A0F86820A0F8FB
:100360006630A0F86420012384F85830534BDAF843
:1003700004101B88DAF80000474D514E216603F047
:100380003003E065002B00F04B8205F1740300930D
:1003900005F178030193EA6E2B6FF7F789FF726816
:1003A0002B6F9B1A07EE903A434B326893ED007A1D
:1003B000EB6EF8EEE77A9B1AEB67384B67EE877ABD
:1003C0001B78FDEEE77A012BC5ED207A03D0022BD6
:1003D00000F0DF8024E2D5ED287A3A4BD5ED215AA2
:1003E00095ED255A95ED156A95ED264AD5ED274AE6
:1003F00035491D68B1EE677ABDEEC77AFDEEE77A42
:1004000017EE10EA17EE90CA0020304A91ED007AFC
:1004100052F8207007EE907AF8EEE77AA2F1140312
:1004200067EEA57A33F81060FDEEE77A283217EE12
:10043000903A9B1B9BB222F810301BB207EE903A09
:10044000F8EEE77A3B4467EE857A4400FDEEE77A02
:10045000CDED037A07EE903AF8EEE77ABDF80C801E
:1004600067EE847AA7EE867AFDEEC77A17EE902AB9
:10047000724531DB6245A8BF62462EE0A40700202A
:10048000202800200C1100207610002010110020E0
:10049000161100202A3400209C260020340F002052
:1004A000A0260020806967FF00007A448A1100209E
:1004B0008C1100207810002078000020D41100203A
:1004C00018110020380F0020680F00201827002086
:1004D00080969800DB0FC940724607EE902AF8EE2E
:1004E000E77A5FED046AC1ED007AFDEEE77A313616
:1004F00017EE903A43449AB2AB78D1ED027A07EE08
:10050000103AB8EE477A4B684F6027EE267AFB1A0E
:1005100088EE077AB6B2622E06EE903AF8EEE66AF8
:1005200037EE067AC6EE866A86EE077A76EEE76AD8
:10053000E7EE267AC1ED047AC1ED027A0FD964EEB6
:10054000A77ABA4EFDEEE77A17EE903AB3F5FA6F56
:10055000A8BF4FF4FA63B342B8BF334600E00023AC
:1005600013441BB240F6B8329342A8BF1346B04AB8
:100570009342B8BF1346AF4AA352AF4A142303FBBA
:10058000002351F8142B1A60002840F04981012003
:100590003BE7AA4BD5F874801F68D4F878903E8961
:1005A000DFEDA78A4FEA58039E4228BF1E46B5F8E2
:1005B000A8301AB29642C3BFD5ED157A9FEDA17A45
:1005C00067EE877AB6B2C1BFFDEEE77A17EE906AA2
:1005D000F618B6B2C8BFA5F8A860D4F8AC50C5EB01
:1005E00009052846F7F7A8FE0028D8BF404241F287
:1005F00093129042CCBF0020012088B307EE905A9E
:10060000B8EEE70A20EE280AFAF7A7FD07EE908A6F
:10061000F8EE677A40F6B83320EE270AFDEEC07A8E
:10062000CDED037ABDF80C20A4F8B02012B29A42A6
:10063000A8BF1A467E4B9A42ACBF09EB02034B445B
:1006400048F6A042934203DDA3F50C43A03B04E02F
:10065000002BBCBF03F50C43A033C4F8B43001E059
:10066000C4F8B490D4F8B450C5F50C53283307EE51
:10067000903AF8EEE77A67EEA88AB0EE680AFAF7E1
:10068000CFFD8DED070AB0EE680AFAF766FDD4EDEE
:10069000317AD4ED2E4AD4ED155A94ED2F4A94EDCB
:1006A000305A65498DED060AB1EE677ABDEEC77A1C
:1006B000FDEEE77A0DF1180E17EE10AA17EE90BABC
:1006C0000020614AFEEC016A32F91030DFF88C91AB
:1006D00007EE903A07EE106AF8EEE77AB8EEC77ABE
:1006E0003C32D6EE877A4FEA400CFDEEE77ACDED4C
:1006F000037ABDF90C30B3F57A7FA8BF4FF47A7353
:100700004B45B8BF4B461FFA83F922F810900FFAF9
:1007100089F207EE902AF8EEE77A27EEA47ABDEE8A
:10072000C77A8DED037A27EE847AD1ED007ABDF891
:100730000C90E7EE257AFDEEE77A17EE902A524507
:1007400003DB5A45A8BF5A4600E0524607EE902AFE
:10075000F8EEE77A9FED3D6AC1ED007ABA7891ED47
:10076000027A06EE902AF8EE666A4A684B6066EEF8
:10077000866A9A1AC8EE266A143106EE102AB8EE76
:10078000C66A76EEA56A86EE256AC5EEA66A36EEDC
:10079000476AA6EE867A01ED017A01ED037A25EE2D
:1007A000077ABDEEC77A17EE103ABDEEE77A4B44F2
:1007B00017EE102A13441BB240F6B8329342A8BF7A
:1007C00013461B4A9342B8BF13461A4A2CF802300C
:1007D0001F4A142303FB0023C3ED007A08B901204C
:1007E0006FE73B7923B1642395FBF3F5194B1D802B
:1007F0003B8898450DD9D4F8AC30A06FC01AF7F7F4
:100800009BFD80EAE072A2EBE07242F210739A4222
:1008100006DD114B01221A700E4BB4F8C8201A8065
:1008200009B0BDEC028BBDE8F08F00BF30F8FFFFD0
:1008300048F4FFFFBC0F0020900F0020380F00206D
:10084000D30237390000C84204270020DB0FC9401B
:10085000680F0020300F0020340F002018FCFFFF2D
:100860000846F5F779BE0F4B1A78692A16D15A88CF
:10087000B2F5FC6F12D11A79BE2A0FD193F8DD2799
:10088000EF2A4FF000000BD113F8012B5040064A1D
:100890009342F9D1B0FA80F04009704700207047C8
:1008A000704700BF00F80308E0FF03082DE9F04F90
:1008B000EB4C85B000214FF4FC62204605F0BBFBF9
:1008C000E84B04F53B721A60E74B00251D70E74BBF
:1008D00004F2B6721A606923237002200323637145
:1008E000FAF76AFD4FF48070FAF766FD4FF416735D
:1008F0002022A4F8663184F86A21FA236E22A4F833
:10090000683184F87C21BC230A22A4F8643184F87D
:100910007D214FF4FA732B22A4F86E3184F87F21E5
:100920000123212284F8623184F87E3184F8802109
:1009300084F886312322002384F88121C4F82032F0
:100940004FF4C872C4F824320523A4F8822184F835
:10095000B457A4F87251A4F87051A4F8745184F8F3
:10096000585184F8595184F85A51A4F85C51A4F8AC
:100970005E51A4F8605184F8635184F86B5184F897
:100980006C51A4F88451A4F8885184F81D5284F85D
:100990001C5284F8285284F82B3240F2DC53A4F81D
:1009A000983140F24C43A4F89A3140F26C73A4F8A9
:1009B0009C3140F27533A4F89E3140F64303A4F80D
:1009C000A03184F8295284F82A5284F8925184F88C
:1009D00093512A4623469918023200254FF01E09EA
:1009E000242A9F4C81F8A25181F8A391F3D14FF4AE
:1009F000FA6340F27E4040F27E57DFF868B2A4F816
:100A0000C831A4F8CC31A4F8D031A4F8D431A4F87A
:100A10004401052340F23A70A4F84C7140F2EA57C1
:100A200001264FF47A78C82219214FF0320A84F84F
:100A3000DE31A4F846014FF4C87340F2DC50A4F84C
:100A40004E7140F2B457A4F8E221039284F8DF110A
:100A50000191A4F8E631A4F84A01029084F8959136
:100A600084F8DD6184F8E06184F8E16184F8E46190
:100A700084F8EA61A4F8507184F8945184F896518E
:100A8000A4F8C681A4F8CA81A4F8CE81A4F8D281C2
:100A900084F8D65184F8DC5184F8E851A4F84881F0
:100AA000A4F852A1A4F8543184F8ED61A4F856A139
:100AB00084F8EB5184F8EC5184F8EE51FBF7EEFE2C
:100AC000DBF8003026744FF0170E83F815E083F83A
:100AD00016E04FF0550EE673A573A58183F803E089
:100AE0004FF00F0E83F805E00199D9714FF0220EF7
:100AF00083F806E021214FF00E0E83F80B9083F867
:100B00000C9083F810E059744FF0350E53214FF0DC
:100B1000640928274FF02D0C83F81AE0D9764FF09E
:100B20005A0E0A2183F81C904FF0780983F80DC003
:100B300083F808E0997483F80A901D705F709F70C5
:100B4000DD7583F804A09D731D76DD735D765F729D
:100B500083F814C04FF4FA7CA3F84EC0DFF820C12C
:100B6000C3F838C0C3F83CC0DFF818C1C3F828C0C8
:100B70004FF07E5CC3F834C0F7EE087ADFF80891D6
:100B8000DFF808C1C3ED087AC3F82C90C3ED097AE9
:100B9000C3F83090C3F848C0F1EE047A02989E770B
:100BA0004FF04B0C4FF0000983F8501083F852506F
:100BB00083F85170C3F84090C3ED117A83F84CC0AC
:100BC00084F8B6E7A4F8C0074FF0410E042084F87B
:100BD000B7E784F8B8A784F8B95784F8BD5784F804
:100BE000BE5784F8BA5784F8BB5784F8BC5783F8CB
:100BF0005C0015200191A3F85850A3F85A50A3F8AF
:100C00005650C3ED187A83F868001948D866194819
:100C100018671948586783F87860184883F8647033
:100C200083F86570FBF778FEDBF800300199039AD2
:100C300083F814614FF4487083F8115183F812510E
:100C400083F8137183F81851A3F816015E4684F8EF
:100C5000D81184F8D921A4F8DA81194618E000BF28
:100C6000202C002048100020602800207010002058
:100C70009A99193FF6287C3F3D0A773FFDB7010856
:100C80008FC2F53C00002040CDCCCC3E000040405F
:100C90000E2202FB05326FF0170082F819010320C3
:100CA00082F81A016FF02F0082F81B01072082F8EA
:100CB0001C016FF0230082F81D01052082F81E013F
:100CC00001355A2081F8200181F821016422FF209A
:100CD000082D81F81F2181F8220101F10E01D7D1E1
:100CE000002183F88911C821A3F88A11142183F8FF
:100CF0008C11A3F890211E214FF4967283F88D1168
:100D0000A3F8922101212822A3F8942183F88E11BF
:100D10002E4B03F1C0021F46C3F8149010339342C8
:100D2000FAD12B480021402205F085F90023294DF6
:100D3000264C5959FA1804330868C2F8AC02382B0B
:100D4000F5D104F50B700021802205F074F905F14E
:100D50003801702204F50B7005F062F9FFF7ACF969
:100D60004FF40020FAF728FB36680125314604F2DB
:100D700084404FF4CC7284F8DC5784F8DA5784F856
:100D8000DB5705F04DF904F21C6031464FF4CC728C
:100D900005F046F9104B1B681A68C4F8C2275A6858
:100DA000C4F8C6279A68C4F8CA271A68C4F8CE27B8
:100DB0005A68C4F8D2279A68C4F8D627022384F860
:100DC000D85484F8703605B0BDE8F08F202C002090
:100DD000CC2E0020D0960108701000201549D1F8C3
:100DE000883043F47003C1F88830134B1A6842F01E
:100DF00001021A605868114A02405A601A6822F0CB
:100E0000847222F480321A601A6822F480221A60F6
:100E10005A6822F4FE025A60DA6A22F00F02DA629D
:100E2000186B074A02401A6300229A604FF0006371
:100E30008B60704700ED00E0001002400CC07FF8AE
:100E4000CCFC00FF074B93F8DC37012B08D1064A96
:100E5000064BD0681B68834234BF002001207047D6
:100E600000207047202C00201000002028060020C1
:100E700038B5094B93F8DC5765B9084C2068F6F78C
:100E800028FD074B25601B78022B03D1BDE83840B5
:100E9000FBF7C3BC38BD00BF202C0020B0280020C9
:100EA000AC280020064B93F8DC371BB1012B05D191
:100EB000F7F786BC034B1868FAF77BBE0020704733
:100EC000202C0020B0280020F8B5011F0646002382
:100ED000083051F8042F02F120043F2C3BD802F1D6
:100EE00008040F2C06D80232032A04D9002B08BFAD
:100EF000012300E002238142EBD1012B30680ED0A8
:100F0000022B1AD0736803F003039B0000F0030068
:100F100043EA0010B36803F00303184317E000F03E
:100F20000F0040F04000F5F717FBB068736800F061
:100F30000F0040EA0310C0B209E000F03F0040F0AB
:100F40008000F5F709FB3079F5F706FB307ABDE84C
:100F5000F840F5F701BB06F10C0734463A46002588
:100F600052F8043D03F18001FF294FEA850510D9AD
:100F700003F50041B1F5803F02D245F0010508E0DC
:100F800003F50003B3F1807F34BF45F0020545F05F
:100F90000305B242E4D165F03F00C0B2F5F7DCFAD8
:100FA00005F00303022B207807D0032B0CD0012B74
:100FB00013D1F5F7D1FA60780FE0F5F7CDFA607844
:100FC000F5F7CAFAA07808E0F5F7C6FA6078F5F701
:100FD000C3FAA078F5F7C0FAE0780434F5F7BCFA64
:100FE000BC424FEAA505DBD1F8BD10B50446C0B23E
:100FF000F5F7B2FAC4F30720BDE81040F5F7ACBA34
:1010000010B504467F2C06D964F07F00C0B2F5F716
:10101000A3FAE409F6E7E0B2BDE81040F5F79CBAA0
:10102000430083EAE070EBE72DE9F047304B93F89B
:10103000DC37012B86B0074601D004464AE005F0B4
:101040003EF803A9054606466846F7F7C9FA039B2A
:10105000049A029713442B443F2B059519D900237A
:10106000684603A90322F7F7E7FA039B3BB9049B01
:101070002BB9204A13705370059BABB301E0F7F70F
:1010800097FA039B049A059E134433447F2B2BD875
:10109000029FDFF86090CA4639461AF8024BC4F145
:1010A0008008B04528BFB0460AEB04004444E4B2CF
:1010B000424604F0B5FF802C89F8004014D1C8EBFB
:1010C0000606504607EB0801324604F0A9FF89F8EE
:1010D000006009E0254614F8011B21B1064B186891
:1010E000FAF773FDF6E7ED1B284606B0BDE8F0877A
:1010F000202C002068270020B02800200FB407B55E
:1011000004AB064953F8042B01930020F9F7F4FED1
:1011100003B05DF804EB04B0704700BF610801083C
:1011200040F2E9330F4A1289920704D4013B9BB283
:10113000002BF7D10BE00C4A40F2E933107009495B
:101140000989C9070AD4013B9BB2002BF7D1074A92
:10115000138801339BB21380FF2070471078C0B210
:10116000704700BF003800400C380040EC270020DA
:1011700030B5174B9B894FF47A733AB311B10D78A0
:10118000013107E0FF2505E0013B9BB24FF6FF74FC
:10119000A3420FD00E4C2489A407F5D50D4C257021
:1011A0000B4D2D89ED070BD4013B9BB24FF6FF751C
:1011B000AB42F5D1084A138801339BB2138005E096
:1011C000247808B104700130013AD6E7012030BD1F
:1011D000003800400C380040EC2700200C4B0D4933
:1011E000DA684378D243C2F30222C2F10402934088
:1011F00002781B010A44DBB282F800330378012233
:10120000580903F01F0302FA03F341F82030704736
:1012100000ED00E000E100E0036823F01F0202F1AE
:10122000804202F5823270B503F01F011468012379
:1012300003FA01F124EA0101116002682A4C22F04C
:101240001F0502F01F02295903FA02F221EA0202E5
:101250002A510279016802F1804221F01F0402F54F
:10126000823201F01F01155903FA01F1294311518E
:1012700002681E4D22F01F0402F01F02615903FA9A
:1012800002F221EA020262510268194C22F01F06A2
:1012900002F01F02315903FA02F221EA02024179F7
:1012A00032511029026812D122F01F0102F01F02F0
:1012B0004E5903FA02F232434A51026822F01F01EA
:1012C00002F01F020859934003430B5170BD01F116
:1012D000804122F01F0001F5823102F01F020C58FC
:1012E000934023430B5070BD0404014008040140A7
:1012F0000C040140F0B5BE4CA3782DED028B013BF0
:10130000012B85B000F26F81E578854240F06B815A
:101310002379022B00F06781B64B5B5D6371A37983
:101320006D00F2EE048A1BB16319B3F9083009E0CD
:101330006319D4ED037AB3F90830F1EE677AC4ED9E
:10134000037A5B4208EE103A2369A94EB8EEC88AC8
:101350001A0388EE288A35D5D6ED037AFDEEE77AB2
:1013600028EE280A17EE903AD6ED057A8DF80A3065
:10137000FDEEE77A17EE903A8DF80B3005F0B0F8F5
:10138000FCEEC07A96ED060A17EE903A20EE280A97
:10139000ADF8083005F0A4F8FCEEC07A96ED070A27
:1013A00017EE903A20EE280AADF80C3005F098F8C8
:1013B000FCEEC07A0C2017EE903A02A9ADF80E3080
:1013C000F5F7BAF9D4ED077A894BF5EE407AF1EEEC
:1013D00010FA60D1D3ED067AB4EEE78AF1EE10FA96
:1013E00004DDDA6883ED068A5A61E8E0F5EEC07A3A
:1013F000F1EE10FA40F3E38093F8202042B1022A84
:1014000000F2DD805A6B83ED078AFA329A63D6E0E8
:10141000D3ED037A38EE678AF7EE007AB4EEE78A06
:10142000F1EE10FAACBF01210021D3ED0A7A69B1C7
:101430009FED717A27EE877ADFED707AB4EEE77A66
:10144000F1EE10FA58BFF0EE477A03E09FED6C7AA8
:1014500067EE877AC3ED0A7A2369654A1B0311D5C3
:101460008DF808105379116B0B440B205A788DF8C6
:101470000920DA7A8DF80A205B7D8DF80B3002A9FD
:10148000F5F75AF90123226B84F82030637913446D
:101490000022DA7291E0B4EEE78AF1EE10FA48BF6A
:1014A00083ED078AA16B636B94ED067AD4ED076A2E
:1014B000591AC943C90F77EE667A59B9B7EE006A6F
:1014C000F4EEC67AF1EE10FA79DDB4EEE68AF1EECA
:1014D00010FA74DDD4ED056A454BB4EEE67AF1EE10
:1014E00010FACCBF0126002666B1D3ED097A9FED34
:1014F000427A67EE877A9FED427AC3ED097AD3ED9F
:101500000B7A0AE0B0EE007AF4EEC77AF1EE10FA48
:1015100008DDD3ED0B7A9FED387A67EE877AC3ED5D
:101520000B7A07E0D3ED097A9FED357A67EE877A7B
:10153000C3ED097AD4ED097A206B627967EEA87A57
:101540001044FCEEE77ACDED017A9DF8043043704B
:10155000D4ED0B7A2769FCEEE77A3F03CDED017AF3
:101560009DF8042042750ED546EA41018DF8081019
:101570008DF80930C37A8DF80A300B2002A98DF856
:101580000B20F5F7D9F894F82020194B022A11D135
:10159000D3ED0A7A9FED1B7A196B67EE877A0022EA
:1015A00083F82020FCEEE77A5A7917EE903A0A4445
:1015B000D37202E0022283F82020F6F7E7FFA27937
:1015C0000B4B0AB1104A00E0104ADA602544D4ED12
:1015D000037AB5F9083000EE103AB8EEC00A80EE92
:1015E000280A37EEC00A05B0BDEC028BF0BD00BF83
:1015F000EC270020A8970108EC51783F6F12833A3E
:101600000AD7833F00007A440000A0410000A0C137
:101610002B4BF0B52B4D1E6805F110002F78F319F8
:101620002C46597801F00401013501F0FF0219B18F
:101630008542F3D10020F0BD224D631B022B0ADD51
:101640001AB102EB82025200D2B215F8013B303BD4
:101650001A44D2B2F1E70021AC420AD919B101EB28
:1016600081014900C9B215F8013B303B1944C9B2A8
:10167000F2E72E2F16D101340420002325787719A4
:1016800003EB83037F785B007F079BB244BF303D51
:101690005B1900F1FF3044BF01349BB210F0FF0032
:1016A000ECD100E0002308484143642000FB031311
:1016B0000620B3FBF0F3054800FB0230F0BD00BF8D
:1016C000900000202828002040420F0080969800BB
:1016D00030B500231A4610498C1894F83C40BCB130
:1016E0002E2C06D1013298B18C180444002584F8C0
:1016F0003C5011440A2491F83C106343A1F130049A
:10170000092C9CBF303B5B180E2A03D80132E2E75C
:10171000184630BD002030BDEC270020104B10B51E
:101720000446185CF9F779F90E4800EB4400B0F96B
:101730004C10B1F57A7F05DBB1F5FA6FA8BF4FF415
:10174000FA6101E04FF47A71A1F57A710A23092058
:1017500091FBF3F1BDE81040C9B2FCF763BA00BFDA
:1017600006B80108EC270020031EB8BF2D2210B5D3
:10177000B8BF58420C46B8BF01F8012B0A22F9F74E
:10178000A7FB00230370204610BD00BF07B5064B22
:101790000093064B01930649064A074B0748F9F7A1
:1017A000ADFC03B05DF804FBB4A7010889A70108EC
:1017B00095AE01088EAE0108A8A701081BB8010864
:1017C00008B5037833B90C4B0C481978BDE80840CC
:1017D000F9F794BC04F0CAFC02280CD8064B187028
:1017E000074B0C2202FB0030064B06301860F9F75D
:1017F000ABFE0548E5E708BD602800203BB80108BE
:10180000D033002070100020ABAA010808B503787F
:101810003BB90B4B0B4893F8B417BDE80840F9F7F8
:101820006DBC04F0A3FC022808D8054B83F8B4076C
:10183000F9F7F4FDF9F7ACFE0348E8E708BD00BF8F
:10184000202C00203FB80108ABAA010838B5037866
:1018500003BB214B1B6801330F2B07D81F490C22F8
:1018600002FB03121C4695682DBB00E01C460134A8
:101870000F2C01DD002400E005D818490C2202FBE2
:1018800004129568BDB99C42F1D11548BDE83840B5
:10189000F9F734BC04F06AFC0F28044605D80F4A57
:1018A0000C2303FB00239D682DB921460D48BDE89C
:1018B0003840F9F723BC084B1C60FAF7E7F82146DB
:1018C0002A460948F9F71AFC0C235C43034B185DC0
:1018D000BDE83840FAF7EEB87C000020AC9701086C
:1018E0004CB8010862B801087AB8010873B50378EA
:1018F00013B9F5F7A5FB3DE01F4901AA04F097FCD9
:10190000002401462646254699B134B1012C08D160
:10191000084604F02BFC064603E0084604F026FCCB
:1019200005461549002001AA04F081FC0134014656
:10193000EAE70B2D02D911480C220BE0022C10D142
:10194000A6F57A73B3F57A7F07D90D484FF47A710B
:101950004FF4FA62F5F7F1FA0CE00A4B03EB45039A
:101960005E80084B084803EB45032946B3F9022083
:10197000F9F7C4FB02B070BD41B1010824AD010804
:10198000EDB401086028002091B8010838B50D4C6D
:1019900023688342054606D1F5F79BFF20460021C8
:1019A0004C2204F048FBE36CAB4209D12846F5F722
:1019B00090FF054800214C22BDE8384004F03BBBB5
:1019C00038BD00BF70220020BC220020034B1A68E3
:1019D000D379591C1344D171187A7047B41100207F
:1019E00010B5FFF7F3FF84B2FFF7F0FF04EB002020
:1019F00080B210BD10B5FFF7F3FF0446FFF7F0FF0C
:101A000004EB004010BD064B10B504462146186893
:101A1000FAF7DBF8034B1B6898796040987110BDAA
:101A2000B8110020B4110020014B1B689879EAE737
:101A3000B411002038B5044624200D46FFF7E3FF1B
:101A40004D20FFF7E0FF002C084C14BF21203E2062
:101A5000FFF7D9FF2368002228469A71FFF7D3FFCA
:101A6000236893F84900BDE83840CCE7B411002062
:101A700001460020DEE710B50446C0B2FFF7C3FF01
:101A8000200ABDE81040BEE710B5044680B2FFF75B
:101A9000F2FF200CBDE81040EDE737B5828883687F
:101AA000044610060D4641BF2B4991F8B4174FF478
:101AB000CC7000FB0133D10544BF2849097802F0FE
:101AC0003F0244BF01EB410103EB8103042A12D022
:101AD00006D8012A0DD0022A32D193F9001030E045
:101AE000102A0AD0202A0AD0082A29D1B3F90010D6
:101AF00027E0197825E0198823E0196821E093EDA3
:101B0000000A6846F9F77AF901461548F9F7F6FA36
:101B100005B3D4ED037A6846B8EEE70AF9F76EF933
:101B200001461048F9F7EAFA94ED040A6846B8EE5F
:101B3000C00AF9F763F901460A48F9F7DFFA09E044
:101B400000210948F9F7DAFA25B10848E168226965
:101B5000F9F7D4FA03B030BD202C00206028002013
:101B6000C9AF0108C2AF01086DAF0108A0B80108F4
:101B7000024B0146D869FAF728B800BF6028002058
:101B800010B5441E14F8011F21B1034BD869FAF7B0
:101B90001CF8F7E710BD00BF6028002010B50378DF
:101BA0001BB90A48BDE81040EAE704F0DFFA044632
:101BB000082899BF2146064806480821F9F79EFAE9
:101BC000601E40B2BDE81040F5F706BEA7B8010898
:101BD000EEB801081AB90108F7B52B492B4B087864
:101BE0002B4D1C682B4B05EB80001A882A4BD0F834
:101BF000C0101B78294800914FF47A71B4FBF1F1C1
